:020000040800F2
:10000000A8950124FD0300082137010879030108A0
:1000100019370108193F0008497A0108000000005B
:10002000000000000000000000000000B13D0108D9
:10003000695B00080000000071390108D146010821
:100040001B0400081B0400081B0400081B04000814
:100050001B0400081B0400081B0400081B04000804
:100060001B0400081B0400081B04000819540008A6
:10007000295400083954000849540008595400080C
:10008000695400081B0400081B040008C95B000831
:10009000E95B0008D95B0008F95B00081B04000855
:1000A0001B0400081B0400081B0400081B040008B4
:1000B0001B0400081B0400081B0400081B040008A4
:1000C0001B0400081B0400081B0400081B04000894
:1000D000293C0108097401082974010839740108D0
:1000E000715B00081B040008000000001B040008EE
:1000F0001B0400081B0400081B0400081B04000864
:100100001B0400081B0400081B0400081B04000853
:100110001B040008F15201081B0400081B0400081E
:100120001B0400081B0400081B0400081B04000833
:100130001B0400081B0400081B0400081B04000823
:1001400000000000000000000000000000000000AF
:100150001B0400081B0400081B0400081B04000803
:100160001B0400081B0400081B0400081B040008F3
:100170001B0400081B0400081B040008000000000A
:100180001B0400081B040008115301081B0400088D
:100190001B0400081B0400081B0400081B040008C3
:1001A0001B0400081B0400081B04000800000000DA
:1001B0001B0400081B0400081B0400081B040008A3
:1001C0001B0400081B0400080000000000000000E1
:1001D00000000000000000001B04000800000000F8
:1001E000000000000000000000000000000000000F
:1001F00000000000000000001B0400081B040008B1
:100200001B0400081B040008000000001B04000879
:100210001B0400081B0400081B0400081B04000842
:100220001B040008000000001B0400080000000080
:100230001B0400081B04000800000000311800081F
:100240001B040008492300081B0400081B040008C5
:100250001B0400081B0400081B0400081B04000802
:100260001B0400081B0400081B0400081B040008F2
:100270001B0400081B0400081B0400080000000009
:100280001B0400081B0400081B0400081B040008D2
:10029000000000001B0400081B0400080000000010
:1002A000000000001B0400081B0400081B040008D9
:1002B000F97301081B0400081B040008095C00080E
:1002C000195C0008B14801081B04000800F002F89E
:1002D00000F084F80AA090E8000C82448344AAF15C
:1002E0000107DA4501D100F079F8AFF2090EBAE85A
:1002F0000F0013F0010F18BFFB1A43F0010318475A
:1003000000E3010020E301000A444FF0000C10F864
:10031000013B13F0070408BF10F8014B1D1108BF83
:1003200010F8015B641E05D010F8016B641E01F823
:10033000016BF9D113F0080F1EBF10F8014BAD1C73
:100340000C1B09D16D1E58BF01F801CBFAD505E091
:1003500014F8016B01F8016B6D1EF9D59142D6D3EB
:10036000704700000023002400250026103A28BF13
:1003700078C1FBD8520728BF30C148BF0B60704717
:10038000692900F06B81642900F06881752900F00B
:1003900065816F2900F0FC81782900F023820368D1
:1003A000DB0928BF41F08001632900F0E286732950
:1003B00000F0E786E32900F0F286002070471FB5C1
:1003C0001DF010FC00F0C6FF0400002000211DF00D
:1003D000CDFA401C60601FBD10B510BD01F0EFF9F3
:1003E0001146FFF7ECFF18F0D3FB01F00DFA03B450
:1003F000FFF7F2FF03BC01F011FA00000A48804742
:100400000A4880470A480047FEE7FEE7FEE7FEE7A6
:10041000FEE7FEE7FEE7FEE7FEE7FEE705480649E2
:10042000064A074B70470000995B0008D94701084E
:10043000CD020008A8650124A8950124A87501240F
:10044000A875012453EA020C00F069802DE9F04BF5
:100450004FF00006002B1FBFB3FA83F503FA05F433
:1004600024FA05F65E4012BF1643B2FA82F502FA8C
:1004700005F4C5F120051EBF22FA05FC44EA0C0470
:10048000203556EA044C4FEA144418BF641C4FF060
:1004900000084FF00009904271EB030C39D300299A
:1004A00019BFB1FA81F701FA07F6B0FA80F700FA3E
:1004B00007F6C7F120071EBF20FA07FC46EA0C0624
:1004C0002037B6FBF4FCA7EB0507103F07F01F0B26
:1004D000CBF120062CFA06F60CFA0BFB44BFB34610
:1004E0000026202FA4BF5E464FF0000B5BEA060CEF
:1004F00008BF4FF0010B19EB0B0948EB0608ABFBEB
:10050000027C06FB02CC0BFB03CCC01B71EB0C0185
:10051000C1E70B46024641464846BDE8F08B13B59D
:10052000084318BF4FF0FF300146AFF30080BDE82D
:100530001C4070470FB41CB5084B06AA7B446946A3
:100540000090059800F0EBFD04460020694600F09D
:10055000F9FD20461CBC5DF814FB0000050C0000F2
:100560000FB47CB50C0009AA009001D02044401EB5
:10057000084B7B4469460190089800F0D0FD054681
:100580001CB10020694600F0DDFD28467CBC5DF80A
:1005900014FB0000D90B000070B5044685690068A3
:1005A000C10601D5302600E02026C00707D070BD67
:1005B000D4E9012130469047206A401C20626D1E1C
:1005C000F6D570BD70B5044685690078C00707D1BF
:1005D00070BDD4E9012120209047206A401C206290
:1005E0006D1EF6D570BD09684A0501D540B2704749
:1005F000C905FCD500B2704709684A0501D5C0B2EB
:100600007047C905FCD580B2704770B50C460546E9
:10061000012A05D02878800600D5EA69002302E087
:10062000012305E05B1C934202D2E05C0028F9D173
:10063000A869E618C01AA861286A184428622846E2
:10064000FFF7AAFF04E0D5E9012114F8010B904758
:10065000B442F8D32846FFF7B5FF70BD2DE9F0414D
:100660000646002410687529314616A510D0FFF7FC
:10067000BAFF002802DA404213A507E031688A0772
:1006800001D512A502E0490704D511A5012401E016
:10069000FFF7B2FF00210A2206F1240709E0B0FBB0
:1006A000F2FCB0FBF2F302FB1C0030307854184629
:1006B000491C0028F3D123462A463046BDE8F041C4
:1006C00000F0CFBC000000002D0000002B00000057
:1006D000200000002DE9FF5F15468A460446DFF83A
:1006E000AC80F8440027D8E900103E46CDE9001060
:1006F00010E03AF816106A4602A800F0D9FD411C35
:1007000007D02178890603D5E269391891420DD8BE
:100710000744761C2078800602D5E069B84205DDE2
:10072000AE42E6DB3AF816000028E2D1A069C01B11
:10073000A0612046FFF730FFD8E90010CDE9001096
:10074000002017E03AF818106A4602A800F0B0FD41
:10075000B0F1FF3F81460BD000250DF1080B05E0FD
:10076000D4E901211BF8050090476D1C4D45F7D3D6
:1007700008F10100B0428046E4DB206A3844206280
:100780002046FFF71FFFBDE8FF9F00001AD50100BC
:1007900070B5044621461068FFF72EFF002104F1D2
:1007A000240505E000F007023032C0086A54491CF5
:1007B0000028F7D12068002308A2050708D500F01B
:1007C0002000084304D0E069012305A2401EE06137
:1007D0002046BDE8704000F044BC0000000000006E
:1007E0003000000070B504460D4621461068FFF742
:1007F00003FF2188090502D50F4A7A4402E00E4A18
:100800007A440E32002104F1240305E000F00F06C3
:100810000009965D5E54491C0028F7D1207800231A
:10082000000704D5702D02D009B1022311322046F1
:10083000BDE8704000F015BC0AD401002DE9F05F5E
:10084000894604464FF0000ADFF874B1FB44C0F853
:1008500020A02046E1688847002874D0252806D0CB
:10086000D4E901219047206A401C2062F1E700266C
:100870005F462046E16888472028054607DB312D82
:1008800005D2781910F8200C08B10643F1E7B0073B
:1008900001D526F00406C4F81CA00027C4F818A04F
:1008A0002A2D09D028461DF027F838B304EB870815
:1008B000303DC8F8185019E059F8041B204604EBE5
:1008C00087029161E1688847012F054618D1E069E8
:1008D000002820DA26F020061DE0D8F8180000EBEA
:1008E000800005EB40003038C8F818002046E16869
:1008F000884705461DF000F80028EED1012F0AD0E8
:100900002E2D08D12046E16888477F1C0546022F1E
:1009100046F02006C4DBA069002803DA404246F016
:100920000106A061F00701D026F010066C2D0BD057
:10093000682D09D04C2D39D06A2D35D0742D35D085
:100940007A2D33D016E038E0E1682F4620468847FC
:10095000B842054609D16C2F26D04FF48060E1687B
:10096000064320468847054604E06C2F1AD04FF412
:10097000807006430DB3A5F14100192802D8203537
:1009800046F400664A462946204626604E46FFF752
:10099000F7FC80B101280BD0F61D26F0070000F10E
:1009A000080956E74020E4E78020D8E70020D6E792
:1009B00006F104094DE7284652E7206ABDE8F09F9A
:1009C000E0D301000FB400B58DB010A909900091DB
:1009D0000B904FF0FF300A9000200C9006487844AE
:1009E0000690064878446A4607900F9909A800F0D7
:1009F000F7FB0DB05DF814FB1F080000370800007E
:100A00002DE9FF5F1D464FF0FF3B91464FF0000878
:100A10005F46D5E90146A96901987F1C8847296A84
:100A2000824688470028F6D1BAF1FF3F0CD0002E4D
:100A300024F4C06419DD600614D5BAF12B0F09D077
:100A4000BAF12D0F0ED103E0584604B0BDE8F09F77
:100A500044F48064A96901987F1C8847761E824609
:100A6000002E02DDBAF1300F03D0B9F1000F26D00D
:100A700032E0A969761E01987F1C44F4007488470F
:100A8000002E824605DDBAF1780F06D0BAF1580F74
:100A900003D0B9F1000F10D01EE0B9F1000F02D061
:100AA000B9F1100F18D1A969761E01987F1C24F4A2
:100AB000007488478246102002E0082000E00A20E7
:100AC000814609E0A96908FB0908761E01987F1C88
:100AD00044F4007488478246002E05DD494650469E
:100AE00000F069FB0028EDDAE96901988847A00564
:100AF00002D46FF00100A8E7E00725D1600613D506
:100B0000600502D5C8F1000000E0404629680A1DD2
:100B10002A600968220501D5087015E0220701D571
:100B2000088011E008600FE02868011D2960006856
:100B3000210502D580F8008006E0210702D5A0F843
:100B4000008001E0C0F8008038467EE72DE9FF5FB5
:100B50004FF000089946144646469169D2E901A72C
:100B6000DDF838B001988847054659EA0B0005D0F2
:100B700009E0A1690198761C88470546216A284644
:100B800088470028F5D1681C03D05FEACA7005D0F9
:100B900015E04FF0FF3004B0BDE8F09F2068011D64
:100BA0002160D0F800800AE05FEACA7001D108F83D
:100BB000015BA169761C01987F1E88470546002FBE
:100BC0001ADD681C18D0B9F1000F0DD0E81705EB3D
:100BD000D060421120F01F0059F822102A1A01207B
:100BE00090400142E0D107E0BBF1000FDCD1284684
:100BF000216A88470028D7D0E16901988847BBF16E
:100C0000000F07D1002E05DD5FEACA7002D1002176
:100C100088F80010A068B84203DDBBF1000F03D0D4
:100C200017B16FF00100B6E73046B4E770B506467D
:100C300000F008FA0468054630460A22002100F058
:100C4000FFFA2C6070BD0000014A00F055BB0000A7
:100C50000000002440EA010310B59B070FD1042ACD
:100C60000DD310C808C9121F9C42F8D020BA19BA77
:100C7000884201D9012010BD4FF0FF3010BD1AB1DC
:100C8000D30703D0521C07E0002010BD10F8013B31
:100C900011F8014B1B1B07D110F8013B11F8014B58
:100CA0001B1B01D1921EF1D1184610BD40EA010371
:100CB000024630B59B0710D14FF0013400E008C266
:100CC00008C91D1B9D4315EAC41FF8D013F0FF018E
:100CD00002F8011B0DD01B0AF8E711F8013B002BAD
:100CE00002F8013B05D011F8013B002B02F8013B53
:100CF000F3D130BD10B5431C02E010F8011B71B1F7
:100D00008107FAD14FF0013202C88C1A8C4314EAE1
:100D1000C211F9D0C01A0A0603D0C01E10BDC01AF5
:100D200010BD0A0401D0801E10BD0902FCD0401E77
:100D300010BD40EA010370B59B072ED14FF001367C
:100D4000042A2AD308C810C99D1B9D43121F15EA07
:100D5000C61517D0D8B2E1B2401A50EA056110D1D9
:100D600098B2A1B2401A50EA05410AD123F07F405F
:100D700024F07F41401A50EA052102D1180EA0EB61
:100D8000146070BDA342DBD018BA21BA884201D9E1
:100D9000012070BD4FF0FF3070BD0AB9002070BD5A
:100DA00010F8013B11F8014B63B1A3420AD1521E66
:100DB00008D010F8013B11F8014B1BB1A34201D13F
:100DC000521EEDD1181B70BD032A40F2308010F086
:100DD000030C00F0158011F8013BBCF1020F6244D6
:100DE00098BF11F801CB00F8013B38BF11F8013B67
:100DF000A2F1040298BF00F801CB38BF00F8013B14
:100E000011F0030300F02580083AC0F0088051F883
:100E1000043B083A51F804CBA0E80810F5E7121D8E
:100E20005CBF51F8043B40F8043BAFF30080D207AD
:100E300024BF11F8013B11F801CB48BF11F8012B79
:100E400024BF00F8013B00F801CB48BF00F8012B9C
:100E5000704710B5203AC0F00B80B1E81850A0E8F8
:100E60001850B1E81850A0E81850203ABFF4F5AF78
:100E70005FEA027C24BFB1E81850A0E8185044BFD4
:100E800018C918C0BDE810405FEA827C24BF51F841
:100E9000043B40F8043B08BF7047D20728BF31F835
:100EA000023B48BF11F8012B28BF20F8023B48BF86
:100EB00000F8012B704702F0FF0343EA032242EAE5
:100EC000024200F00AB802F0FF0343EA032242EABA
:100ED000024200F024B84FF000020429C0F0128052
:100EE00010F0030C00F01B80CCF1040CBCF1020FDD
:100EF00018BF00F8012BA8BF20F8022BA1EB0C01B2
:100F000000F00DB85FEAC17C24BF00F8012B00F8A7
:100F1000012B48BF00F8012B70474FF0000200B5CD
:100F2000134694469646203922BFA0E80C50A0E80C
:100F30000C50B1F12001BFF4F7AF090728BFA0E8BA
:100F40000C5048BF0CC05DF804EB890028BF40F886
:100F5000042B08BF704748BF20F8022B11F0804FC8
:100F600018BF00F8012B704710B5044610F0030FAE
:100F700008BF11F0030F40F015804FF0013E121F23
:100F8000C0F20E8051F8043BA3EB0E0C2CEA030CCC
:100F90001CEACE1C08BF40F8043BF0D0A1F10401CC
:100FA00002F10402521E08DB11F8013B00F8013B7C
:100FB000002BF7D11146FFF78EFF204610BD000031
:100FC00030B44FF0013C50F8042BCCFA52F451F8F5
:100FD000043BD51A20D1FCB950F8042BCCFA52F4BA
:100FE00051F8043BD51A17D1B4B950F8042BCCFAF8
:100FF00052F451F8043BD51A0ED16CB950F8042BB9
:10100000CCFA52F451F8043BD51A05D1002CDAD0B1
:1010100030BC4FF00000704729BAB1FA81F111F0ED
:101020001801D1F120008440F2D1CA40CB4012F027
:10103000FF0213F0FF0330BCD01A704770477047AF
:101040007047000000487047B010002410B5FFF74B
:10105000F9FF006810BD10B50446FFF7F3FF046008
:1010600010BD2DE9F0470D4699469246044600F121
:1010700024080168880604D5E06921F01001216088
:1010800000E00120A84201DD471B00E00027A16924
:101090007A1902EB0900081AA0612078C00602D470
:1010A0002046FFF779FA002608E0D4E901211AF872
:1010B00006009047206A401C761C20624E45F4DBF7
:1010C0002078C0060AD52046FFF766FA06E0D4E984
:1010D000012130209047206A401C2062381EA7F171
:1010E0000107F4DC07E0D4E9012118F80500904776
:1010F000206A401C2062281EA5F10105F3DC204671
:10110000FFF760FA2078000602D50220BDE8F087DC
:101110000120FBE701694A1C02610878704700B5AD
:101120008FB0CDE901310021059105497944CDE920
:10113000031011466846FFF781FB0FB000BD0000A9
:10114000E5FFFFFF0A6802F8010B0A607047D1E96A
:1011500000239A4202D2531C0B601070704710B5E6
:10116000436913B1AFF3008001E0FFF74EFA0120AD
:1011700010BD127800F124010A7000224A70012289
:10118000EDE711684FF0FF32E9E710B5436913B19D
:10119000AFF3008001E0FFF79DFA012010BD128837
:1011A00000F1240182840022C2840122EDE711684B
:1011B0004FF0FF32E9E73A2800D2303820F0200221
:1011C000412A01D3A2F13700884201D34FF0FF300A
:1011D0007047000002681144137801601846704798
:1011E000D160054979445161044979441162002173
:1011F0001161114600F0BCB8EDFFFFFF6F01000068
:10120000426842B1016811F8013B23B1521EC0E9A6
:101210000012184670470121C160881E704742685D
:101220005AB1C368016843B983688B4205D0491E2F
:10123000521CC0E90012002070474FF0FF30704789
:101240002DE9F04791460F4680460446002614F8E3
:10125000015B2DB100F076F80068405DC007F6D163
:101260002B2D02D02D2D18D0641E4A46394620461B
:1012700000F038FA27B13968A14201D1C7F80080DF
:101280004FF0020471050BD54042002803DDFFF743
:10129000D9FE0460A007BDE8F08746F48066E4E765
:1012A0000028F8DAFFF7CEFE04606FF00040F2E7A6
:1012B0002DE9F04116460C46054600F043F8036858
:1012C00093F80101012807D0FF2C12D8185D80B1D6
:1012D00001202C70BDE8F081D3F807013246214689
:1012E00003F20713C7182846BC46BDE8F0410023A7
:1012F00060474FF0FF30EDE72DE9F04115460E460F
:10130000040002D12C6804B90BA4204600F049FA6D
:101310000444207870B127463146384600F031FA4F
:101320000444207810B1002004F8010B38462C60EA
:10133000BDE8F0810027F9E7000000000048704791
:10134000B010002410B500F005F8001D10BD00BF5E
:101350001DC6010000487047D010002410B5044697
:10136000FFF7F0FF0068005D00F0010010BD000015
:101370002DE9F34F4FF0000A0C4656468DB0012080
:101380000C9001F10C000B9062690B9801219047C1
:10139000051E2DD0252D2CD0216A8847C0B1626949
:1013A0000B9801219047216A88470028F7D162698C
:1013B000411E0B98904700E0761CA1690D98884764
:1013C000216A88470028F7D1E1690D988847DBE753
:1013D000A1690D988847A842074601D1761CD3E73A
:1013E000E1690D9888477F1C02D1BAF1000F6FD0D8
:1013F0006BE162690B9800273D46394690472A28E1
:1014000004D162690B98012190470125DFF8D08251
:1014100062690B9801219047A0F130010A290AD294
:101420004745E5DC07EB870100EB4107303FDFD4A0
:1014300045F01005ECE7E90601D46FF000476C2891
:101440000AD04C2814D0682815D06A280DD07428EA
:101450001CD07A281AD01DE062690B9801219047B0
:101460006C2802D045F0040514E045F002050DE0BB
:1014700045F020050AE062690B9801219047682831
:1014800002D045F0080505E045F4006562690B9857
:1014900001219047C4E9015765283DD019DC58283F
:1014A0007AD00CDC452837D004DC252826D041280A
:1014B0009ED131E046282FD0472899D12CE05B28D7
:1014C00077D0612828D063287CD0642823D15AE0C3
:1014D000F6E06F2848D008DC66281DD067281BD0AE
:1014E000692821D06E2816D127E0702845D07328AE
:1014F00068D0752847D078280DD14DE0A1690D98A6
:101500008847252805463FF469AFE1690D9888476B
:101510006D1C3FF46AAFD8E00D9923466A466FF020
:101520000100AFF30080C5E045F0400023464FF0D6
:1015300000026060A80736D43EE0E8077FF447AFBA
:101540002068011D21600068290501D506701BE790
:10155000290701D5068017E7A90703D5F117C0E9C8
:10156000006111E706600FE745F0400023464FF0A9
:1015700008026060A80716D41EE040F60E0125EAB6
:101580000100606016E045F0400023464FF00A027B
:101590006060A80707D40FE045F040006060A8072E
:1015A00008D5234610220D996FF00100AFF300809B
:1015B00080E007E0102223460D996FF00100FFF74D
:1015C0001FFA77E04FF0000963284F46C8464B46A4
:1015D000CB4602D05B2806D038E0E80601D40120D3
:1015E000A060012732E06269D4F80CB00B980121A9
:1015F00090475E2807D14FF0010949466269D4F847
:101600000CB00B989047216939B900210A4603AB09
:1016100043F82120491C0829FADBD8B3216949B3D2
:1016200008F1010862690B98012190475D28F4D107
:10163000B9F1000F09D0002003A951F82020D243AE
:1016400041F82020401C0828F7DB03AB2069002864
:1016500020794FEA40701ED05B462246CDF80080CC
:10166000CDE901970D9900286FF0010020DAAFF362
:1016700000801FE0C11703AA00EBD1614B1121F0DC
:101680001F0102EB8302411A1368012088400343C3
:101690001360C7E719E00D99224600286FF001009A
:1016A000009702DAAFF3008004E0FFF74FFA01E0A1
:1016B000AFF3008000280ADA401C06D10C9820B154
:1016C0004FF0FF300FB0BDE8F08F5046FAE7E90762
:1016D00001D10AF1010A064400200C9054E60000F2
:1016E000CCCCCC0C2DE9F05F824615468B4600270A
:1016F0000AF10104B9460078302801D09DB113E009
:1017000014F8010B0127782803D0582801D045B1DF
:101710000AE00DB1102D07D1002714F8010B102598
:1017200002E0082500E00A250026B0460EE005FB91
:10173000080005FB06F101271FFA80F801EB1046AF
:10174000B6F5803F00D3B94614F8010B2946FFF7E0
:1017500032FD0028EBDABBF1000F05D00FB1641E9B
:1017600000E05446CBF80040B9F1000F06D0FFF777
:1017700069FC02210160C81EBDE8F09F48EA0640EE
:10178000FAE730B503461D781DB10A4603E0AC42C6
:1017900001D1181A30BD12F8014B002CF7D15B1C97
:1017A000F1E730B503461D783DB10A4612F8014B0A
:1017B0001CB1AC42FAD15B1CF5E7181A30BD754676
:1017C000FFF7BCFDAE4605006946534620F0070012
:1017D000854618B020B5FEF721FEBDE820404FF049
:1017E00000064FF000074FF000084FF0000BAC462A
:1017F000ACE8C009ACE8C009ACE8C009ACE8C00975
:1018000021F007018D46704710B50446AFF3008004
:101810002046BDE81040FEF7EABD0000014918204F
:10182000ABBEFEE72600020070470000000000008B
:1018300041F60870C2F2004005F086BB00000000CF
:1018400010B50446006842F2001140F48070C4F202
:101850000201884218D142F20830C4F20200006846
:1018600010F4403F18D00AF0F7FF6168B1F5803FEF
:1018700005D0B1F5403F2BD0B1F5003F29D1090C7F
:10188000B0FBF1F025E000BF46F20830C5F60200DB
:10189000006810F4403FE6D14FF40020002109F029
:1018A000DBFE6168A1F580224FEAB2420A2A10D815
:1018B000DFE802F00606060606063C3E404244000B
:1018C0006FF0010202EA5141B0FBF1F001E000BF0C
:1018D00080084BF62141C0F2BE01884206D820683C
:1018E000816821F44071816010BD00BF47F641015D
:1018F000C0F27D11884207D820680122816862F316
:101900000921816010BD00BF21684FF28102C0F241
:10191000FA229042886805D8022262F30920886082
:1019200010BD00BF40F44070886010BD0009D0E7D2
:101930004009CEE78009CCE7C009CAE7000AC8E73A
:10194000B0B52DED028B044600284FF0FF005FD0AC
:101950000D4600295CD095ED020A95ED032A20EE94
:10196000001A95ED013A20EE020A95ED002AB7EE35
:10197000008A03EE031A02EE030A31EE011A30EE7A
:10198000000A78EE410A1BF093F995ED002A95EDD7
:10199000014A95ED023A95ED035A22EE031A84EDC1
:1019A000010A05EE441A31EE011AB0EEC16AB4EE36
:1019B000486AF1EE10FA0FDAB0EE410A1AF012FF9F
:1019C00095ED002A95ED014A95ED023A95ED035A01
:1019D00084ED020A09E000BF11EE100A40F6DB7147
:1019E000C3F6C97161F31E00A06023EE030A24EE62
:1019F000031A05EE050A02EE051A30EE002A31EE52
:101A0000010A78EE420A1BF053F9002084ED000A27
:101A100040B2BDEC028BB0BDB0B500286ED0B7EEC1
:101A2000001A04460D46002981EE000A80ED040AE2
:101A30004FF07E5020604FF00000C4E90100E060EC
:101A400059D095ED010A95ED001AB7EEC00AB7EE30
:101A5000C11A1BF049F895ED001AB5EE401AF1EEE7
:101A600010FA0DD195ED011AB5EE401AF1EE10FA0B
:101A700006D195ED021AB5EE401AF1EE10FA41D0FA
:101A8000B7EEC00B9FED351AB4EE410AF1EE10FA35
:101A90004CDCB5EE400AF1EE10FA47DB9FED302A40
:101AA000B4EE420AF1EE10FA2CDCB4EE410AF1EE8B
:101AB00010FA27DB9FED2B1AB4EE410AF1EE10FA73
:101AC00004DCB4EE420AF1EE10FA43DA40F2C560EB
:101AD00044F62D21C3F64D70C3F60D4120604AF245
:101AE0005640616044F2AD71CBF63930C3F61971DE
:101AF000C4E90201002040B2B0BD00BFFF2040B2E7
:101B0000B0BD00BF40F2C56044F62D21C3F64D7054
:101B1000C3F60D4120604AF25640616044F2AD7157
:101B2000CBF63930C3F6197112E000BF45F66E10DE
:101B300045F20C31C3F67F70C3F6B011206048F651
:101B4000AB00616049F28551CBF6BB30C3F69751CB
:101B5000C4E90201002040B2B0BD00BFDB0FC9BF25
:101B6000DB0F49C00000B4C200218160C0E9001150
:101B70007047000000000000B0B52DED108B8EB056
:101B8000044600284FF0FF0003D0002918BF002AA8
:101B900004D140B20EB0BDEC108BB0BD40F21805C0
:101BA0004EF69E70C2F20045002BC3F62750286007
:101BB00000F0D28193ED009A93ED01AAB5EE409A20
:101BC00093ED028AF1EE10FA04BFB5EE40AAF1EEF1
:101BD00010FA00F0BB8192ED000A94ED011A92ED2B
:101BE000016A92ED027A94ED004A21EE405A60EECD
:101BF000040A94ED022A66EE041A94ED033A67EEA5
:101C0000042AD1ED004A06EE425AF5EE404A47EE6C
:101C1000020A47EE411A46EE012A07EE435A46EE03
:101C2000430AB6EE006A40EE031A40EE422A91EDF6
:101C3000010AF1EE10FA65EE063A91ED025A60EEF5
:101C4000860A21EE867A22EE866A04BFB5EE400A45
:101C5000F1EE10FA00F088818DED080A20EE000AFE
:101C60008DED0D6A8DED0C7A04EEA40ACDED0B3AE4
:101C7000CDED0A0A8DED095A05EE050ACDED074AAC
:101C80000EF07EFB2AEE0A1A8DED060A09EE091AFD
:101C900008EE081AB0EE410A0EF072FB94ED00CA8D
:101CA00029EE00FA7CEE0CBA94ED03BA6AEE008AD3
:101CB00094ED013A28EE00EAD4ED029A2FEE2B0AB9
:101CC0002CEE0C8A8DED010A68EEABAA20EE0B0A11
:101CD0002FEE081A2EEE2B2A08EE880A73EE03EA7E
:101CE0000AEECB1A03EE420A6FEE2ECA02EE291A52
:101CF00023EE034A09EEAC0A8DED034A28EEAE2A24
:101D00000FEE041A08EEC40A69EEA9FA39EEA99A90
:101D100009EE821A08EEAF0A2EEE2E2A2EEE094A9E
:101D20002BEE0BDA02EE0B1A0BEE040A2CEE03AAD2
:101D30000FEE6F1A08EECD0A63EE0BDA0FEE4D1AB6
:101D400020EE000A01EE010A23EE291A8DED021A97
:101D50003BEE0B1A8DED051A2CEE291A8DED041AA7
:101D60000EF00EFB94ED011A94ED022A2AEE813A50
:101D70009DED014ADDED031A28EE897A3DEEAD5A5C
:101D8000DDED070A04EE423A94ED034A3AEE0A6AA0
:101D9000F6EE004A0BEEE95ADDED047A0EEE083A53
:101DA000F0EE616A09EE0B6ADDED02AA7DEEE72A2C
:101DB0009DED058A0CEE843A09EE8BAA4CEE4BAAF7
:101DC0000EEE613A07EE043A9DED067A00EEC75A30
:101DD000DDED080A00EEC76AF0EE473A0EEE6F3A04
:101DE000B7EE007A71EEA10A74EEEF1A0EEE0D3A1C
:101DF00087EE000A37EE607A7FEEAF0A28EE05BA6A
:101E000028EE068A37EE607A71EECD0A62EE831A0A
:101E1000DDED092A02EEE37A6AEE032A40EE201A8B
:101E2000F1EE000A0BEEC58A40EE2A2A61EE203A56
:101E300062EE200A0BEE86BA2EEE86AA00EEC78A64
:101E400074EEE60AF8EE004A2EEE85CA07EE63BA93
:101E500070EEEF0A09EE45AA09EE06CA31EECF5A36
:101E600032EEE86A62EE031A61EE032A60EE043A8B
:101E700037EEAD7A60EE830A01EEC5AA72EEE35A40
:101E800060EE244A40EE070A94ED007A05EE86AA39
:101E900044EE842A24EE034A60EE025A67EE036A97
:101EA00033EE033A20EE077A75EEA67A52EE246AF4
:101EB00041EE433A04EE05BA71EEC71A02EE437AD8
:101EC00030EECE2A20EE011A07EE86BA06EE858A9B
:101ED00031EE040A03EE82BA02EE85CA00EE068AEB
:101EE00005EE82AA01EE86CA07EE028A2BEE0B0AE5
:101EF00001EE02CA0AEE0A0A08EE080A0CEE0C0A03
:101F00000EF03EFA20EE0A1ADDED0A0A20EE0B2A48
:101F1000DDED0B3A20EE083A9DED0C7A20EE0C0A2E
:101F20009DED0D6A95ED004A44EE413A94ED011A9B
:101F300044EE420A94ED022A04EE437A94ED033A09
:101F400004EE406A94ED004A14E000BFB5EE408A0A
:101F5000F1EE10FA7FF43FAE20460EB0BDEC108BD0
:101F6000BDE8B04000F040B8B5EE405AF1EE10FACE
:101F70007FF472AE94ED045A00EE851A03EE854AA2
:101F800007EE052A06EE053A84ED011A84ED004AB3
:101F900021EE010A84ED022A84ED033A04EE040ADC
:101FA00002EE020A03EE030A0EF0EAF994ED001ABB
:101FB00094ED012A94ED023A94ED034A20EE011AC1
:101FC000002020EE022A84ED001A20EE031A84ED90
:101FD000012A20EE040A84ED021A84ED030A40B2BD
:101FE0000EB0BDEC108BB0BDB0B52DED108B04461E
:101FF00000284FF0FF0003D0002918BF002A03D1AA
:1020000040B2BDEC108BB0BD40F2180542F6023074
:10201000C2F20045C3F6075094ED011A92ED016A31
:10202000286092ED027A92ED000A94ED003A21EEDA
:10203000405A94ED022A60EE030A94ED034A66EEDC
:10204000031A91ED00EA67EE032AB5EE40EA06EEC8
:10205000425A91ED01DA47EE020A91ED02CA47EECB
:10206000411A46EE012A07EE445A46EE440AB6EEFD
:10207000006A40EE041A40EE422AF1EE10FA04BF64
:10208000B5EE40DAF1EE10FA25EE06AA20EE86BA99
:1020900021EE869A22EE868A00F090802DEE0D0ABF
:1020A0000EEE0E0A0CEE0C0A0EF06AF9B1EE001AF2
:1020B00094ED013A94ED034A94ED007A24EE046A1B
:1020C000D4ED023A23EE015A67EE071A2EEE002AEB
:1020D00074EE040A65EE062A61EE811A77EE074A6D
:1020E00042EE602A61EEA35A63EE816A43EE212A32
:1020F0006DEE001A42EE245A2CEE000A41EEE42A5C
:1021000046EE865A33EEA36A27EE017A41EEE05A94
:10211000F2EE000A22EE06DA32EEC5CA63EEA32A18
:1021200063EE204A63EE037A07EE22DA63EEA00A3A
:1021300004EEA7CA07EE27DA35EEE6EA04EEA2CAF5
:1021400027EE817A07EEA0EA33EE033A27EE04FA8F
:1021500000EE05CA00EEA2EA02EE43FA22EE811A70
:1021600001EEC3DA00EE26EA04EE01FA2CEE0C0AC8
:1021700001EEC6FA0DEE0D0A0EEE0E0A0FEE0F0A74
:102180000EF0FEF820EE0D1A95ED004A20EE0C2A16
:1021900020EE0E3A20EE0F0A04EE41AA94ED011A49
:1021A00004EE42BA94ED022A04EE439A94ED003A0A
:1021B00004EE408A94ED034A06E000BFB5EE40CA43
:1021C000F1EE10FA7FF46AAF94ED045A0BEE051AA3
:1021D0000AEE053A09EE052A08EE054A84ED011AD1
:1021E00084ED003A21EE010A84ED022A84ED034ACF
:1021F00003EE030A02EE020A04EE040A0EF0C0F82F
:1022000094ED001A94ED012A94ED023A94ED034AFC
:1022100020EE011A002020EE022A84ED001A20EEA2
:10222000031A84ED012A20EE040A84ED021A84EDDB
:10223000030A40B2BDEC108BB0BD000000000000EE
:10224000A0B1B0B504460D4600F09AFB48212046E7
:10225000FEF741FE287803226988A56400F090FC0F
:102260000020BDE8B04040B2704700BFFE2040B241
:102270007047000000000000002908BF704770B5DB
:1022800096B00C46816C01AA002308780026498884
:1022900000F01AFB20B116B0BDE87040704700BFD7
:1022A0009DF812009DF814209DF813109DF815302C
:1022B0009DF817509FED1C1A090341EA00510006D2
:1022C0009DF8160041EA021103F00F0241EA1311D2
:1022D0004FEA004048BF01F1704140EA02609DF8BA
:1022E000182040EA052000EE101A1044190748BFD4
:1022F00000F17040B8EEC00A02EE100A9DF811001D
:10230000207080EE010AB8EEC22A84ED010AC4E909
:102310000366C4E9056682EE010A84ED020A16B07E
:10232000BDE87040704700BF8096184B0000000069
:10233000B1EE601A80FE602AB4EE401AF1EE10FA97
:1023400031FE020A7047000041F6F070C2F2004010
:1023500005F05EBD0000000041F260200821C2F2DD
:102360000040406816F0C0BE10B50320002101F007
:102370007BFA41F260249220C2F200440122002341
:1023800004F8010F0020214601F06AFBE11D002046
:102390001322012301F03CFB002010BD00000000CF
:1023A000022001214FF0FF3216F0E2BE00000000D3
:1023B0009FED010A704700BF0000C8430000000005
:1023C00041F260201021C2F20040406816F08CBE3D
:1023D00010B50720002101F047FA41F26024822065
:1023E000C2F200440122002304F8010F002021461C
:1023F00001F036FB04F10E0100200622012301F05A
:1024000007FB002010BD0000042001214FF0FF3227
:1024100016F0AEBE000000002DE9F04100284FF09C
:10242000FE0700F08F810E46002900F08B8141F2FB
:1024300060280546C2F2004898F8000020B1FD2748
:1024400078B2BDE8F08100BF16F046FF0028C8F85A
:10245000040000F07F8144464BF27E60EE6224F877
:10246000010F012001F014FB0320002101F0FCF911
:10247000002002220023214601F0F2FA032001216C
:1024800001F0F2F94BF214602080012001F000FB12
:102490000720002101F0E8F9002002220023214654
:1024A00001F0DEFA0720012101F0DEF91E2001F023
:1024B000EFFA012001F0ECFA0320002101F0D4F939
:1024C0009E202070002001220023214601F0C8FA3E
:1024D000002002220023214601F09AFA0320012164
:1024E00001F0C2F9012001F0D3FA0320002101F02C
:1024F000BBF900200122002321468026267001F02E
:10250000AFFA002002220023214601F081FA0320C5
:10251000012101F0A9F960781E2840F017810120FF
:10252000012501F0B5FA0720002101F09DF944468C
:1025300000200122002304F8016F214601F090FAE7
:10254000002002220023214601F062FA0720012127
:1025500001F08AF920780F2840F0F8800A2001F075
:10256000EBF80B2001F0E8F842F669020020C0F613
:1025700000020121002701F063FA42F259310A20DA
:10258000C0F6000101F018F942F2C1310B20C0F68B
:10259000000101F011F944464AF6402024F8010FE9
:1025A000012001F075FA0320002101F05DF90020FF
:1025B00002220023214601F053FA0320012101F0F9
:1025C00053F940F241102080012001F061FA03200C
:1025D000002101F049F9002002220023214601F0E8
:1025E0003FFA0320012101F03FF940F6530020801B
:1025F000012001F04DFA0320002101F035F90020FF
:1026000002220023214601F02BFA0320012101F0D0
:102610002BF94FF48B602080012001F039FA032060
:10262000002101F021F9002002220023214601F0BF
:1026300017FA0320012101F017F940F27D402080B4
:10264000012001F025FA0320002101F00DF90020FE
:1026500002220023214601F003FA0320012101F0A8
:1026600003F9322001F014FA40F20F10208001200B
:1026700001F00EFA0720002101F0F6F800200222F6
:102680000023214601F0ECF90720012101F0ECF8CC
:102690004FF444702080012001F0FAF90720002156
:1026A00001F0E2F8002002220023214601F0D8F9CF
:1026B0000720012101F0D8F816202080012001F028
:1026C000E7F90720002101F0CFF8002002220023C3
:1026D000214601F0C5F90720012101F0C5F84FF4AA
:1026E0008C702080012001F0D3F90720002101F037
:1026F000BBF8002002220023214601F0B1F9072097
:10270000012101F0B1F848F215002080012001F00C
:10271000BFF90720002101F0A7F8002002220023C2
:10272000214601F09DF90720012101F09DF80A20C2
:1027300001F0AEF90A2088F8005001F011F80B20E2
:1027400001F00EF878B2BDE8F08100BFFC2778B246
:10275000BDE8F081FE2778B2BDE8F08100000000FE
:1027600000283FD041F260219FED203AC2F20041A3
:10277000B1F90920B1F90DC0B1F90B3000EE102A02
:1027800002EE10CA01EE103A4FF60003CFF6FF73C7
:10279000B8EEC00AB8EEC11AB8EEC22A80EE030A3B
:1027A00081EE031A80ED040A82EE030A80ED051A19
:1027B00080ED060AB4EE001A4A7EB3EE072A897E3F
:1027C000D20042EA51120021B1EB922F18BF1A43F6
:1027D00000EE102AB8EEC00A00EE012A80ED0A2AA7
:1027E00048B27047FE2148B2704700BF00A0AA451A
:1027F00090B341F260219FED1A3AC2F200419FED81
:10280000194AB1F90F20B1F91130B1F9131000EEE6
:10281000102A01EE103A02EE101AC16AB8EEC00A90
:1028200091ED015AB8EEC11AB8EEC22A80EE030A41
:1028300081EE031A82EE032A91ED003A10EE043A7B
:1028400091ED020A11EE045A12EE040A80ED073AE5
:1028500080ED085A80ED090A6FF00100704700BF53
:102860006F12034235FA8E3C10B5032000F08CFF46
:1028700041F26024C2F2004438B90320012100F083
:10288000F3FF6068022116F02FFC072000F07CFFA8
:10289000002818BF10BD0720012100F0E5FF606887
:1028A0000421BDE8104016F01FBC0000000000002D
:1028B000182001214FF0FF3216F05ABC0000000032
:1028C00070470000000000002DE9F04141F2F014D3
:1028D000C2F200442778012F0ED1154682B10E4670
:1028E0000746A0686421984616F06AFB60B1FB2099
:1028F00040B2BDE8F08100BFFD2040B2BDE8F081EC
:10290000FE2040B2BDE8F081E06800E0006978B3E5
:102910000178B94202D14168B14217D0006938B399
:102920000178B94202D14168B1420FD00069F8B1D3
:102930000178B94202D14168B14207D00069B8B10B
:102940000178B942E2D14168B142DFD18668A0681E
:1029500016F0A2FB7EB1002230462946434616F00F
:1029600033FA002818BF4FF0FF3040B2BDE8F081C5
:10297000A06816F091FBFC2040B2BDE8F081000099
:102980002DE9F04F89B041F2F017C2F200473878D4
:1029900020B1FD2040B209B0BDE8F08F07F1100072
:1029A0006021FEF7BAFA43F6081041F60811C2F2A8
:1029B000004041F60C120024C0F8804CC0F8844C52
:1029C000445042F29051845042F294524450845008
:1029D00042F6C100C0F600007860002016F01CFB33
:1029E0000028B86000F0C68042F2C02501AEC2F2F5
:1029F000004541F21009284631464FF0010A87F898
:102A000000A0CDE901444FF0020BC0F20209CDE96C
:102A100003BACDE90544079406F006FC2846314682
:102A2000CDF808A04FF08048CDF80480CDE903BA76
:102A3000CDE90544079406F0F7FB002100220023AE
:102A40002846009406F038FCA9F10F010022284620
:102A500006F026FB3878012809D142F69140C0F6ED
:102A60000000F86143F2C150C0F60000386142F244
:102A7000C020C2F2004007F097FA42F2603501AE82
:102A8000C2F20045314628460024CDE90144CDE993
:102A900003BBCDE90544079406F0C6FB01A8314607
:102AA000CDE904B480E8000D2846CDE9064406F0DF
:102AB000BBFB0121012200232846009406F0FCFB09
:102AC00000222846494606F0EBFA387843F2190A04
:102AD000C0F6000A012806D143F2C150C7F844A04D
:102AE000C0F60000386342F26030C2F2004007F0E6
:102AF0005BFA42F200450DF10408C2F2004541467E
:102B000028460226CDE90144CDE90366CDE9054416
:102B1000079406F089FB012002904FF0804001905D
:102B200028464146CDE90366CDE90544079406F001
:102B30007BFB0121012200232846009406F0BCFB08
:102B400000222846494606F0ABFA3878012806D11B
:102B500043F2C150C7F864A0C0F60000386542F2E5
:102B60000040C2F2004007F01FFA002040B209B056
:102B7000BDE8F08FFF2040B209B0BDE8F08F000043
:102B80002DE9F04141F2F018C2F2004898F8003007
:102B9000012B0FD114460D460646002A08BF0A2411
:102BA000D8F80800642116F00BFA38B1FB2040B2C7
:102BB000BDE8F081FD2040B2BDE8F081D8F80C00FE
:102BC00001E000BF0069F8B10178B14202D141686B
:102BD000A94240D00069B8B10178B14202D1416840
:102BE000A94238D0006978B10178B14202D1416878
:102BF000A94230D0006938B10178B142E2D14168D0
:102C0000A942DFD127E000BF142000F045FEB8B193
:102C1000074654210022204616F01EF9B860B8B1CC
:102C2000D8F80C003861D8F808003E707D603C731D
:102C3000C8F80C7016F030FA002040B2BDE8F08100
:102C4000D8F8080016F028FAFE2040B2BDE8F0815E
:102C5000384600F06DFDD8F8080016F01DFAFF2088
:102C600040B2BDE8F081000041F2F011C2F2004133
:102C70000A78012A04D138B14860002040B2704778
:102C8000FD2040B2704700BFFE2040B270470000F8
:102C90002DE9F04FAFB06846402100F10D0942F236
:102CA000C020C2F2004006F04FFB41F2F0180028AD
:102CB000C2F2004800F0868042F2C0260DF1940A6C
:102CC000C2F200460DF1540B06E000BF4021304631
:102CD00006F03AFB002875D04021304652465B464C
:102CE00006F03EFB00286DD126986FF06041002869
:102CF0004FF0020708BF40F2FF71259AB0F1804FF4
:102D000001EA020500F14041B1FA81F0279B08BFBA
:102D10000327D8F80420B3F1005F18BF47092846FD
:102D200012B1284639469047D8F80C1001E000BF90
:102D300009690029CAD00A7812B94A68824218D0B3
:102D400009690029C2D00A7812B94A68824210D0B3
:102D500009690029BAD00A7812B94A68824208D0B3
:102D600009690029B2D00A78002AE1D14A68824272
:102D7000DED18C68002CA9D028998DF80070CDE99F
:102D800001504EF2880001F00F01C0F601006F46BD
:102D9000455C0F398DF80C5007EB050000F10D0074
:102DA00018BFC5F14001FEF796F8484659462A4635
:102DB000FEF70AF8002200232046394616F098F85C
:102DC00084E700BF42F260304021C2F2004006F0CA
:102DD000BBFA002800F0888042F260360DF1940AB8
:102DE000C2F200460DF1540B06E000BF4021304610
:102DF00006F0AAFA002877D04021304652465B46BA
:102E000006F0AEFA00286FD126986FF060410028D6
:102E10004FF0020708BF40F2FF71259AB0F1804FD2
:102E200001EA020500F14041B1FA81F0279B08BF99
:102E30000327D8F80420B3F1005F18BF47092846DC
:102E400012B1284639469047D8F80C1001E000BF6F
:102E500009690029CAD00A78012A02D14A68824247
:102E60001AD009690029C1D00A78012A02D14A681A
:102E7000824211D009690029B8D00A78012A02D10A
:102E80004A68824208D009690029AFD00A78012A2D
:102E9000DED14A688242DBD18C68002CA6D028990A
:102EA0008DF80070CDE901504EF2880001F00F015D
:102EB000C0F601006F46455C0F398DF80C5007EBEA
:102EC000050000F10D0018BFC5F14001FEF703F841
:102ED000484659462A46FDF777FF00220023204640
:102EE000394616F005F881E742F200404021C2F26F
:102EF000004006F029FA002800F0888042F20046DF
:102F00000DF1940AC2F200460DF1540B06E000BF29
:102F10004021304606F018FA002877D0402130468C
:102F200052465B4606F01CFA00286FD126986FF0D7
:102F3000604100284FF0020708BF40F2FF71259A58
:102F4000B0F1804F01EA020500F14041B1FA81F091
:102F5000279B08BF0327D8F80420B3F1005F18BFF0
:102F60004709284612B1284639469047D8F80C1030
:102F700001E000BF09690029CAD00A78022A02D1FB
:102F80004A6882421AD009690029C1D00A78022A07
:102F900002D14A68824211D009690029B8D00A7862
:102FA000022A02D14A68824208D009690029AFD0BA
:102FB0000A78022ADED14A688242DBD18C68002C72
:102FC000A6D028998DF80070CDE901504EF2880006
:102FD00001F00F01C0F601006F46455C0F398DF816
:102FE0000C5007EB050000F10D0018BFC5F14001C2
:102FF000FDF771FF484659462A46FDF7E5FE0022D7
:1030000000232046394615F073FF81E72FB0BDE855
:10301000F08F0000000000002DE9F04FAFB06846CF
:10302000412100F10D0942F2C020C2F2004006F039
:103030008BF941F2F0180028C2F2004800F08680B7
:1030400042F2C0260DF1940AC2F200460DF1540B73
:1030500006E000BF4121304606F076F9002875D021
:103060004121304652465B4606F07AF900286DD180
:1030700026986FF0604100284FF0020708BF40F229
:10308000FF71259AB0F1804F01EA020500F140413D
:10309000B1FA81F0279B08BF0327D8F80420B3F1C9
:1030A000005F18BF4709284612B1284639469047A5
:1030B000D8F80C1001E000BF09690029CAD00A78CD
:1030C00012B94A68824218D009690029C2D00A7828
:1030D00012B94A68824210D009690029BAD00A7828
:1030E00012B94A68824208D009690029B2D00A7828
:1030F000002AE1D14A688242DED18C68002CA9D036
:1031000028998DF80070CDE901504EF2880001F049
:103110000F01C0F601006F46455C0F398DF80C5069
:1031200007EB050000F10D0018BFC5F14001FDF7E8
:10313000D2FE484659462A46FDF746FE00220023A5
:103140002046394615F0D4FE84E700BF42F26030D5
:103150004121C2F2004006F0F7F8002800F0888014
:1031600042F260360DF1940AC2F200460DF1540BA2
:1031700006E000BF4121304606F0E6F8002877D08F
:103180004121304652465B4606F0EAF800286FD1EE
:1031900026986FF0604100284FF0020708BF40F208
:1031A000FF71259AB0F1804F01EA020500F140411C
:1031B000B1FA81F0279B08BF0327D8F80420B3F1A8
:1031C000005F18BF4709284612B128463946904784
:1031D000D8F80C1001E000BF09690029CAD00A78AC
:1031E000012A02D14A6882421AD009690029C1D055
:1031F0000A78012A02D14A68824211D0096900295D
:10320000B8D00A78012A02D14A68824208D00969F6
:103210000029AFD00A78012ADED14A688242DBD188
:103220008C68002CA6D028998DF80070CDE901504B
:103230004EF2880001F00F01C0F601006F46455CB8
:103240000F398DF80C5007EB050000F10D0018BF89
:10325000C5F14001FDF73FFE484659462A46FDF7B5
:10326000B3FD002200232046394615F041FE81E7D8
:1032700042F200404121C2F2004006F065F8002809
:1032800000F0888042F200460DF1940AC2F2004636
:103290000DF1540B06E000BF4121304606F054F812
:1032A000002877D04121304652465B4606F058F858
:1032B00000286FD126986FF0604100284FF0020778
:1032C00008BF40F2FF71259AB0F1804F01EA020574
:1032D00000F14041B1FA81F0279B08BF0327D8F8DD
:1032E0000420B3F1005F18BF4709284612B12846F1
:1032F00039469047D8F80C1001E000BF0969002951
:10330000CAD00A78022A02D14A6882421AD00969D0
:103310000029C1D00A78022A02D14A68824211D01B
:1033200009690029B8D00A78022A02D14A68824283
:1033300008D009690029AFD00A78022ADED14A688C
:103340008242DBD18C68002CA6D028998DF80070C1
:10335000CDE901504EF2880001F00F01C0F60100E6
:103360006F46455C0F398DF80C5007EB050000F1F6
:103370000D0018BFC5F14001FDF7ADFD48465946A7
:103380002A46FDF721FD002200232046394615F08C
:10339000AFFD81E72FB0BDE8F08F00000000000016
:1033A0002DE9F0479AB041F2F017C2F200473F789A
:1033B000012F0FD10446022817D801F0FE001D4648
:1033C00017460E4602280BD055B9FE2040B21AB05F
:1033D000BDE8F087FD2040B21AB0BDE8F08700BF1D
:1033E000DDF888A0BAF1400F04D9FF2040B21AB02E
:1033F000BDE8F0870DF1040864214046FDF78DFD1E
:10340000032EF2D860B24DF68452C0F6010252F893
:103410002090DFE806F0030D071100BF019700219F
:1034200000200EE001974FF00050002109E000BF9E
:103430000197002003E000BF4FF0005001974FF0CC
:1034400080410390D9F808000291B0F5407F07D081
:10345000B0F5807F0AD14FF40010002108E000BFD2
:103460004FF400104FF4801102E000BF0021002053
:10347000CDE90610002005904FF400000890BAF145
:10348000090F4FF001000990504622D3BAF10D0FF9
:1034900002D209201DE000BFBAF1110F02D20A20AA
:1034A00017E000BFBAF1150F02D20B2011E000BFE8
:1034B000BAF1190F02D20C200BE000BFBAF1210FB4
:1034C00002D20D2005E000BF0F20BAF1310F38BF46
:1034D0000E2008F12407049038465146FDF71DFDE3
:1034E000002D18BFBAF1000F04D1484606F08CF841
:1034F00048B90EE0384629465246FDF765FC484675
:1035000006F082F828B101A948463A4605F010FEB7
:1035100030B343F6081040F68841C2F2004014FB75
:103520000102D2F8803CD2F8846C013303F01F050D
:10353000B5420CD002F5486714FB010064213A68DB
:1035400002FB010001A96422FDF783FC3D6000201D
:10355000B54208BF4FF0FF3040B21AB0BDE8F08767
:10356000002040B21AB0BDE8F08700000000000063
:1035700061B180B582B091F804C00A684B1D012189
:10358000CDF800C0FFF70CFF02B080BD6FF0010066
:10359000704700000000000061B180B582B091F872
:1035A00004C00A684B1D0021CDF800C0FFF7F8FEEB
:1035B00002B080BD6FF00100704700000000000005
:1035C0002DE9F04FA3B0684642F2C02500F124086F
:1035D000C2F2004519AE00BF2846314605F0B4FFDF
:1035E0000028F9D043F6081742F2C025C2F200477E
:1035F000C2F2004564246E46D7F8800CD7F8841CCC
:10360000884220D0284605F0FFFF00281EBFD7F8CB
:10361000800CD7F8841C884215D0D7F8840C64221B
:1036200000FB04713046FDF714FCD7F8840C3146DA
:103630000130424600F01F00C7F8840C284605F010
:1036400077FD0028D8D042F2603519AEC2F20045AD
:103650002846314605F078FF0028F9D042F260355F
:1036600041F6081441F60C16C2F200454FF0640A08
:10367000E9463859B95988421DD0284605F0C4FF9B
:1036800000281EBF3859B959884214D0B85964224D
:1036900000FB0A7000F688414846FDF7DAFBB8598E
:1036A00049460130424600F01F00B851284605F057
:1036B0003FFD0028DDD042F2004519AEC2F20045C0
:1036C0002846314605F040FF0028F9D042F2004973
:1036D00042F2905442F29455C2F200494FF0640A0B
:1036E00041F6101B6E463859795988421DD048461C
:1036F00005F08AFF00281EBF38597959884214D036
:103700007859642200FB0A7000EB0B013046FDF78C
:10371000A0FB785931460130424600F01F00785135
:10372000484605F005FD0028DDD023B0BDE8F08F48
:1037300016F096BF0000000000F0FE000A2809D134
:1037400080B5282006F000FF0020BDE8804040B290
:10375000704700BFFF2040B270470000000000002B
:1037600000F0FE000A2809D180B5282006F000FFED
:103770000020BDE8804040B2704700BFFF2040B24B
:1037800070470000000000000C2801D9002070479D
:1037900080B54DF6A051C0F6010101EBC00231F831
:1037A0003010506806F00CFE0138B0FA80F0400985
:1037B00080BD00000000000021B10C2806D9FF20C8
:1037C00040B27047FE2040B2704700BF4DF6A05295
:1037D000C0F6010232F83000C2071FD182071FD4A1
:1037E00042071FD402071FD4C2061FD482061FD46B
:1037F00042061FD402061FD4C2051FD482051FD45F
:1038000042051FD402051FD4C2041FD482041FD452
:1038100042041FD4000424D50F201CE000201AE02D
:10382000012018E0022016E0032014E0042012E03A
:10383000052010E006200EE007200CE008200AE03A
:10384000092008E00A2006E00B2004E00C2002E03A
:103850000D2000E00E2041F2A842C2F2004242F8E0
:103860002010002040B270470C2803D9FF2040B23E
:10387000704700BF80B50A464DF6A051C0F6010161
:1038800001EBC00331F83010586806F0A1FD0020AC
:10389000BDE8804040B2704716F0BEB9000000009D
:1038A000062803D9FF2040B2704700BF4DF63C61A7
:1038B000B7EE001AC0F60101062851F8301080FE5C
:1038C000410A9FED1E1A0A6880FE010AD16A01F1C1
:1038D000010101EE101AB8EE411A20EE010ABCEE09
:1038E000C00A10EE101A11D8DFE800F004100A1018
:1038F0000A10040002F134000160002040B2704759
:1039000002F138000160002040B2704700F0FB0374
:10391000012B05D102F13C000160002040B270474C
:10392000032805D102F140000160002040B2704739
:1039300002F15C000160002040B27047000000000E
:1039400010B52DED028B062804D9FF2040B2BDEC46
:10395000028B10BD0446B0EE408A08F0A5FF4DF67C
:103960003C61BFEE001AC0F6010151F834104A68FC
:103970000132B0FBF2F000EE100A0022B8EE400A6D
:1039800080EE080A30EE010ABCEEC00A10EE100A02
:10399000B2EB104F04D0FF2040B2BDEC028B10BD43
:1039A0000A68D062C860002040B2BDEC028B10BD36
:1039B000062803D9FF2040B2704700BF80B54DF6FE
:1039C0003C62C0F6010202EBC00152F83000898867
:1039D0000BF01EFA0020BDE8804040B270470000A6
:1039E000062803D9FF2040B2704700BF80B54DF6CE
:1039F0003C62C0F6010202EBC00152F83000898837
:103A00000BF0D6FA0020BDE8804040B270470000BD
:103A100080B518B1FF2040B280BD00BF42F66820DB
:103A2000C2F2004013B10AF067F802E0142309F073
:103A300067FE002818BF012040B280BD00000000D2
:103A400052B141F2F043C2F2004303EB401040F8A0
:103A50002120002040B27047FE2040B27047000095
:103A600080B518B1FF2040B280BD00BF42F668208B
:103A7000C2F2004013B10AF0F3FA02E014230AF094
:103A800033F9002818BF012040B280BD00000000BB
:103A900070B5044615F020F90546FF2615F000F92B
:103AA000411C05290CD80120884010F0310F0CD1A1
:103AB00010F0060F0CD0204605F0DEFA13E000BF30
:103AC0006FF00041884218BF002670B270BD00BF81
:103AD0004FF47A70B0FBF5F1B4FBF1F0A14288BF6E
:103AE000012015F0B1F8002670B270BD0000000092
:103AF00018F01EBB000000002DE9F04115F0ECF8B5
:103B0000044618F015FB4EF218074FF47A78CEF2FF
:103B10000007B8FBF4F404FB00F63D6818F008FB5E
:103B200060433968864200FB08F008BF294657F811
:103B3000042C01FB08F10132B1FBF2F1401A002123
:103B400000F57A70BDE8F08142F66C4242F6BC6145
:103B5000C2F20042012818BF0022C2F20041002830
:103B600018BF1146084670470068C169C90658BFAA
:103B7000704745F200010323C4F2000101F5404201
:103B8000904241F2105208BF0123411AC2F2004292
:103B900018BF194601EBC10102EB8101102202623C
:103BA000086A08B1004700BF70470000000000002D
:103BB00080B5012802D9FF2040B280BD8446FE2096
:103BC000002918BF002A01D140B280BD42F66C4ED8
:103BD00042F6BC60C2F2004EBCF1010F18BF4FF0BC
:103BE000000EC2F20040BCF1000F18BF70461BB1BE
:103BF0000CF0EAF840B280BD0CF0DEF940B280BDB6
:103C000032B1FF23012898BF082905D958B270475F
:103C1000FE2358B2704700BF00EBC00041F21053C2
:103C2000C2F2004303EB8000002340F8212058B289
:103C3000704700000000000080B5012802D9FF2075
:103C400040B280BD8446FE20002918BF002A01D161
:103C500040B280BD42F66C4E42F6BC60C2F2004EED
:103C6000BCF1010F18BF4FF0000EC2F20040BCF1D2
:103C7000000F18BF70461BB10CF036FA40B280BD81
:103C80000CF0A2FA40B280BDB0B578B10446017420
:103C900001202070FFF72CFF217C0025C4E90205DC
:103CA0000846FFF79DFE68B2B0BD00BFFF2568B2B1
:103CB000B0BD0000000000002DE9F0472DED0A8B9B
:103CC00070B104460078002800F08A8071B10129A3
:103CD00040F086804DF6086AC0F6010A0AE000BF8F
:103CE000FF2568B2BDEC0A8BBDE8F0874DF6746A1B
:103CF000C0F6010AB2EE08AAB6EE008A4FF000083C
:103D00004FF001099FED4DBA00279FED4DCA00BF4E
:103D10001AF827000AEB8706FF283ED0717801EBDE
:103D2000410100EB81000C3000EE100AB8EEC00A31
:103D300030EE0B0A80EE0A0A19F0B8F920EE0C9A60
:103D40002078B5EE409AF1EE10FA25DD002847D034
:103D500084F80090FFF7CCFE217CB0EE490AC4E95C
:103D600002080846FFF7ECFD217CB0EE480A054644
:103D70000846FFF795FD28434CD1207880B384F89E
:103D80000090FFF7B5FE217CC4E902080846FFF762
:103D90000FFE60B13EE000BF48B184F80090FFF72D
:103DA000A7FE217CC4E902080846FFF719FE7088C7
:103DB000FFF76EFE207848B184F80090FFF798FE78
:103DC000217CC4E902080846FFF70AFE1420FFF729
:103DD0005FFE20780C2F09D0002807F1010797D14A
:103DE000FF2568B2BDEC0A8BBDE8F08700284FF0D4
:103DF00000053FF476AF01202070FFF779FE217CAB
:103E0000C4E902050846FFF7EBFD68B2BDEC0A8B7A
:103E1000BDE8F08720780028E2D001202070FFF76D
:103E200067FE217C0022C4E902020846FFF7D8FDA4
:103E3000FF2568B2BDEC0A8BBDE8F08700008AC29E
:103E40000000DC430000000010B52DED048B18B31A
:103E50000446007800B3B0EE608AB0EE409A0120CC
:103E60002070FFF745FE217CB0EE490A0022C4E92C
:103E700002020846FFF764FD217CB0EE480A0446C2
:103E80000846FFF70DFD204318BF4FF0FF3040B24A
:103E9000BDEC048B10BD00BFFF2040B2BDEC048B15
:103EA00010BD00000000000010B598B10446007875
:103EB00080B101202070FFF71BFE217C0022C4E9A5
:103EC00002020846FFF774FD002818BF4FF0FF30CC
:103ED00040B210BDFF2040B210BD00000000000045
:103EE00010B598B10446007880B101202070FFF72A
:103EF000FFFD217C0022C4E902020846FFF770FDA5
:103F0000002818BF4FF0FF3040B210BDFF2040B274
:103F100010BD000000000000FEE7000000000000EF
:103F20002DE9F0412DED0E8B044600284FF0FE00E8
:103F300000F0AA810D46002900F0A681FFF7DCFD04
:103F4000D4E90023801A994119F01CFE00EE100AF2
:103F50009FEDEE1A80EE010A84ED020AFFF7CCFD18
:103F60002F78227DC4E90001BA4200F09580E06814
:103F70000DF072FAE06806300DF06EFAE0680C3071
:103F80000DF06AFAE06812300DF066FAE068183059
:103F90000DF01EF8E0681E300DF01AF804F2D4405F
:103FA00004F579760FF0BCFC04F5A2600FF0B8FCC4
:103FB00030460FF0B5FC04F584600FF0B1FC04F25C
:103FC0005C400FF0ADFC04F593600FF0A9FC04F524
:103FD00021700CF05DFB04F544700CF059FB9FED73
:103FE000CC8A04F2C450B0EE480A0CF081FCB0EE6A
:103FF000480A04F2E4500CF07BFCB0EE480A04F2EC
:1040000004600CF075FCB0EE480A04F224600CF079
:104010006FFCB0EE480A04F244600CF069FCB0EEAC
:10402000480A04F264600CF063FCE0680026C4E90E
:10403000E766C4E9E966C4F8AC639FEDB60AC4F864
:10404000B06394ED1EAA90ED798A9FEDB3BA38EE75
:10405000009AB0EE480AF0EE4A0AB0EE4B1A01F0B0
:104060009BF9B0EE40CAB0EE490AF0EE4A0AB0EE53
:104070004B1A01F091F9B0EECC1AB0EEC00AB4EED2
:10408000401AF1EE10FAC8BF012639FE080A27755A
:1040900084EDED0A84F8C06304F1C40794ED060AC8
:1040A000D4ED0A0A94ED291AD4ED261A384613F0F5
:1040B00067FD04F5D276D4ED0E0A94ED120A94ED64
:1040C000291AD4ED261A304613F05AFD9FED939A23
:1040D00094ED3EEAB0EE490A9FED91AAB7EE00BA20
:1040E0009FED90CAB0EE4CDA0EEE4E0A80EE0A8AD0
:1040F000B0EEC80AB4EE4B0AF1EE10FA37DCB0EEBF
:10410000480A18F0E3FA19F033F99FED871AB0EE78
:10411000402A9FED864A28EE013A20EE044A9FEDA0
:10412000840A03EE004A02EE410A9FEDF11A31EED5
:10413000433AB0EEC44A20EE000A03EE030A9FEDB4
:10414000ED3A24EE033A23EE013AB1EEC01A22EE24
:10415000038AB4EE411AF1EE10FA80F1CD819FEDA1
:10416000EC0A21EE000A2EEE000A88EE00DAB0EE2C
:10417000490A94ED76EA0EEE4E0A80EE0A8AB0EE17
:10418000C80AB4EE4B0AF1EE10FA37DCB0EE480A7A
:1041900018F09CFA19F0ECF89FEDE61AB0EE402A00
:1041A0009FEDE54A28EE013A20EE044A9FEDE30A2E
:1041B00003EE004A02EE410A9FEDE21A31EE433A65
:1041C000B0EEC44A20EE000A03EE030A9FEDDC3A8B
:1041D00024EE033A23EE013AB1EEC01A22EE038A2E
:1041E000B4EE411AF1EE10FA80F18C819FEDD60AFF
:1041F00021EE000A2EEE000A88EE00CA1DEE100A1B
:1042000040F20108C7F6807820F00040B0F1FF4F7F
:1042100040D894ED5D0AB3EE041A3DEE000A00208A
:1042200084ED5D0AB4EE410AF1EE10FAC8BF012038
:1042300084F878011CEE100A20F0004040452FD38E
:10424000207D032840D8DFE800F00375454B00BF10
:10425000E0680DF029FBE06806300DF025FBE06812
:104260000C300DF021FBE06812300DF01DFBE06812
:1042700018300CF055FFE0681E300CF051FF20465E
:10428000294600F069FA002040B2BDEC0E8BBDE873
:10429000F08100BF1CEE100A20F000404045CFD254
:1042A00094ED950AB3EE041A3CEE000A002084ED6A
:1042B000950AB4EE410AF1EE10FAC8BF012084F865
:1042C0005802207D0328BED9FD2040B2BDEC0E8BE4
:1042D000BDE8F0812046294600F03EFA2046FFE086
:1042E0002046294600F038FA95ED020A94ED2F1A7F
:1042F0009FED962A204600EE021A94ED300A84EDD6
:104300002F1A95ED021A01EE420AE7E000247449E3
:1043100000000000DB0F4940DB0FC9402ECCE23D1E
:10432000BDAEDF3D0000C07FCDCC4C3DC52030BCD4
:1043300031082C3D2046294600F00EFAB0EE490A1D
:1043400094ED3EEA9FED7ACAB0EE4CDA0EEE4E0ADC
:1043500080EE0A8AB0EEC80AB4EE4B0AF1EE10FA0B
:1043600037DCB0EE480A18F0B1F919F001F89FED0A
:10437000711AB0EE402A9FED704A28EE013A20EE05
:10438000044A9FED6E0A03EE004A02EE410A9FEDD9
:104390006D1A31EE433AB0EEC44A20EE000A03EE45
:1043A000030A9FED673A24EE033A23EE013AB1EE99
:1043B000C01A22EE038AB4EE411AF1EE10FA80F12F
:1043C000A9809FED610A21EE000A2EEE000A88EE18
:1043D00000DA94ED76EA0EEE4E9A89EE0A8AB0EE95
:1043E000C80AB4EE4B0AF1EE10FA36DCB0EE480A19
:1043F00018F06CF918F0BCFF9FED4E1AB0EE402A91
:104400009FED4D4A28EE013A20EE044A9FED4B0AFB
:1044100003EE004A02EE410A9FED4A1A31EE433A9A
:10442000B0EEC44A20EE000A03EE030A9FED443AC0
:1044300024EE033A23EE013AB1EEC01A22EE038ACB
:10444000B4EE411AF1EE10FA6AD69FED3F0A21EE62
:10445000000A2EEE000A88EE00CA1DEE100ABBEE1E
:10446000048A1CEE101A9FED319AF0EE490A20F0F2
:10447000004038EE4D1A4045B0EE480A21F00040A9
:1044800038EE4C2A38BFB0EE410A4045384638BFB6
:10449000B0EE428A13F06CFE04F1AC0104F1B002FC
:1044A000384613F0DDFDB0EE480AF0EE490A30461A
:1044B00013F05EFE04F1B80104F1B402304613F0CB
:1044C000CFFD95ED010A9FED211A20EE010A20464D
:1044D00084ED2F0A95ED010A20EE010A84ED300AE1
:1044E00000F022FD002040B2BDEC0E8BBDE8F08153
:1044F000F6285C3E0000B44319F002F8B0EE401A12
:104500002DE600BF18F0FCFFB0EE401A6EE600BFCB
:104510004A0C823E18F0F4FFB0EE401A51E700BF9B
:1045200018F0EEFFB0EE401A8FE700BF0000000069
:104530000000C07FCDCC4C3DC52030BC31082C3DA7
:104540000000B443F6285C3E4A0C823ECDCC4C3E83
:10455000F0B581B02DED028BFF2600281CBF0D4663
:10456000002905D170B2BDEC028B01B0F0BD00BFD7
:10457000B0EE408AB5EE400AF1EE10FAF2DD0446E4
:10458000C56000202075FEF7FBF90CF0E1FFE06844
:104590000DF0FEF8C0B9E06806300DF0F9F898B9F2
:1045A000E0680C300DF0F4F870B9E06812300DF0EE
:1045B000EFF848B9E06818300CF02AFD20B9E0683F
:1045C0001E300CF025FD28B1FF2670B2BDEC028B29
:1045D00001B0F0BDE06824300CF0F6FAB0EE480A05
:1045E00004F1C40005F12C0113F07AFDB0EE480A85
:1045F00004F5D27005F1480113F072FDB0EE480ADF
:1046000005F5C27704F2D44001213A4604F57976E3
:104610000FF03AF9B0EE480A04F5A26001213A46DB
:104620000FF032F9B0EE480A05F5927201213046DA
:104630000FF02AF9B0EE480A04F5846005F5A2727D
:1046400001210FF021F9B0EE480A05F5B27604F227
:104650005C40012132460FF017F9B0EE480A04F52C
:104660009360012132460FF00FF905F1640604F55D
:10467000217031460BF0F0FF04F5447031460BF029
:10468000EBFFB0EE480A04F2C450D5ED7E0A0CF000
:10469000D7F8B0EE480A04F2E450D5ED7E0A0CF0EB
:1046A000CFF8B0EE480A04F20460D5ED7E0A0CF0B3
:1046B000C7F8B0EE480A04F22460D5ED7E0A0CF08B
:1046C000BFF8B0EE480A04F24460D5ED7E0A0CF063
:1046D000B7F8B0EE480A04F26460D5ED7E0A0CF03B
:1046E000AFF8F3EE0E0AB0EE480A04F284600CF064
:1046F000A7F8E0680CF0B0FEE06806300CF0ACFE05
:10470000E0680C300CF0A8FEE06812300CF0A4FE5B
:10471000E06818300CF05CFCE0681E300CF058FCCF
:1047200004F567702A210026C4F8C863FCF7F5FB7E
:10473000E068D0F8D411C4F8CC13D0F8D811C4F87C
:10474000D013D0F8DC01C4F8D40370B2BDEC028BF6
:1047500001B0F0BD000000002DE9F04381B02DED67
:10476000108B90B0044600284FF0FE0000F09283BA
:104770008846002900F08E8398ED010A94F8C00362
:1047800030EE000A94EDEC3A002804F521760AAFE9
:10479000D4F80001B1EE401A0A90D4F804010B904D
:1047A000D4F89C030C9000FE010A94ED021A31EE3D
:1047B000012AD4F8A0030D90D4F8A40030EE430AE7
:1047C0000E90B1EE424A3046394680FE422AB4EE9F
:1047D000404AF1EE10FA34FE020A94EDEA2A33EE72
:1047E000000A84EDEB0A84EDEC0A01EE002A94ED58
:1047F000250AB1EE400A8DED0F0A84EDEA2A0BF08E
:10480000A3FF04F54475D4E97801CDE90A012846EF
:1048100039460BF099FF94ED3E0A30460BF0D0FD7F
:1048200094ED760A28460BF0CBFD4CF6CD410027DF
:10483000CBF6CC51089198F80010D4F8A80398ED65
:10484000020A06900329D4F8AC03CDE90477079057
:1048500009971FD1B5EE400AF1EE10FA1AD094F87C
:10486000780100285BD004A930460BF021FF3046C8
:104870000BF09EFE94F85802002874D004A9284634
:104880000BF016FF28460BF093FE94EDD71A94ED2B
:10489000EF0A8CE09FEDEF1AE06820EE010AD4EDFC
:1048A0001E0AC4EDEE0A9FEDEC2A90ED791A9FEDF9
:1048B000EBAA31EE022A30EE018AB0EE4A1A30EE4F
:1048C000029AB0EE480A00F067FDB0EE40BAB0EED2
:1048D000490AB0EE4A1AD4EDEE0A00F05DFDB0EEE2
:1048E000CB1A04F57970B0EEC00AB4EE401A9FED11
:1048F000DC1AF1EE10FAC8BF012739FE080AD4ED20
:10490000021AD4ED1E0A84EDED0A84F8C0730EF08D
:104910000BFF84EDEF0A94F878010028A3D14DF243
:104920000A7004A9C3F62360049030460BF0C0FE61
:1049300094ED400A9FEDCB1A31EE400A94EDBD1A7A
:1049400094EDBE2A0020C4F8D00221EE000A94EDB6
:10495000411AC4F8BC0302EE410A84EDB50A94F88A
:10496000580200288AD14DF20A7004A9C3F62360C8
:10497000049028460BF09CFE94ED780A9FEDB91A3E
:1049800031EE400A94EDE01A94EDE12A0020C4F8DB
:104990005C0321EE000A94ED791AC4F8BC0302EE20
:1049A000410A9FEDAF1A84EDD80AB0EE410AB4EE89
:1049B000002AB0EE404A94EDB43A9FEDA98AD4EDB6
:1049C000021A04F5846011EE020A94ED251A03EE32
:1049D000024AD4ED2A0A04F1C40604F5D27984ED22
:1049E000300AB0EE480A84ED2F4A0EF09DFE94F88E
:1049F000780148B194F858020FF2FC41002808BF32
:104A0000043191ED001A01E09FEDDF1AB1EE412A69
:104A100098ED04AA80FE411AB4EE402AF1EE10FA95
:104A200032FE019AFFF768F84FF47A720023FBF721
:104A300009FD94F8C513D4F8C83394F8C4230029A9
:104A4000A0EB030110D07AB90122A4F8C423C4F862
:104A5000C803E268D2F8C431994292ED75FA23D2C4
:104A6000B0EE4F0A27E000BF9FED7E1A042A0AEE3F
:104A7000011A31EE090A31EE49FA00F21382DFE839
:104A800012F01A000500070015022102E1E700BF3D
:104A9000E2689FEDBEFAD2F8C831994292ED768A6B
:104AA000DED3032101E000BF022184F8C413B0EE7D
:104AB0004F0AC4F8C803DFEDB5BA02AF80FE6B0A37
:104AC000DFEDB38A0021002230463B4680FE28BA43
:104AD0000025009513F0E4FA3B1D00210022484612
:104AE000009513F0DDFAD4ED021A94ED411AD4EDDD
:104AF000400A04F25C4094ED780AD4ED3ECA0EF010
:104B000013FEB0EE40AAD4ED021A94ED400A94EDE3
:104B1000791AD4ED780A04F5936094ED76EA0EF0F4
:104B200003FEB0EE409AB0EE4B0A04F2D440D4ED4E
:104B3000021AD4ED3E0A9DED021A0EF0F5FDDFEDEE
:104B4000EC9AD4ED3EDAB0EE691ADFEDEDAAB7EEDD
:104B500000DAB0EE40BA0DEEED1A81EE2ACAB0EEE0
:104B6000CC1AB4EE4D1AF1EE10FA03DD9FEDE50A12
:104B700038E000BFB0EE4C0A17F0A8FD18F0F8FBC3
:104B80009FEDE11AB0EE402A9FEDE04A2CEE013A8B
:104B900020EE044A9FEDDE0A03EE004A02EE410ACF
:104BA0009FEDDD1A31EE433AB0EEC44A20EE000A22
:104BB00003EE030A9FEDD73A24EE033A23EE013ABF
:104BC000B1EEC01A22EE03CAB4EE411AF1EE10FAA9
:104BD00080F182819FEDD10A21EE000A2DEE800A3C
:104BE0008CEE000A10EE100ADFEDC20AB2EE04CA23
:104BF0008FFE6BFAF0EE60BA20F00040B0F1FF4F8C
:104C000094F8C40398BFF0EE40BA032813D02CEEFA
:104C10008C0AD4EDB5CA20EE0AAA94ED400A18F029
:104C2000A7FB0CEE80BA9FEDBE0A3BEE00BA94EDF6
:104C3000B50A7AEE000A3BEE6B0A30468FFE28AAD0
:104C400038EE000A13F094FA70B10020C4E92B008A
:104C500011E000BFDB0FC93FDB0F4940DB0FC9404C
:104C6000000000000AD7233E04F1AC0104F1B002B9
:104C7000304613F0F5F9B0EE4A0A012604F5A260B9
:104C8000D4ED021AD4ED760A9DED031AC7F68076AC
:104C90000EF04AFD94ED76FAB0EE40AA4FEE4F9A30
:104CA00089EEAABAB0EECB1AB4EE4D1AF1EE10FAB4
:104CB00002DD9FED940A37E0B0EE4B0A17F006FDD7
:104CC00018F056FB9FED901AB0EE402A9FED8F4AE8
:104CD0002BEE013A20EE044A9FED8D0A03EE004AC6
:104CE00002EE410A9FED8C1A31EE433AB0EEC44A0F
:104CF00020EE000A03EE030A9FED863A24EE033A03
:104D000023EE013AB1EEC01A22EE03BAB4EE411A14
:104D1000F1EE10FA80F1E6809FED800A21EE000AA4
:104D20002FEE000A8BEE000A10EE100ADFED710A7A
:104D300094F8C413B0EE60BA20F00040B04238BF1F
:104D4000B0EE40BA032913D02EEE0C0A94EDD8CA67
:104D500020EE099A94ED780A18F00AFB0CEE00AAEE
:104D60009FED6F0A3AEE00AA94EDD80A79EE000A98
:104D70003AEE4B0A484638EE000A13F0F9F948B10A
:104D80000020C4E92D000CE00AD7A33C7B14AE3E02
:104D9000CDCCCC3D04F1B80104F1B402484613F087
:104DA0005FF9BFEE001A94ED2F0AB0EE412AB4EE7F
:104DB000410AF1EE10FA08DBB0EE4D2AB4EE4D0ACE
:104DC000F1EE10FA01DCB0EE402A94ED300A84EDE9
:104DD0002F2AB4EE410AF1EE10FA08DBB7EE001A02
:104DE000B4EE410AF1EE10FA01DCB0EE401A9FED8C
:104DF0004D0A84ED301AB0EE401A94ED2B2AB4EE31
:104E0000402AF1EE10FA08DB9FED451AB4EE412A74
:104E1000F1EE10FA01DCB0EE421A84ED2B1AB0EE7E
:104E2000401A94ED2C2AB4EE402AF1EE10FA08DB79
:104E30009FED3B1AB4EE412AF1EE10FA01DCB0EE20
:104E4000421A84ED2C1AB0EE401A94ED2D2AB4EEDD
:104E5000402AF1EE10FA08DB9FED311AB4EE412A38
:104E6000F1EE10FA01DCB0EE421A94ED2E2A84ED38
:104E70002D1AB4EE402AF1EE10FA08DB9FED280A55
:104E8000B4EE402AF1EE10FA01DCB0EE420A002046
:104E900084ED2E0A40B210B0BDEC108B01B0BDE81D
:104EA000F08300BF002084F8C40304E6E268D2F86F
:104EB000CC3192ED788A994292ED77FAFFF4D0AD39
:104EC0000421F2E5E268D2F8D0219142FFF4F3AD7B
:104ED000002184F8C413ECE518F012FBB0EE401A80
:104EE00078E600BF18F00CFBB0EE401A14E700BFE4
:104EF0002ECCE23D00000000CDCC4C3D0AD7A33CB7
:104F0000BDAEDF3D0000C07FCDCC4C3DC52030BCE8
:104F100031082C3D0000B443F6285C3E4A0C823E2A
:104F200000007042000070C2002808BF7047B0B592
:104F300086B0044601AD0020CDE90300CDE90100B3
:104F4000E068D4F8AC10059129460CF00DFBE06840
:104F5000D4F8B0100591063029460CF005FBE06846
:104F6000D4F8B41005910C3029460CF0FDFAE06835
:104F7000D4F8B8100591123029460CF0F5FAE06823
:104F8000183094ED2F0A0CF0D3F8E06894ED300A55
:104F90001E300CF0CDF806B0BDE8B0407047000000
:104FA00050B1017D022907D190F8C413002918BF20
:104FB0007047012180F8C513704700000000000011
:104FC000002800F0038110B52DED0A8B04460CF08B
:104FD000D7FD0CF0E5F9E0680CF062FA40B100F1A1
:104FE0001C0304F1180C806A0ECB8CE80E00606282
:104FF00094ED060A9FED778A30EE081A9FED769AB7
:10500000B4EE490AE068F1EE10FA00F1060031FE54
:10501000000AB1EE400A84ED060A0CF041FA40B1F4
:1050200000F11C0304F1280C806A0ECB8CE80E0002
:10503000606394ED0A0AE06830EE081A0C30B4EEB2
:10504000490AF1EE10FA31FE000AB1EE400A84ED91
:105050000A0A0CF025FA40B100F11C0304F1380CE7
:10506000806A0ECB8CE80E00606494ED0E0AE06856
:1050700030EE081A1230B4EE490AF1EE10FA31FEA1
:10508000000AB1EE400A84ED0E0A0CF009FA40B1B4
:1050900000F11C0304F1480C806A0ECB8CE80E0072
:1050A000606594ED120AE06830EE081A1830B4EE2C
:1050B000490AF1EE10FA31FE000AB1EE400A84ED21
:1050C000120A0BF03DFF40B100F11C0304F1580C33
:1050D000806A0ECB8CE80E006066E0681E300BF034
:1050E0002FFF40B100F11C0304F1680C806A0ECB65
:1050F0008CE80E00606794ED0B0A9FED381A20EEE5
:10510000010A94ED172A94ED1B4A94ED263A9FED7F
:10511000349A94ED3FBA02EE010A94ED0F2A22EE82
:10512000012A04EE012A94ED3E1A94ED414A30EE34
:10513000430A21EE048A00EE098A94ED400A32EE19
:1051400043AA18F015F994ED761A94ED792A21EE18
:1051500002CA0BEE008A94ED780A0AEE09CA94EDB1
:10516000779A18F005F909EE00CAB6EE002AB3EEF8
:10517000041AD4F8A003C4F8A40338EE0C0A20EEF5
:10518000020A94ED5D2AB4EE412AF1EE10FA08DA33
:1051900094ED952AB4EE412AF1EE10FAB8BF9FEDD6
:1051A000110A04F284600BF01BFB94ED021A94EDDB
:1051B000E72A00EE012A84EDE80A002084EDE72AC0
:1051C000BDEC0A8BBDE8104040B27047FE2040B2F3
:1051D000704700BFDB0FC9C0DB0F494035FA8E3C7A
:1051E00096438B3D0000000090ED001AF5EE400A5A
:1051F00031EE000AF1EE10FA0BDDB4EE600AF1EECA
:1052000010FA09DAB5EE400AF1EE10FA01DA30EEE2
:10521000200A80ED000A704730EE600A80ED000A37
:10522000704700000000000010B52DED088B00282D
:1052300044D030EEC11AB0EE429A9FED262A0446C1
:105240009FED253AB0EE628A31EE022AB4EE431A9F
:105250009FED233AF1EE10FA32FE011A9FED1F2A5C
:1052600031EE022AB4EE413AF1EE10FA32FE011AA2
:1052700031EE000A90ED001A30EE01AAB0EE610A9C
:10528000B0EE621AF0EE4A0A00F086F8B0EE40BACC
:10529000B0EE490AF0EE4A0AB0EE481A00F07CF887
:1052A00094ED002A82FE4B1AB4EE4B2AF1EE10FA6E
:1052B00008DCB4EE401AF1EE10FA03DBBDEC088B0B
:1052C00010BD00BF81FE000A84ED000ABDEC088B12
:1052D00010BD00BFDB0FC9C0DB0F4940DB0FC94069
:1052E000DB0F49C00000000010B52DED0A8B00282F
:1052F00046D030EE600AB0EE41AA9FED231AB0EE20
:10530000429A9FED222A044630EE011AF0EE4A0A34
:10531000B4EE420A9FED1F2AF1EE10FAB0EE618A58
:1053200031FE000A9FED1A1A30EE011AB4EE402A3F
:10533000F1EE10FA31FE00CA90ED000AB0EE491A03
:105340003CEE00BAB0EE4B0A00F026F8B5EE400A8B
:10535000F1EE10FA03DD3AEE4C0A84ED000AB0EEED
:105360004B0AF0EE480AB0EE491A00F015F8B5EE17
:10537000400AF1EE10FA03DA38EE4C0A84ED000A26
:10538000BDEC0A8B10BD00BFDB0FC9C0DB0F49406D
:10539000DB0FC940DB0F49C030EE600AB5EE401AA2
:1053A000F1EE10FA16DDB6EE002A21EE022AB4EE76
:1053B000420AF1EE10FA03DD30EE410A704700BFF9
:1053C000B1EE422AB4EE420AF1EE10FAA8BF7047DD
:1053D00030EE010A7047000080B502A20DF02CFBF0
:1053E000002080BD4369616C6C6FEFBD9E28E28830
:1053F000A0E383BBCF893C2029E28C92E298850D03
:105400000A0000000000000040F63850C2F20040E0
:10541000704700000000000041F67870C2F20040C2
:1054200002F0F6BC0000000042F26800C2F2004048
:1054300002F0EEBC0000000042F2E000C2F20040C8
:1054400002F0E6BC0000000042F25810C2F2004038
:1054500002F0DEBC0000000042F24820C2F2004030
:1054600002F0D6BC0000000042F2D010C2F20040B0
:1054700002F0CEBC0000000040F20F42D0F800C0A5
:10548000C4F20202944511DC6F22C4F20202944578
:1054900022DC3F22C4F20202944539DC1022C4F21D
:1054A000020294455AD0282254E000BF40F26F42D5
:1054B000C4F2020294451BDC40F23F42C4F20202F5
:1054C00094452DDC40F21042C4F20202944545D0CE
:1054D00040F228423EE000BF9F22C4F202029445FF
:1054E00028DC7022C4F20202944537D0882231E0D1
:1054F00040F29F42C4F20202944523DC40F2704223
:10550000C4F20202944529D040F2884222E000BF52
:105510004022C4F20202944520D058221AE000BF73
:1055200040F24042C4F20202944517D040F2584281
:1055300010E000BFA022C4F2020294450ED0B822AF
:1055400008E000BF40F2B842C4F20202944505D020
:1055500040F2A042C4F20202944519D16FF00F024A
:105560004AF6AB2352FA8CF2CAF6AA23A2FB033105
:105570000AA35F2AC1F302115B5C40F2FF312CEAFF
:105580000101C36588BF043181650846704700BFCB
:105590002CF0FF0181650846704700BF0006101619
:1055A000000610160000000070B540F26F44D0F8FD
:1055B00000C0C4F20204D0F858E0A4451ADC9F25CC
:1055C000C4F20205AC4533DC5725C4F20205AC45F4
:1055D0005ADC1025C4F20205AC4500F0988028255D
:1055E000C4F20205AC4500F092804025C4F20205E9
:1055F0008AE000BF45F22F45C5F60205AC452DDC1B
:1056000040F2B745C4F20205AC454BDC40F27045B0
:10561000C4F20205AC457AD040F28845C4F20205D6
:10562000AC4574D040F2A045C4F202056CE000BF66
:1056300040F22745C4F20205AC4543DCA025C4F284
:105640000205AC4563D0B825C4F20205AC455ED076
:1056500040F21045C4F2020556E000BF45F26B452A
:10566000C5F60205AC453FDC45F23045C5F60205FE
:10567000AC454CD045F24445C5F60205AC4546D094
:1056800045F258453EE000BF5825C4F20205AC453E
:105690003DD07025C4F20205AC4538D08825C4F24F
:1056A000020531E040F2B845C4F20205AC452ED007
:1056B00045F20845C5F60205AC4528D045F21C4523
:1056C00020E000BF40F22845C4F20205AC451ED0E0
:1056D00040F24045C4F20205AC4518D040F25845AE
:1056E000C4F2020510E000BF45F26C45C5F60205A4
:1056F000AC450CD045F29445C5F60205AC4506D044
:1057000045F28045C5F60205AC4540F0D580456EB2
:10571000C66E002E866E6E601CBFD0E91C566E6091
:10572000A44515DC9F24C4F20204A4452CDC5724B4
:10573000C4F20204A44551DC1024C4F20204A445BE
:105740007AD02824C4F20204A44575D040246FE026
:1057500045F22F44C5F60204A44529DC40F2B744C3
:10576000C4F20204A44545DC40F27044C4F20204D1
:10577000A44561D040F28844C4F20204A4455BD041
:1057800040F2A04454E000BF40F22744C4F20204B7
:10579000A4453FDCA024C4F20204A4454CD0B824A4
:1057A000C4F20204A44547D040F2104440E000BFD8
:1057B00045F26B44C5F60204A44555DC45F230447D
:1057C000C5F60204A44561D045F24444C5F602047E
:1057D000A4455BD045F2584454E000BF5824C4F2BD
:1057E0000204A44528D07024C4F20204A44523D0A6
:1057F00088241DE040F2B844C4F20204A4451BD042
:1058000045F20844C5F60204A4453FD045F21C44C5
:1058100038E000BF40F22844C4F20204A4450BD093
:1058200040F24044C4F20204A44505D040F258447A
:10583000C4F20204A4453FD18468C06D00F01F008B
:105840003F2505FA00F0CEF80800DCF80000402CF7
:1058500020F48020CCF80000CCF8043023D0CCF821
:105860000810CCF80C2070BD45F26C44C5F602045B
:10587000A4450BD045F28044C5F60204A44505D0EA
:1058800045F29444C5F60204A44515D1C46D806860
:1058900004F01F040125402805FA04F4CEF8044062
:1058A000CCF8043004D1CCF80820CCF80C1070BD32
:1058B000CCF80810CCF80C2070BD000000000000EF
:1058C000B0B5D8B141F27C24C2F20044207818B1BE
:1058D000FD2568B2B0BD00BF13F0FEFC606068B18A
:1058E00045F621320020C0F6000203210025FEF714
:1058F00087F90120207068B2B0BD00BFFE2568B2F4
:10590000B0BD00000000000010B538B13421002403
:1059100000F8244BFBF701FB60B210BDFE2460B21F
:1059200010BD000000000000B0B508B305460446F5
:1059300055F8100F01466FF3DF21A1F5B671B1F5EF
:10594000A56F11D8C0F3CA21A1F5B671B1F5A56F45
:105950000AD8A988800D40EA81206FF3DF20A0F5E6
:10596000B670B0F5A56F07D9FF2040B2B0BD00BF3B
:10597000FE2040B2B0BD00BF11F4405F4FF0FF0009
:1059800000F0C5808AB2B2F5804FC0F0C080C1F38C
:105990004A01A1F5B671B1F5A56F00F2B8800120FA
:1059A0002070FEF7A9F82A6894F81CC013466FF31C
:1059B000DF23BCF1000F00EE103AA369C4E9020135
:1059C000C2F3CA20A988B8EE401A9FED520AE363D9
:1059D00031EE001A31EE012A01EE100A4FEA925020
:1059E00040EA81206FF3DF20B8EE413A04EE100A5E
:1059F0009FED491AC1F34A0082EE012A05EE100A12
:105A000033EE003AB8EE444A84ED0B2A4FEA913265
:105A100084F83920B8EE455AE28A34EE004A4FF055
:105A2000000033EE033A6065C1F3013135EE005AF0
:105A300034EE044A84F8381083EE013A628735EE7A
:105A4000052A84ED0C3A84EE013A627F84ED093A2E
:105A500082EE012A84ED0A2A18BF4FF0010C002AB9
:105A600084F840C018BF0122E38B84F852C084F848
:105A70004120DDB203F0010184F84210C5F340017A
:105A800084F84310C5F3800184F84410C5F3C001C5
:105A900084F84510C5F3001184F84610C5F3401191
:105AA00084F84710C5F3801184F84810E90984F898
:105AB0004910C3F3002184F84A10C3F3402184F84D
:105AC0004B10C3F38025218C84F84C5002EE101A41
:105AD00084F85320C3F3C02184F84D10C3F3003180
:105AE00084F84E10C3F34031B8EE422A84F84F10C8
:105AF000C3F3803184F8501032EE000AD90B84F8D9
:105B0000511030EE000A80EE010A84ED0D0A40B219
:105B1000B0BD00BF000080C40000A544000000002C
:105B200041F27C200121C2F20040406813F0DCBA4F
:105B300010B504460020FEF707F804F11001122208
:105B40000AF042F9002818BF4FF0FF3010BD0000E6
:105B500080B502460120012113F00AFB0138B0FA9A
:105B600080F0400980BD0000704700000000000088
:105B700080B54FF4806004F023FB4FF48050BDE803
:105B8000804004F01DBB0000EFF3108072B600BF30
:105B9000FEE700000000000044F60400C5F6020025
:105BA000816841F0020181600168890409D40168BB
:105BB00089045CBF01685FEA814102D401688904FD
:105BC000F2D570470000000042F2C020C2F200404F
:105BD00003F026BD0000000042F2C020C2F20040E7
:105BE00003F01EBD0000000042F26030C2F200402F
:105BF00003F016BD0000000042F26030C2F2004027
:105C000003F00EBD0000000042F20040C2F200406E
:105C100003F006BD0000000042F20040C2F2004066
:105C200003F0FEBC0000000010B54FF0000CC2F8FD
:105C300000C08C4500F08680047844F02003202BBF
:105C400028D0447844F02003202B11D0847844F0ED
:105C50002003202B14D0C47844F02003202B17D02D
:105C60000430047844F02003202BEAD112E000BF76
:105C700001305FFA84FEBEF1200F10D01FE000BF9C
:105C800002305FFA84FEBEF1200F08D017E000BF9B
:105C9000033000BF5FFA84FEBEF1200F0FD14478BD
:105CA000202C11D18478202C16D1C478202C1BD123
:105CB00010F8044F5FFA84FEBEF1200FEFD0BEF162
:105CC000000F3FD00AE000BFE4B301300CF1010C3B
:105CD0008C45AED10EE000BFA4B302300CF1010C34
:105CE0008C45A6D106E000BF64B303300CF1010C73
:105CF0008C459ED1022144F02003DBB2202B1ED024
:105D000043184C1E146013F8014C44F02004202C5E
:105D10001AD01160445C44F02004202C16D04C1C96
:105D200014605C7844F02004202C11D08C1C14608A
:105D30009C78043144F02003DBB2202BE0D10239FF
:105D400007E000BF002010BD012102E0012100E0BA
:105D50000121002908BF084610BD00000000000016
:105D60002DE9F04741F2A44A9046C2F2004A894622
:105D70000646DAF800307BB11C68A3684846414605
:105D800032469847002818BFBDE8F0870020CAF8BF
:105D90000000BDE8F08700BF41F2A405C2F2004553
:105DA000CAF8005005E000BF6D68CAF80050002D29
:105DB00061D02C6827683846FAF79CFF0246305CB1
:105DC00040F020002028EFD130463946FAF7B1FFE5
:105DD0000028E9D194F90CC0BCF1000FCDD400210A
:105DE000334600221F78202F06D119E039440122C2
:105DF00004331F78202F13D087B30022012758784F
:105E0000202817D050B3002201279878202817D0D7
:105E100020B300220127D878202817D1E6E700BF59
:105E2000012A4FF001024FF0000718BF01315878E6
:105E30002028E7D139440122002798782028E7D18B
:105E4000394401220027D8782028CFD030B1002251
:105E500004331F78202FCFD1E2E700BF012A08BF0B
:105E60000139C8B25FFA8CF1884218BF002D0DD1FC
:105E7000002D7FF482AF4EF255114846C0F6010165
:105E80004246FBF771F80020BDE8F0874EF2FD01B5
:105E90004846C0F601014246FBF766F876E7000087
:105EA000B0B5A8B10446082013F0B6FED0B105463F
:105EB00014F096FB40F214002C60C2F20040002265
:105EC0006A60016805604D6014F0B2FB0120B0BD4E
:105ED0004FF0500080F31188BFF36F8FBFF34F8FE7
:105EE000FEE700BF4FF0500080F31188BFF36F8FC3
:105EF000BFF34F8FFEE7000070B54FF0FE0608B30A
:105F00000C46F9B158210546FBF707F820890A220B
:105F100028830026206861686961286120782E70D6
:105F20006188FCF72DFE2078A1880A22FCF728FE64
:105F30002078E1880A22FCF723FE20780A222189B2
:105F4000FCF71EFE70B270BDB0B5002818BF002A65
:105F500000D1B0BD438A8B4246D192F800C015797A
:105F60005378547991789FED9A2A5B0192F803E077
:105F700043EA4C339FED904A43EAD10C4FEA8E231B
:105F800000EE10CA61F3944343EA85019379D27914
:105F900041EA9411DB0101EE101A64F3D433B8EE38
:105FA000400A43EA520203EE102AB8EE411A20EEEC
:105FB000020AB8EE433A21EE021A80EE040A23EEFA
:105FC000022A9FED843A81EE041A30EE030A82EE33
:105FD000042A80ED070A31EE031A80ED081A32EE2A
:105FE000030A80ED090AB0BD838A8B4244D111783F
:105FF0009FED752A53789FED704A9578D4785B01B0
:1060000043EA41311379A40241EAD50C517965F391
:1060100094449579D27944EA8303ED0100EE10CAE5
:1060200061F3D43543EA911345EA520101EE103A87
:1060300003EE101AB8EE400AB8EE411AB8EE433A31
:1060400020EE020A21EE021A23EE022A9FED5F3AA9
:1060500080EE040A81EE041A82EE042A30EE030A6E
:1060600031EE031A80ED0A0A32EE030A80ED0B1AB4
:1060700080ED0C0AB0BD00BFC38A8B4248D11178B5
:106080009FED4C2A53789578D4785B0143EA4131EF
:106090001379A40241EAD50C517965F394449579BA
:1060A000D27944EA8303ED0100EE10CA43EA91136A
:1060B00061F3D43501EE103A45EA5201B8EE400AD8
:1060C00003EE101AB8EE411A20EE020A9FED3C2AA8
:1060D000B8EE433A21EE021A23EE022A9FED363A39
:1060E00080EE030A81EE031A82EE032A9FED333A13
:1060F00030EE030A9FED333A80ED0E0A31EE030ACB
:1061000080ED0D0A32EE030A80ED0F0AB0BD00BF2C
:10611000038B8B4218BFB0BD51789FED251A937841
:10612000BFEE005AD4789D0845EA8111157900EE3A
:10613000101A210163F30D315379947941EA151155
:106140009B00D27965F38D2302EE101A43EA941373
:10615000B8EE400A64F30D2203EE103A04EE102A62
:10616000B8EE422A30EE000AB8EE433AB8EE444A9E
:1061700032EE022A33EE033A80EE010A34EE044A8C
:1061800082EE012A83EE013A84EE011A30EE050A0E
:1061900080ED100A32EE050A80ED110A33EE050A91
:1061A00080ED120A31EE050A80ED130AB0BD00BF82
:1061B00000FC7F4600003443F8FFFF490000B4C2F2
:1061C0000000B443000034C31F858B421F850BC2FF
:1061D0003333EB4233336BC2002869D0F0B595B04E
:1061E0000446007C6D460023618A2A46FCF76CFB5E
:1061F000B0FA80F14FEA511778B905F10D0600BFEA
:10620000618A20463246FFF79FFE207C0023618A88
:106210002A46FCF759FB0028F2D0207CA18A6D4663
:1062200000232A46FCF750FB80B905F10D0600BF9C
:10623000A18A20463246FFF787FE207CA18A0023F0
:106240002A46FCF741FB0028F2D00127207CE18A96
:106250006D4600232A46FCF737FB78B905F10D0699
:10626000E18A20463246FFF76FFE207CE18A002358
:106270002A46FCF729FB0028F2D00127207C6D4636
:10628000218B00232A46FCF71FFBA8B11FBBFDF79B
:1062900033FCD4E90223801A48F2A162C0F2010261
:1062A0009941801A71F100001BD30020207018E082
:1062B000FE2040B2704700BF05F10D06218B20463D
:1062C0003246FFF741FE207C0023218B2A46FCF753
:1062D000FBFA0028F2D001202070FDF70DFCC4E984
:1062E0000201002015B0BDE8F04040B27047000048
:1062F0002DE9F0412DED028B82B0044600284FF0CD
:10630000FF0000F039810E46002900F035819046EB
:10631000FDF7F2FBD4E90023801A994117F032FC13
:1063200000EE100A9FED971A80EE010A84ED020A32
:10633000FDF7E2FB3778257CC4E90001BD423DD082
:1063400004F17C000DF0ECFA04F1B8000DF0E8FA6D
:1063500004F1F4000DF0E4FA04F598700DF0E0FAA1
:106360009FED898A04F5BE70B0EE480A0AF0C0FAC3
:10637000B0EE480A04F5CE700AF0BAFAE0680830C8
:106380000AF0EEFA04F17000FBF7EEFB012F08BFF4
:10639000002D03D094ED730A0AE000BF94ED5D0A6E
:1063A00094ED5E1A30EE010AB6EE001A20EE010AF4
:1063B00084ED1D0AD4F8C4012067277496ED010A04
:1063C00094ED021A20EE010AB7EE081AE06890ED8B
:1063D0002B2A20EE010AB5EE402A8DED010AF1EEDE
:1063E00010FA10DDD4ED7A0AD4ED5B1A94ED1C0A94
:1063F00094ED711A94ED5C2A01A8DFED642AFEF792
:1064000013FF9DED010A04F17007DFED600A3846C5
:10641000FEF7EAFEE06896ED020A94ED021A90EDAE
:106420002C2A20EE010AB5EE402A8DED000AF1EE8D
:1064300010FA10DDD4ED7E0A94ED1D0AD4ED5D1A3C
:1064400094ED5E2A94ED731A6846DFED502AFEF74C
:10645000EBFE9DED000A04F17406DFED4C0A3046B8
:10646000FEF7C2FE207C411E022942D3032807D03A
:10647000002870D10020C4F8BC019FED430A68E0F9
:10648000B8F1000F35D098F8000090B3E068D8F864
:106490000410216790ED2B1A98ED020AB5EE401A10
:1064A000B1EE400AF1EE10FA84ED1D0A0DDD94ED17
:1064B0005B1AD4ED5C1AD4ED710A94ED7A0A9FED63
:1064C000332A3846FEF710FFE06890ED2C0AB5EE4F
:1064D000400AF1EE10FA0CDD94ED5D1AD4ED5E1A6F
:1064E000D4ED730A94ED7E0A9FED282A3046FEF71C
:1064F000FBFE9FED258A04F17C00B0EE481AD4ED36
:10650000021A94ED1C0AD4ED710A0DF00DF9B0EEEB
:10651000481A04F1B800D4ED021AD4ED760A0DF051
:1065200003F9B0EE481A84ED6F0A04F1F400D4EDDB
:10653000021A94ED1D0AD4ED730A0DF0F5F8B0EED1
:10654000481A04F59870D4ED021AD4ED750A0DF0CE
:10655000EBF884ED700A04F5BE7094ED6F0A0AF052
:106560003FF984ED6F0A04F5CE7094ED700A0AF0DD
:1065700037F9002084ED700A40B202B0BDEC028B06
:10658000BDE8F0810024744900000000DB0FC94021
:10659000B0B52DED028B00286AD00446B0EE408ADB
:1065A000C16000250574FCF7EBF9B0EE480AE1681C
:1065B00004F17C0001F13C0200210DF065F9B0EE20
:1065C000480AE16804F1B80001F11C0201210DF054
:1065D0005BF9B0EE480AE16804F1F40001F17C02D5
:1065E00000210DF051F9B0EE480AE16804F5987009
:1065F00001F15C0201210DF047F9E168B0EE480AB3
:1066000004F5BE70D1ED270A0AF01AF9E168B0EE80
:10661000480A04F5CE70D1ED270A0AF011F9E068B6
:1066200090ED290A90ED2A2A90ED2B1A90ED2C3A44
:1066300030EE011A84ED5C0A84ED5B1A32EE031A27
:1066400084ED5D1A84ED5E2A0BF0C6FBE06808302D
:106650000AF0BAFAE06808300AF082F9E16804F159
:1066600018001031FFF748FC68B2BDEC028BB0BDDA
:10667000FF2568B2BDEC028BB0BD00000000000039
:1066800010B586B00446C06894ED700A0BF038FC73
:10669000B1EE040A0020CDE9030094ED6F1A0290D8
:1066A00049F69A1021EE000AC3F699600590E06859
:1066B0008DED010A0BF0C0FAE06801A908300AF07C
:1066C000C7F906B010BD000010B538B30446C06865
:1066D0000BF0A2FCE0680BF037FB48B100F10803B7
:1066E00004F5FC7C40690ECB8CE80E00C4F8040273
:1066F000E06808300AF0F0FAE06808300AF07CF947
:1067000048B100F11C0304F5F47C806A0ECB8CE8E0
:106710000E00C4F8F401002040B210BDFF2040B2CA
:1067200010BD00000000000010B310B50446183082
:10673000FFF752FD606BC4F8DC01E16CC4F8C411D2
:10674000216DC4F8C811616DC4F8CC11216CC4F876
:10675000D011616CC4F8D411A16CC4F8D811A16B2C
:10676000E06BC4E978100020BDE8104040B27047EB
:10677000FF2040B27047000070470000000000009A
:10678000704700000000000070470000000000009B
:10679000704700000000000070470000000000008B
:1067A000B0B582B090F85C20012A03D102210846DE
:1067B00002B0B0BD42F2083200230193C4F20202DB
:1067C0000093A2F542740368A34227D14FF6006CF0
:1067D0004FF60055CFF6FF7CCFF6FF7552F80C4010
:1067E000535923435B0719D4D1F800E01368BEF175
:1067F000000F23F440441DD04B68234313605359CA
:1068000052F80C502B43DB0722D1136840F61F755A
:106810008968AB4341EA0E01194316E0016E41F06D
:10682000200101660121002280F85C20084602B0A8
:10683000B0BD00BF1460515952F80C301943C9075C
:1068400008D1116840F61F73994311600021EAE7EF
:106850000021E8E70021E6E72DE9F04181B00022C0
:10686000009290F85C20012A04D10221084601B070
:10687000BDE8F0810368012280F85C209A68520725
:1068800000F1FC8246F2083C4FF6FF78C5F6020C98
:10689000C0F20F08ACF5427E0A68734516D0B2F11B
:1068A000FF3F13DD92FAA2F512EA080FB5FA85F55B
:1068B0004FF0010608BF950E920E05F01F0506FA6F
:1068C00005F5DE693543DD6101E000BF920E4D68DC
:1068D0001F2402F01F02C5F3012605F01F05AC407E
:1068E00003EB8606AA40376B27EA0404224332638F
:1068F0009A689C68E40844EA9202D20740F0298131
:106900000A6807268D687345C2F34064C2F30452D7
:1069100003EB840406FA02F6676905FA02F227EA35
:10692000060642EA0602626110D041F20002C5F694
:106930000042126802F07042B2F1805F6ED14A6983
:10694000DC680E2505EA54069CE000BF4FF60454AF
:106950000A69CFF6FF74042A4D695CF8046067D1B8
:106960004FF65852CFF6FF725CF802201C6E0E688C
:10697000C4F3846416EA0802C6F3846596FAA6F6A0
:10698000B6FA86F6374608BF2F46BC420CD11A6EBF
:1069900022F000421A660C6804EA0802C4F3846517
:1069A00094FAA4F4B4FA84F65C6E37465C6E002A5E
:1069B00008BF2F46C4F38464BC420CD15A6E22F047
:1069C00000425A660C6804EA0802C4F3846594FA2B
:1069D000A4F4B4FA84F69C6E37469C6E002A08BF75
:1069E0002F46C4F38464BC420CD19A6E22F000425C
:1069F0009A660C6804EA0802C4F3846594FAA4F465
:106A0000B4FA84F6DC6E002ADC6E08BF2E46C4F3AE
:106A10008462B24200F099809BE000BFDC684A6962
:106A2000DD68E4064FEA55052AD405F00E0629E094
:106A30000624ACF52A7704EA96040E6805FA04F4F5
:106A400006F0F8452C4357F8226044F0004447F81C
:106A500022400A69CC6957F8225025F080752C43F2
:106A600047F822400A6991F8204057F82250012C3B
:106A700025F0007508BF05F1007547F8225068E061
:106A800005F008060F6903F16005042F20D12A687C
:106A90000C6802F0F842B2EB846F4FEA846241D195
:106AA0002C6824F000442C605C6E04F0F84494429E
:106AB0003DD09C6E04F0F844944241D19C6E24F089
:106AC00000449C66DC6E04F0F844944241D13CE002
:106AD0000C68B24055F8276004F0F84406F0004610
:106AE0002243324345F827200A6991F8214055F89E
:106AF0002260012C26F0004608BF06F1004645F84A
:106B000022600A7E0C691D69013A04F01F04B2FA82
:106B100082F225F4F0455209D202A2402A431A61BA
:106B200017E000BF5C6E04F0F8449442C1D15C6E83
:106B300024F000445C669C6E04F0F8449442BDD09E
:106B4000DC6E04F0F844944203D1DA6E22F0004285
:106B5000DA669A68D20711D173450A68CD680FD0FA
:106B600005F01804D3F8C01028FA04F402EA080665
:106B7000B14314402143C3F8C01012E0002182E168
:106B80004FF6A85105F01806CFF6FF7128FA06F661
:106B900002EA080716405CF80140BC4334434CF855
:106BA00001400021C4F2527101F52D04A54240F0CC
:106BB000138146F20004C5F60204A3422CD042F22F
:106BC0000014C4F20204A3423CD042F20004C4F216
:106BD0000204A34250D11F24C1F2F044A24275DD49
:106BE00040F2FF74C2F63064A2425FDD40F600045A
:106BF000C2F63064A24200F0BF8041F20004C3F24A
:106C00006024A24200F0B2800024C4F22134A242E7
:106C100000F0CD80B6E000BF1F21C1F2F0418A42F2
:106C20002CDC0721C0F690418A426DDC0221C0F2C3
:106C300030418A4254D00421C0F660018A4216D005
:106C4000AAE000BF1F21C1F2F0418A4228DC0721DF
:106C5000C0F690418A4245DC0221C0F230418A42AE
:106C60003ED00421C0F660018A4240F08B80402172
:106C7000C1F620119BE000BF002198E040F2FF71B7
:106C8000C2F630618A4253DC2021C1F2F0418A42CF
:106C900034D040F20041C2F600218A4211D07BE09C
:106CA00040F2FF71C2F630618A4253DC2021C1F20A
:106CB000F0418A4222D040F20041C2F600218A42CD
:106CC00060D140F60001C2F6306170E00721C0F6E5
:106CD00090418A4206DC0221C0F230418A42C0D192
:106CE000012164E00821C0F690418A421CD01021A5
:106CF000C1F2C0018A4211D044E000BF40F200213D
:106D0000C2F2B05153E000BF0821C0F690418A4260
:106D10000AD01021C1F2C0018A423DD140F20011D7
:106D2000C2F2801143E000BF8021C1F650513EE025
:106D300040F60001C2F630618A421DD042F20001E5
:106D4000C3F290618A4227D144F20001C3F6C02108
:106D50002DE000BF40F60001C2F630618A420BD040
:106D600041F20001C3F260218A420BD142F20001DC
:106D7000C3F290611BE000BF41F20001C3F2602149
:106D800015E000BF00240021C4F68434A24204BFF1
:106D90000021C4F6B8710AE044F200040021C3F6F1
:106DA000C024A24204BF48F20001C3F6F06173455B
:106DB00012D091FAA1F44FF6C135B4FA84F4C0F2BE
:106DC0000A05294208BF8C0E04F01F01012404FAB1
:106DD00001F1DC692143D961B2F1FF3F02DD0021FD
:106DE00051E000BF42F2000142F20016C4F202017B
:106DF000C4F2020601F5807401F54275A3426446AF
:106E000008BF2C468B4208BF2C4643F48075B54220
:106E100025682BD18C68D1F808112143C9072DD1E1
:106E2000002105F0E074CCF252718A4208BF15F4DB
:106E300000012FD00021CCF221318A4208BF15F089
:106E400080712BD00021CCF684318A424FF00001B2
:106E500019D115F4800208BF734514D1DCF8001075
:106E600021F0E071214341F4800156E04FF60051DA
:106E7000CFF6FF715CF80110C907D1D0016E41F067
:106E8000200101660121002280F85C20084601B043
:106E9000BDE8F081734505D00021F4E7734535D096
:106EA0000021F0E7DCF8001042F6635221F0E071B7
:106EB000C0F23E52214341F40001CCF8001040F2F0
:106EC0000C01C2F2004109688909A1FB0212910973
:106ED000022202EB41010091009919B30099013996
:106EE0000091009901B30099013900910099E9B12D
:106EF0000099013900910099D1B1009901390091AF
:106F0000009900294FF00001E8D1BCE7DCF800103F
:106F100021F0E071214341F08071CCF80010002194
:106F2000B1E700BF0021AEE70021ACE70021AAE7EE
:106F30000021A8E7000000007047000000000000EA
:106F400070470000000000002DE9F04F81B046F2CC
:106F5000083942F2000804460068C5F60209C4F286
:106F6000020808F5807B08F542774A4601685845D3
:106F700008BF3A464045436808BF3A4603EA010560
:106F8000A90716680CD5206EC00603D4206E40F405
:106F9000006020662046FFF7EFFB206802210160B9
:106FA00015F00C0F06F01F0A44D0216EC90603D459
:106FB000216E41F400712166C16811F4406F33D134
:106FC0000146584508BF4146814218BF0946BAF1FB
:106FD000000F08BF0146BAF1050F08BF0146BAF11C
:106FE000090F08BF0146C96889041DD40168090753
:106FF0001AD5816849070FD4416821F00C0141601E
:10700000206E20F480702066206EC0040CD4206EA8
:1070100040F00100206607E0206E40F0100020667E
:10702000606E40F0010060662046FFF785FF206833
:107030000C21016015F0600F22D0216EC90603D427
:10704000216E41F4005121660146584508BF414672
:1070500006F01E02814218BF0946BAF1000F08BFB0
:107060000146062A08BF0146C26C12F4C07FC268FE
:10707000C9686BD02046FFF783FB20686021016060
:1070800029060BD4E90515D4A90520D4E9062BD48B
:10709000690549D401B0BDE8F08F00BF206E40F40F
:1070A00080302066204600F003FA206880210160CD
:1070B000E905E9D5206E40F4003020662046FFF750
:1070C00067FB20684FF480710160A905DED5206E52
:1070D00040F4802020662046FFF75EFB20684FF4D6
:1070E00000710160E906D3D5E16B69B1BAF1000F17
:1070F00052D0584508BFB946404508BFB946D9F8EF
:10710000001011F4404F0BD0206E40F480602066D8
:10711000606E40F0020060662046FFF711FF2068B5
:10712000102101606905B5D5216E41F480412166C9
:10713000616E41F0080161664FF480610160204694
:1071400001B0BDE8F04FFFF71FBB00BF8B0106D5B4
:1071500002F4406201F40053D2187FF48BAF89022D
:1071600001683FF587AF11F040013FF483AF8168BC
:10717000090715D4416821F060014160206E20F4B8
:1071800080502066206EC0053FF574AF206E40F041
:10719000010020666EE700BFC1688907B4D1BFE770
:1071A000206E40F010002066606E40F001006066C6
:1071B00060E7000000000000B0B582B0044600287F
:1071C0004FF00000019009D0206E58B1206881680E
:1071D000890012D48168C90019D54EE001252846DE
:1071E00002B0B0BD204600F067F90020606684F868
:1071F0005C00206881688900ECD54FF6C072816818
:10720000C5F6FF72114081608168C90035D44FF620
:10721000C0718268C5F6FF7101F18051114042F6DC
:10722000635201F18051816040F20C01C0F23E5284
:10723000C2F2004109688909A1FB0212012101EB98
:10724000921101910199C1B10199013901910199FD
:1072500000291FBF01990139019101991FBF002920
:107260000199013901911CBF0199002905D00199AB
:107270000139019101990029E6D18168C90009D439
:10728000216E012541F010012166616E41F001017E
:10729000616600E000258168226E02F01002C1F3F1
:1072A00080018918216E07D041F010000125206669
:1072B000284602B0B0BD00BF21F4817146F2100C27
:1072C000023121668168C5F6020CC90724D142F259
:1072D000001240F48071C4F20202914242F20001B5
:1072E000C4F2020140F0A0808A68D1F808311A4344
:1072F000D20711D101F5807201F5427390421A460E
:1073000018BF0CF53E72884208BF1A4661681368C0
:1073100023F47C1319431160617EE36BACF1100E12
:10732000704543EA413121D0A268114394F82020EE
:10733000012A41EA024306D1616A0022CFF6FE72B9
:1073400002EB41410B43A16A29B101F47871E26A71
:10735000194341EA0203704516D04CF20302C1689A
:10736000CFF6F07211401943C1601FE0D4E9023238
:10737000082B41EA02015DD00C2B5FD01C2B61D1A0
:1073800010231943D2E700BF44F207025CF8041C43
:10739000CFF6F072114019434CF8041CDCF80010D1
:1073A000626B21F040611143CCF800108168826863
:1073B000D20842EA9101C90765D1217E70454FEAA2
:1073C000813103D0226B114304E000BF94F83820D0
:1073D00041EA4201C26844F203039A431143C16087
:1073E00094F84410012919D14FF61E017045CFF6CB
:1073F00000412DD0026902EA010C0021D4E91223D8
:10740000CFF6FF7101EB02414CEA0302236D1143F9
:10741000626D1943114341F0010102E0016921F05D
:107420000101016123E000BF5CF8082CD2073FF4A2
:1074300061AF71E70023194378E700BF08231943C0
:1074400074E700BF182B18BF002319436EE700BF75
:10745000DCF800201140D4E912231143226D1943B6
:10746000636D1143194341F00101CCF8001001692B
:10747000226C21F07041704541EA0201016102D0A5
:107480002046FAF7DDF920682169026B012922F014
:107490000F0102D1E269013A114301630121206E1B
:1074A00061F301002066284602B0B0BD0000000074
:1074B00070470000000000002DE9F04186B004464E
:1074C00046F20002C5F602020020216805909142B2
:1074D000049067D042F20000C4F20200814240F002
:1074E000948044F2E0400025C5F60200C5F602058E
:1074F00001AE4FF0030850F8081C002741F02001AE
:1075000040F8081C50F8081C01F020010091009977
:10751000016841F001010160016801F00101009181
:107520000099016841F0040101600068314600F0F3
:10753000040000900098202001902846CDF8088093
:10754000039702F049FE10203146CDE9010805F508
:107550000060039702F040FE41F678751020C2F2F9
:107560000045C4F2020028600920C5E901074FF474
:10757000806028614FF4006068614FF40050A8619A
:107580004FF48070EF60C5E9070728466F6201F08D
:107590005BF808B1FEF7F8FAA565AC6306B0BDE884
:1075A000F08100BF44F2E04141F6F075C5F60201FA
:1075B000C2F200450A6842F080720A600A6801F669
:1075C000287102F080720092009A29601121E8600F
:1075D000C5E901104FF4806129614FF400616961D0
:1075E0004FF400512862C5E90610284601F02CF836
:1075F00008B1FEF7C9FA7F2005210022A565AC631A
:1076000002F0C6FF7F2002F0B3FF06B0BDE8F081B4
:107610002DE9F041044602F0E3FE0CB3054694F870
:107620003500022820D140F20F472668C4F2020735
:1076300040F26F48BE42C4F202081DDC6F20C4F263
:10764000020086422ADC3F20C4F20200864241DC6E
:107650001020C4F20200864263D028205CE000BF04
:107660000120BDE8F08100BF80206065012000217D
:1076700084F83410BDE8F08146451BDC40F23F4001
:10768000C4F2020086422DDC40F21040C4F2020037
:10769000864246D040F228403EE000BF9F20C4F220
:1076A0000200864228DC7020C4F20200864238D0F4
:1076B000882031E040F29F40C4F20200864223DC81
:1076C00040F27040C4F2020086422AD040F2884064
:1076D00022E000BF4020C4F20200864221D05820A0
:1076E0001AE000BF40F24040C4F20200864218D0C7
:1076F00040F2584010E000BFA020C4F202008642D1
:107700000FD0B82008E000BF40F2B840C4F2020039
:10771000864206D040F2A040C4F20200864240F009
:1077200099813146306820F01E0041F8140B6FF04B
:1077300080000A68464500EA020008601ADC9F20C3
:10774000C4F20200864233DC5720C4F202008642B3
:107750005ADC1020C4F20200864200F097802820F4
:10776000C4F20200864200F091804020C4F2020080
:107770008AE000BF45F22F40C5F6020086422DDCAC
:1077800040F2B740C4F2020086424BDC40F2704047
:10779000C4F20200864279D040F28840C4F202006E
:1077A000864273D040F2A040C4F202006CE000BFF9
:1077B00040F22740C4F20200864243DCA020C4F21B
:1077C0000200864262D0B820C4F2020086425DD038
:1077D00040F21040C4F2020056E000BF45F26B4098
:1077E000C5F6020086423FDC45F23040C5F6020095
:1077F00086424BD045F24440C5F60200864245D051
:1078000045F258403EE000BF5820C4F202008642D4
:107810003CD07020C4F20200864237D08820C4F2E7
:10782000020031E040F2B840C4F2020086422DD09E
:1078300045F20840C5F60200864227D045F21C40BA
:1078400020E000BF40F22840C4F2020086421DD072
:1078500040F24040C4F20200864217D040F2584045
:10786000C4F2020010E000BF45F26C40C5F6020011
:1078700086420BD045F29440C5F60200864205D000
:1078800045F28040C5F60200864204D1206E0168B0
:1078900021F480710160306820F00100306000BF89
:1078A0003068C00710D002F09BFD401B0628F7D3BC
:1078B00020206065032084F835000120002184F831
:1078C0003410BDE8F08100BF2068B84210DC6F21A1
:1078D000C4F2020188421DDC3F21C4F20201884249
:1078E00034DC1021C4F20201884255D028214FE037
:1078F00040451BDC40F23F41C4F2020188422DDCCE
:1079000040F21041C4F20201884245D040F22841C1
:107910003EE000BF9F21C4F20201884228DC7021B2
:10792000C4F20201884237D0882131E040F29F4101
:10793000C4F20201884223DC40F27041C4F2020129
:10794000884229D040F2884122E000BF4021C4F2A1
:107950000201884220D058211AE000BF40F2404185
:10796000C4F20201884217D040F2584110E000BF33
:10797000A021C4F2020188420ED0B82108E000BF65
:1079800040F2B841C4F20201884205D040F2A04161
:10799000C4F20201884261D1D4E9161202F01F023A
:1079A0003F2303FA02F28A60404561DC9F21C4F262
:1079B0000201884214DC5721C4F20201884227DC0C
:1079C0001021C4F20201884200F0A8802821C4F2EC
:1079D0000201884200F0A2804021C4F202019BE033
:1079E00040F22741C4F20201884221DCA021C4F206
:1079F0000201884200F09280B821C4F2020188425C
:107A000000F08C8040F21041C4F2020184E000BF1B
:107A10005821C4F20201884200F080807021C4F233
:107A2000020188427AD08821C4F2020174E000BFCA
:107A300040F22841C4F2020188426FD040F2404136
:107A4000C4F20201884269D040F25841C4F20201F6
:107A500062E000BF6FF00E0031466AE6D4E916120C
:107A600002F01F02012303FA02F24A6040459DDD45
:107A700045F22F41C5F60201884217DC40F2B741BA
:107A8000C4F20201884227DC40F27041C4F20201D4
:107A9000884243D040F28841C4F2020188423DD07E
:107AA00040F2A041C4F2020136E000BF45F26B4152
:107AB000C5F6020188421FDC45F23041C5F60201DD
:107AC00088422BD045F24441C5F60201884225D0B8
:107AD00045F258411EE000BF40F2B841C4F2020135
:107AE00088421BD045F20841C5F60201884215D0F4
:107AF00045F21C410EE000BF45F26C41C5F60201A3
:107B000088420BD045F29441C5F60201884205D067
:107B100045F28041C5F6020188420BD1616EA26E2A
:107B2000E06E4A6030B1016821F480710160D4E9EF
:107B30001C014160012084F835000020002184F8F8
:107B40003410BDE8F081000080B5D8B190F8351050
:107B5000022919D140F20F420168C4F20202914297
:107B600016DC6F23C4F20203994227DC3F23C4F2E0
:107B7000020399423EDC1023C4F2020399425FD013
:107B8000282359E0012080BD80214165012080BD6E
:107B900040F26F43C4F2020399421BDC40F23F43C0
:107BA000C4F2020399422DDC40F21043C4F20203F6
:107BB000994245D040F228433EE000BF9F23C4F2E3
:107BC0000203994228DC7023C4F20203994237D0A1
:107BD000882331E040F29F43C4F20203994223DC40
:107BE00040F27043C4F20203994229D040F2884324
:107BF00022E000BF4023C4F20203994220D0582360
:107C00001AE000BF40F24043C4F20203994217D089
:107C100040F2584310E000BFA023C4F2020399428F
:107C20000ED0B82308E000BF40F2B843C4F202030C
:107C3000994205D040F2A043C4F20203994275D1A3
:107C400091424FF0040280F8352011DC6F20C4F21D
:107C50000200814222DC3F20C4F20200814239DC72
:107C60001020C4F20200814259D0282054E000BF05
:107C700040F26F40C4F2020081421BDC40F23F4000
:107C8000C4F2020081422DDC40F21040C4F2020036
:107C9000814244D040F228403EE000BF9F20C4F221
:107CA0000200814228DC7020C4F20200814236D0FA
:107CB000882031E040F29F40C4F20200814223DC80
:107CC00040F27040C4F20200814228D040F2884065
:107CD00022E000BF4020C4F2020081421FD05820A1
:107CE0001AE000BF40F24040C4F20200814216D0C8
:107CF00040F2584010E000BFA020C4F202008142D0
:107D00000DD0B82008E000BF40F2B840C4F2020035
:107D1000814204D040F2A040C4F2020081420868CF
:107D200020F001000860002080BD00BF0A6822F03A
:107D30000E020A6045F25742C5F6020291420A68F5
:107D400022F001020A600FDC45F22F42C5F6020262
:107D5000914219DC45F20842C5F60202914229D04F
:107D600045F21C4222E000BF45F27F42C5F6020206
:107D7000914213DC45F25842C5F60202914219D0F5
:107D800045F26C4212E000BF45F23042C5F60202F5
:107D900091420FD045F2444208E000BF45F29442C0
:107DA000C5F60202914205D045F28042C5F60202B4
:107DB00091421AD1D0E9181CD0E916E30A6822F4DE
:107DC00080720A6003F01F01012202FA01F1CEF86D
:107DD0000410816ECCF80410C16E31B10A6822F42F
:107DE00080720A60D0E91C124A60012180F83510C7
:107DF000026D002180F834100AB190470021084636
:107E000080BD000000000000406D704700000000D1
:107E10002DE9F04782B00021019140F20C010446A7
:107E2000C2F2004148F2B512C1F64E32A56D0968A2
:107E300040F26F490068C4F20209A1FB02184845EC
:107E40002E68296816DC9F21C4F2020188422DDCCD
:107E50005721C4F20201884252DC1021C4F202010F
:107E600088427BD02821C4F20201884276D040218A
:107E700070E000BF45F22F42C5F60202904229DCB5
:107E800040F2B742C4F20202904245DC40F2704137
:107E9000C4F20201884261D040F28841C4F202017A
:107EA00088425BD040F2A04154E000BF40F227413D
:107EB000C4F2020188423FDCA021C4F202018842E0
:107EC0004CD0B821C4F20201884247D040F21041A0
:107ED00040E000BF45F26B42C5F60202904275DCFD
:107EE00045F23042C5F60202904200F0818045F230
:107EF0004442C5F6020290427AD045F2584273E0FD
:107F00005821C4F20201884228D07021C4F2020133
:107F1000884223D088211DE040F2B842C4F2020218
:107F200090421BD045F20842C5F6020290425FD053
:107F300045F21C4258E000BF40F22841C4F2020161
:107F400088420BD040F24041C4F20201884205D081
:107F500040F25841C4F20201884261D1E16D082229
:107F600001F01F0140F20F4A8A40C4F2020A324275
:107F700000F0E98050454FF0040313DC6F27C4F292
:107F80000207B8426CDC3F27C4F20207B84200F394
:107F9000A7801027C4F20207B84200F0C880282743
:107FA000C0E000BF484567DC40F23F47C4F202072B
:107FB000B84200F39D8040F21047C4F20207B84275
:107FC00000F0B58040F22847ACE000BF45F26C42BB
:107FD000C5F6020290420BD045F28042C5F602027D
:107FE000904205D045F29442C5F60202904217D164
:107FF0000268E36D570703F01F0315D504279F4060
:1080000017EA010610D011046F6045D4910603D41D
:10801000016821F004010160216C002940F0F68222
:1080200002B0BDE8F08700BF97073DD502279F400B
:1080300017EA010638D011046F6000F1ED82910655
:1080400009D4016821F00A010160012084F835009B
:10805000002084F83400E16B002940F0D782DFE78C
:108060009F27C4F20207B8424CDC7027C4F2020713
:10807000B8425CD0882755E040F29F47C4F202071F
:10808000B84247DC40F27047C4F20207B8424ED013
:1080900040F2884746E000BFD00300F1C382A16CE4
:1080A000002940F0B382BBE71207B9D508229A40F5
:1080B0001140B5D0016821F00E010160012000FAE5
:1080C00003F16960606584F835000020E16C84F894
:1080D00034000029A4D02046884702B0BDE8F087CC
:1080E0004027C4F20207B84221D058271AE000BF47
:1080F00040F24047C4F20207B84218D040F2584755
:1081000010E000BFA027C4F20207B8420FD0B82782
:1081100008E000BF40F2A047C4F20207B84206D010
:1081200040F2B847C4F20207B84218BF08230768F4
:108130001F4208D0036823F004030360AA60626D45
:1081400042F00102626501228A4032426FD05045FE
:1081500010DC6F23C4F2020398421DDC3F23C4F2FB
:108160000203984234DC1023C4F20203984256D032
:1081700028234FE048451BDC40F23F43C4F2020392
:1081800098422DDC40F21043C4F20203984246D0DC
:1081900040F228433EE000BF9F23C4F2020398420E
:1081A00028DC7023C4F20203984238D0882331E0DF
:1081B00040F29F43C4F20203984223DC40F2704332
:1081C000C4F2020398422AD040F2884322E000BF62
:1081D0004023C4F20203984221D058231AE000BF82
:1081E00040F24043C4F20203984218D040F2584390
:1081F00010E000BFA023C4F2020398420FD0B823BE
:1082000008E000BF40F2A043C4F20203984206D047
:1082100040F2B843C4F20203984240F00B82436933
:108220001B0604D5AA60626D42F002026265042258
:108230008A4032426FD0504510DC6F23C4F20203F3
:1082400098421DDC3F23C4F20203984234DC102321
:10825000C4F20203984256D028234FE048451BDC65
:1082600040F23F43C4F2020398422DDC40F2104337
:10827000C4F20203984246D040F228433EE000BFD9
:108280009F23C4F20203984228DC7023C4F2020345
:10829000984238D0882331E040F29F43C4F2020371
:1082A000984223DC40F27043C4F2020398422AD081
:1082B00040F2884322E000BF4023C4F20203984208
:1082C00021D058231AE000BF40F24043C4F2020319
:1082D000984218D040F2584310E000BFA023C4F2E7
:1082E000020398420FD0B82308E000BF40F2A04339
:1082F000C4F20203984206D040F2B843C4F202032B
:10830000984240F09F8103689B0704D5AA60626D84
:1083100042F004026265102202FA01F1314200F0DB
:10832000818050454FF0080210DC6F23C4F2020335
:1083300098421DDC3F23C4F20203984234DC102330
:10834000C4F20203984256D028234FE048451BDC74
:1083500040F23F43C4F2020398422DDC40F2104346
:10836000C4F20203984246D040F228433EE000BFE8
:108370009F23C4F20203984228DC7023C4F2020354
:10838000984238D0882331E040F29F43C4F2020380
:10839000984223DC40F27043C4F2020398422AD090
:1083A00040F2884322E000BF4023C4F20203984217
:1083B00021D058231AE000BF40F24043C4F2020328
:1083C000984218D040F2584310E000BFA023C4F2F6
:1083D000020398420FD0B82308E000BF40F2A04348
:1083E000C4F20203984206D040F2B843C4F202033A
:1083F000984218BF04220368134213D0A960016891
:108400004903016808D4C90508D4016821F00801AE
:108410000160216C21B905E008034FD4216C09B13A
:1084200020468847E06D00F01F01202000FA01F28D
:10843000324200F0AB8020681023504510DC6F27DB
:10844000C4F20207B8421DDC3F27C4F20207B8425B
:1084500038DC1027C4F20207B8425AD0282753E06C
:1084600048451BDC40F23F47C4F20207B84231DC0A
:1084700040F21047C4F20207B8424AD040F22847FF
:1084800042E000BF9F27C4F20207B8422CDC7027ED
:10849000C4F20207B8423CD0882735E040F29F473B
:1084A000C4F20207B84227DC40F27047C4F2020768
:1084B000B8422ED040F2884726E000BFA16C0029C8
:1084C000AED1AFE74027C4F20207B84221D0582707
:1084D0001AE000BF40F24047C4F20207B84218D089
:1084E00040F2584710E000BFA027C4F20207B8428C
:1084F0000FD0B82708E000BF40F2A047C4F202073F
:10850000B84206D040F2B847C4F20207B84218BFDA
:10851000022307681F4239D0AA6094F83520042A44
:1085200002681BD122F016020260426922F080022A
:108530004261226C0AB9A26C1AB1026822F00802E8
:1085400002603F208840A860012084F83500216D3A
:108550000020002984F8340058D161E551030168F6
:108560000CD4C9050ED4016821F01001016001206E
:1085700084F83500002084F8340003E0080301D4B7
:10858000616C00E0E16B09B120468847606D00280E
:108590003FF446AD606DC00734D0042084F8350048
:1085A00020684FEA9821026822F001020260019AD5
:1085B000013201928A421AD80268D20717D0019A72
:1085C000013201928A4212D80268D2070FD0019A72
:1085D000013201928A420AD80268D20707D0019A72
:1085E000013201928A4202D80268D207DFD10068C4
:1085F000C0074FF0030008BF012084F835000020B9
:1086000084F83400E16C00293FF40AAD2046884725
:1086100002B0BDE8F08700BFD00307D4616C002929
:10862000F4D1FDE4216C0029F0D1F9E4E16B0029DB
:10863000ECD1F5E4026804228A4032427FF4FBADBB
:1086400069E600BF026866E62DE9F04381B00446A2
:1086500001F0C6FE002C00F0128140F26F48054682
:108660002068C4F20208404516DC9F21C4F20201D2
:1086700088422DDC5721C4F20201884254DC1021CB
:10868000C4F20201884200F07E802821C4F2020177
:10869000884278D0402171E045F22F41C5F60201B1
:1086A000884229DC40F2B741C4F20201884247DC2B
:1086B00040F27041C4F20201884264D040F2884125
:1086C000C4F2020188425ED040F2A04156E000BFF1
:1086D00040F22741C4F20201884241DCA021C4F2E9
:1086E000020188424FD0B821C4F2020188424AD028
:1086F00040F2104142E000BF45F26B41C5F6020175
:10870000884200F3C18045F23041C5F6020188423B
:1087100000F0CD8045F24441C5F60201884200F0E8
:10872000C68045F25841BDE05821C4F2020188429A
:1087300029D07021C4F20201884224D088211DE092
:1087400040F2B841C4F2020188421CD045F208410F
:10875000C5F60201884200F0AA8045F21C41A1E062
:1087600040F22841C4F2020188420CD040F240415C
:10877000C4F20201884206D040F25841C4F202011C
:10878000884240F09782022184F83510002184F855
:108790003410016821F0010101600168C90708D0A7
:1087A00001F01EFE401B052864D820680168C90737
:1087B000F6D148F23F0204F108060168CFF61062D4
:1087C0001140D4F818C06CCE1143D4F8249019434A
:1087D000E3692943256A0E43B9F1040F46EA0C0602
:1087E00043EA060343EA050303D1D4E90B653343A7
:1087F0002B43666843F48011A6F13F07A6F12905D3
:10880000042FA6F1470238BF0B46062DA6F14F0EE6
:1088100038BF0B46022A26F0030238BF0B46BEF1D2
:10882000040F38BF0B46742A08BF0B46B9F1040F7A
:108830000360416921F0070141EA090140F0F48039
:10884000D4E90A53002B41EA050100F0ED80BCF5A4
:10885000005F00F0CF80BCF1000F40F0D780022D08
:1088600000F0D780012D00F0CB80002D00F0D180EA
:10887000DAE000BF20206065032084F83500012085
:1088800001B0BDE8F08300BF45F26C41C5F60201BE
:1088900088420CD045F28041C5F60201884206D0DC
:1088A00045F29441C5F60201884240F0038202215C
:1088B00084F83510002184F834100168A268A2F110
:1088C0008003E768B3FA83F3402A4FEA53134FEA71
:1088D00083336FF3101108BF1023226941EAD701D7
:1088E00067691943A36941EAD201E26941EAD70104
:1088F00041EAD3014CF6CD4341EAD2014AF6F832BF
:10890000CAF2FD72276A0244CCF6CC43A2FB0323D1
:1089100041EA171101606FF0030000EA9300E0657F
:108920002046FCF7A9FDE16D012201F01F0102FACA
:1089300001F141602068404540F3858045F22F41B8
:10894000C5F60201884217DC40F2B741C4F20201C9
:10895000884229DC40F27041C4F20201884200F0F2
:10896000BC8040F28841C4F20201884200F0B58028
:1089700040F2A041ACE000BF45F26B41C5F60201F8
:10898000884223DC45F23041C5F60201884200F0FE
:10899000A48045F24441C5F60201884200F09D8062
:1089A00045F2584122E000BF40F2B841C4F2020152
:1089B000884200F0928045F20841C5F602018842E3
:1089C00000F08B8045F21C4110E000BF45F26C4185
:1089D000C5F60201884200F0808045F29441C5F658
:1089E0000201884200F0798045F28041C5F602011B
:1089F00070E000BF032D17D8DFE805F00E0B0E0264
:108A0000A3F1C072B2FA82F2520904E0032D03D33B
:108A10000AD1C3F300623AB140206065012084F8B6
:108A2000350001B0BDE8F08341612046FCF724FD2C
:108A3000E16D3F2201F01F0102FA01F1816020681F
:108A400040453FF77BAF9F21C4F20201884211DC11
:108A50005721C4F20201884220DC1021C4F2020135
:108A600088423AD02821C4F20201884235D0402100
:108A70002EE000BF40F22741C4F20201884219DC17
:108A8000A021C4F20201884227D0B821C4F2020119
:108A9000884222D040F210411AE000BF5821C4F2AF
:108AA0000201884219D07021C4F20201884214D018
:108AB00088210DE040F22841C4F2020188420CD026
:108AC00040F24041C4F20201884206D040F25841CF
:108AD000C4F20201884240F0E58045F2574C45F669
:108AE000FC0EC5F6020CC5F6020E604512DC45F21E
:108AF0002F41C5F60201884220DC45F20841C5F647
:108B00000201884234D045F21C41C5F60201884278
:108B10002ED085E045F27F41C5F6020188421BDC7C
:108B200045F25841C5F60201884221D045F26C4118
:108B3000C5F6020188421BD072E000BF45F2304109
:108B4000C5F60201884213D045F24441C5F6020140
:108B500088420DD064E000BF45F29441C5F60201A1
:108B6000884205D045F28041C5F60201884257D1BE
:108B70006FF007014CF6CD4251FA80F1CCF6CC42B1
:108B8000A1FB0212AEF1FC05AEF17C061309A2684E
:108B900003F01F01802A4FF0010205EB83052566D3
:108BA00002FA01F26666A26602D10021616000E06D
:108BB0006168CBB2013907292B60726016D85E1E3E
:108BC000082E19D260450EF1440219DC45F22F41FE
:108BD000C5F60201884245DC45F20841C5F60201AE
:108BE000884255D045F21C414EE000BF002060672E
:108BF000C4E91B0056E000BFD4E91B02616F4EE0E0
:108C000045F27F41C5F60201884235DC45F2584104
:108C1000C5F6020188423BD045F26C4134E000BF0A
:108C20006FF00F014AF6AB2251FA80F1CAF6AA2280
:108C3000A1FB021240F20F43C4F2020308251109FE
:108C4000984203F1AA060B4688BF05EB121340F6C3
:108C50000005B042C4F2020505F1800628BF0B46AC
:108C600095E700BF45F23041C5F6020188420FD0BA
:108C700045F2444108E000BF45F28041C5F60201DB
:108C8000884205D045F29441C5F60201884213D1CD
:108C900001210EEB8300B140E0662267616700238B
:108CA0000360516000206065012184F8351001B037
:108CB000BDE8F0834020DEE540F60000C4F202008B
:108CC00000F1FC0E00F5A072E2E7000000000000D9
:108CD000B0B500283CD0054690F83400012801D1F9
:108CE0000220B0BD012085F8340095F83500012838
:108CF00028D1022085F835000020686528680468BE
:108D000024F0010404602846FCF74EFC40F20F42B8
:108D10002868C4F2020240F26F419042C4F202019C
:108D200018DC6F23C4F20203984225DC3F23C4F20F
:108D3000020398423CDC1023C4F2020398425ED046
:108D4000282357E04FF400606865002085F8340060
:108D50000120B0BD88421BDC40F23F43C4F2020355
:108D600098422DDC40F21043C4F20203984246D0F0
:108D700040F228433EE000BF9F23C4F20203984222
:108D800028DC7023C4F20203984238D0882331E0F3
:108D900040F29F43C4F20203984223DC40F2704346
:108DA000C4F2020398422AD040F2884322E000BF76
:108DB0004023C4F20203984221D058231AE000BF96
:108DC00040F24043C4F20203984218D040F25843A4
:108DD00010E000BFA023C4F2020398420FD0B823D2
:108DE00008E000BF40F2B843C4F20203984206D044
:108DF00040F2A043C4F20203984240F02F8103687E
:108E00000B2464F3440303602B6C1BB1036843F031
:108E100008030360884219DC9F23C4F202039842CE
:108E200032DC5723C4F20203984259DC1023C4F207
:108E30000203984200F096802823C4F2020398426D
:108E400000F090804023C4F2020389E045F22F43F2
:108E5000C5F6020398422DDC40F2B743C4F2020388
:108E600098424BDC40F27043C4F20203984279D03E
:108E700040F28843C4F20203984273D040F2A04308
:108E8000C4F202036CE000BF40F22743C4F20203C5
:108E9000984243DCA023C4F20203984262D0B82374
:108EA000C4F2020398425DD040F21043C4F20203C0
:108EB00056E000BF45F26B43C5F6020398423FDC23
:108EC00045F23043C5F6020398424BD045F2444385
:108ED000C5F60203984245D045F258433EE000BF34
:108EE0005823C4F2020398423CD07023C4F2020318
:108EF000984237D08823C4F2020331E040F2B843ED
:108F0000C4F2020398422DD045F20843C5F602038D
:108F1000984227D045F21C4320E000BF40F228438E
:108F2000C4F2020398421DD040F24043C4F202034F
:108F3000984217D040F25843C4F2020310E000BF39
:108F400045F26C43C5F6020398420BD045F29443B8
:108F5000C5F60203984205D045F28043C5F60203E8
:108F6000984274D12B6E1C68E40303D51C6844F44A
:108F700080741C60EB6E1BB11D6845F480751D602C
:108F8000904211DC6F21C4F2020188421EDC3F21B5
:108F9000C4F20201884235DC1021C4F20201884289
:108FA00055D0282150E000BF88421BDC40F23F41F1
:108FB000C4F2020188422DDC40F21041C4F20201E9
:108FC000884244D040F228413EE000BF9F21C4F2D5
:108FD0000201884228DC7021C4F20201884236D0A6
:108FE000882131E040F29F41C4F20201884223DC33
:108FF00040F27041C4F20201884228D040F2884118
:1090000022E000BF4021C4F2020188421FD0582153
:109010001AE000BF40F24041C4F20201884216D07B
:1090200040F2584110E000BFA021C4F20201884282
:109030000DD0B82108E000BF40F2B841C4F20201EF
:10904000884204D040F2A041C4F202018842016883
:1090500041F0010101600020B0BD00BF036805249C
:1090600064F3430303602B6C002B3FF4D3AE03681F
:1090700043F00403CDE60000B0B5044601F0B0F9BA
:1090800040F204010546C2F20041621C097818BF93
:109090000C4400BF01F0A4F9401BA042FAD3B0BDBC
:1090A00090F89830013B012B0ED80068836D0B427D
:1090B00012D0836D0B408B4216D1C36D43F0020377
:1090C000C3658B0514D418E000F19C010120022235
:1090D0000B681A430A607047C36D43F00103C36510
:1090E0008B0505D409E000BF0323C3658B0504D5B8
:1090F000D0F8E0301343C0F8E0304B0504D5D0F889
:10910000E4301A43C0F8E4204FF6FF72436DC3F613
:10911000CF720A401A4342658A0F4AF614010020B2
:10912000C4F200010B681A430A6070470000000097
:109130002DE9F04390F89830022B19D10668D6F843
:10914000C03013F07C5F1DD0D6F8C4309B0223D40E
:10915000D6F8C4304D68002D0D69C3F3044C8B68FC
:1091600024D00C682B43234343F0804E22E000BF01
:10917000D0F89C1041F00801C0F89C100120BDE817
:10918000F08300BFD0F89C1041F02001C0F89C1083
:109190000120BDE8F08300BFD0F89C1041F40071BD
:1091A000C0F89C100120BDE8F08300BF0C682B4381
:1091B00043EA844E836ED0F88450D1E907970CFBC4
:1091C00003F48B6949EA0767D1F81480D1F80C9051
:1091D0001F4305EB840347EA080745F824E047EA04
:1091E00009475F60CF6887B14EF2780508330332D4
:1091F0000024C0F6010500BF171957F8037C1F5162
:10920000CF680434EF5DBC42F6D3012101FA0CF1C2
:10921000C6F8D010C0F894100020BDE8F08300001C
:10922000704700000000000080B590F89820013AD7
:10923000012A0BD80A68002ACA680FD00B69072ACE
:1092400043EA427E18D18B691BE000BFD0F89C1026
:1092500041F00201C0F89C10012080BD072A19D1FD
:109260000A69D1F81CC012048B6942EA0C221A4325
:1092700042F0605218E000BFD1F808C04B6943EAE1
:109280008C73006F496800EBC10240F831E00020A8
:10929000536080BD8B68D1F810C09B0743EAC2625F
:1092A0004B6942EA0C421A434968C06E40F82120DB
:1092B000002080BD0000000090F898C0BCF1010FB4
:1092C0000ED19200006842EA0111DDF800C041EAC7
:1092D000430141EA0C01C0F880100020704700BF34
:1092E000D0F89C1041F00401C0F89C100120704798
:1092F00010B34AF200010068C4F2000188420FD0A6
:109300004DF20041C4F2000188420BD04AF2004104
:10931000C4F20001884218BF7047012003E000BF7B
:10932000002000E0022041F2F011C2F2004101EB06
:109330004010C06A00B10047704700000000000004
:109340007047000000000000B422402908BFA4229A
:109350000068805800F07F007047000000000000A7
:109360002DE9F04390F89870022F11D1402919D1BE
:109370000668D6F8A07017F4FE0F2FD0D6F8A470A8
:109380007F0635D0D6F8A470FF013BD400273CE01F
:10939000D0F89C1041F00801C0F89C100120BDE8F5
:1093A000F08300BF41290FD10668D6F8B07017F4DA
:1093B000FE0F13D0D6F8B4707F0619D0D6F8B4706B
:1093C000FF012BD400272CE0076D8F4206D900F156
:1093D0007C04456D4FF0000C0E462BE0D0F89C103D
:1093E00041F02001C0F89C100120BDE8F08300BFCF
:1093F000D0F89C1041F48071C0F89C100120BDE8A9
:10940000F08300BFD6F8A070FF0FD6F8A46000F17B
:109410007404C6F30526F519466C0AE0D6F8B07058
:10942000FF0FD6F8B46000F17804C6F30526F519ED
:10943000C66CAC467543246804EB850E54F8257061
:1094400017F08047576054F8257027F0604608BF32
:10945000C7F38A46166054F8257007F000579760E6
:1094600054F8254004F000441461BEF80440D4616F
:10947000BEF8064014F00F04D460DEF8044004F493
:1094800080145461DEF8044004F4001494619EF8E2
:10949000074004F07F041462DEF804404FEAD474FD
:1094A000546229D04EF278080024C0F6010800BFAB
:1094B0000EEB0406651C377A1F55D76818F807703D
:1094C000BD423FBF1F19757A7D70D5683EBF18F841
:1094D0000590A51C4D450FD2B57ABD70D56818F81A
:1094E0000590E51C4D4507D2F57A0434FD70D5682A
:1094F00018F80550AC42DBD3402905D10068C0F80C
:10950000A8C00020BDE8F083412905D10068C0F85B
:10951000B8C00020BDE8F0831F2909D800680122E7
:1095200002FA01F1C0F898100020BDE8F08300BFF6
:10953000006801F01F01012202FA01F1C0F89C103D
:109540000020BDE8F083000080B590F89820022A42
:1095500040D10268D2F8F03013F47C1F42D0D2F828
:10956000F4309B0646D0D2F8F430D0F88000C3F334
:10957000042C50F83C3013F080434B6050F83CE032
:109580002EF0604308BFCEF38A430B6050F83C30A6
:1095900003F000538B6000EBCC0350F83C0000F06C
:1095A000004008619888C861D88800F00F00C86042
:1095B000586800F480104861586800F40010886111
:1095C000586800F440004862D87908620020C2F868
:1095D000F8C080BDD0F89C1041F00801C0F89C1084
:1095E000012080BDD0F89C1041F02001C0F89C10F3
:1095F000012080BDD0F89C1041F48071C0F89C100F
:10960000012080BD000000000068D0F8C40000F018
:109610003F0070470000000070470000000000009D
:109620002DE9F04F87B004464AF61000C4F200005E
:1096300001684AF61400C4F200000268206802EAD9
:10964000010A056DD0F85490076DD0F85480036D71
:109650000293436D0193036D0693436D0593036D70
:109660000493436D0393436D066D06EA030B5FEAB3
:10967000CB530BD54FF4807101654AF610010020E1
:10968000C4F2000108602046FFF7C6FF05EA09069C
:109690004AF610095FEA4B50C4F200094FEA8A7596
:1096A0000ED52068D0F8DC10D0F8E42011404FF43B
:1096B000806202650020C9F80000204600F0A8FC86
:1096C00008EA070806F4704655B1206800210165D4
:1096D0000AF00300C9F8000020462946FFF7A0FD64
:1096E000DDE9011000EA010708F00F0546B1206826
:1096F000314606650020C9F80000204600F0D8FC7D
:1097000007F0F00645B12068294605650020C9F834
:109710000000204600F0F8FB46B12068314606659F
:109720000020C9F80000204600F016FC5FEA0B504C
:1097300000F1B6805FEA8B5000F1C0805FEA0B3029
:1097400000F1CF805FEACB3000F1D9805FEA4B3087
:10975000DDE9031000EA010509D520684FF48021F6
:1097600001650020C9F80000204600F049FC5FEACE
:109770008B30DDE9051000EA010005F060710CD5C1
:1097800022684FF4003313650022C9F80020D4F892
:109790009C2042F08002C4F89C2000F0715539B141
:1097A000206801650020C9F800002046FFF7C8FDC9
:1097B000206845B105650021C9F80010D4F89C1057
:1097C0002943C4F89C10A9F5016188425ED1606804
:1097D000816889075AD0016A426A036A476A114060
:1097E00003EA070202F03005D0F82080D0F8249078
:1097F000026A049211F00F01D0F824B0026A0692B6
:10980000426A0592466AD0F820A003D00162204641
:1098100000F0EAFB08EA09072DB1606829460562F5
:10982000204600F0E9FB06EA0A0007F4C07540068E
:10983000049800EA0B060AD560684023C16BC26B2E
:10984000090C02F03F020362204600F0D1FBDDE983
:10985000051000EA010706F4FC462DB160682946B0
:109860000562204600F0BCFB07F4F02036B16168C9
:109870000E62D4F89C103143C4F89C1030B161687A
:109880000862D4F89C100843C4F89C00D4F89C00EB
:10989000002847D0204607B0BDE8F04FFFF728BDAD
:1098A00020684FF4006101650020C9F800002046DF
:1098B00000F026FC5FEA8B507FF540AF2068D0F8BF
:1098C000D810D0F8E02011404FF40072026500205B
:1098D000C9F80000204600F0C3FB5FEA0B307FF5BB
:1098E00031AF20684FF4002101650020C9F8000065
:1098F000204600F005FB5FEACB307FF527AF2068FC
:109900004FF4803101650020C9F80000204600F0C6
:109910007BFB5FEA4B30DDE9031000EA01053FF510
:109920001CAF24E707B0BDE8F08F00000000000086
:109930002DE9F04F85B0A8B34AF200080446C4F2FE
:1099400000080068404531D094F89810A9B38169A7
:1099500021F01001816100F043FD05462068816916
:10996000090705D500F03CFD401B0B28F6D310E09D
:10997000816941F00101816100F032FD054600BFBF
:1099800020688169C90721D100F02AFD401B0B28FE
:10999000F6D3D4F89C0040F00100C4F89C000320EA
:1099A00084F89800012005B0BDE8F08F08F58071BB
:1099B000616094F898100029C9D1002084F89900BA
:1099C000204600F0B9F92068C1E700BF816941F085
:1099D00002018161217C826922F04002012918BFC5
:1099E00040328261617C826922F48042012908BF91
:1099F00002F580428261A17C826922F480520129B1
:109A000018BF02F580528261816921F44073D4E964
:109A100002120B438361836923F0A403836103690A
:109A200023F010030361AAB1022A0FD0012A03D147
:109A3000826942F004020CE08369032A43F0800348
:109A40008361036943F01002026103D1826942F02D
:109A500020028261D4E90572E369561E6FF0FF02AD
:109A6000256A02EB0323B1F5407F43EA4663A5F183
:109A7000010646EA030640F20003CFF6FF7303EB4C
:109A8000074746EA0701C16110D1D4E90B65D4E963
:109A90000917013F02EB06226FF00F063A4306EB6F
:109AA00005173A4303EB01411143C160236E2BB10B
:109AB000616ED0F8C0201143C0F8C010E16DCDE94F
:109AC0000313D9424DF63851C0F6010109D0D0F840
:109AD000C820A36E22F0070251F823301A43C0F8C1
:109AE000C820D4F840A0BAF1000F09D0D0F8BC20AB
:109AF000636C22F0070251F823301A43C0F8BC20EF
:109B0000A76C57B1D0F8BC20E36C22F0700251F87A
:109B1000233042EA0312C0F8BC20D4F850C0BCF194
:109B2000000F0AD0D0F8BC20636D22F4E06251F837
:109B3000231042EA0121C0F8BC10404504D16168FD
:109B40008A6822F003028A600021C4F89410C4F8E5
:109B50009C10012184F898104FF6FC72D0F8841004
:109B6000D4F83C9021EA0203656CD4E90D1202920C
:109B7000019543EA8103C0F88430D0F8843023F49F
:109B80007F0343EA0243C0F884305318D0F888605A
:109B90006FF38F0646EA8306C0F88860D0F88860C5
:109BA00003EB490326F4FE0646EA0946C0F888603E
:109BB000D0F8A0606FF38F0646EA8306C0F8A06075
:109BC000D0F8A06005FB0A3326F4FE0646EA0A46F2
:109BD000C0F8A060D0F8B0606FF38F0646EA830645
:109BE000C0F8B060D0F8B06026F4FE0646EA07463A
:109BF000C0F8B060E66CD0F8AC506FF38F0506FB90
:109C000007337E4345EA8305C0F8AC50D4F854804E
:109C100008FB0C35D0F8F0306FF38F0308FB0CFC19
:109C200043EA8503C0F8F030D0F8F0E0A36D2EF4DD
:109C30007C1242EA0342C0F8F02005EB4302D0F860
:109C4000C0506FF38F0545EA8202C0F8C020D0F8FB
:109C5000C020DDF80CB022F47C1242EA0B42C0F8BE
:109C6000C020019AD0F8C05025F07C5502FB0AFEB6
:109C70004AF20002C4F20002DDF810A002EB8101FA
:109C8000029A01F5406145EA0A6501EB8207C0F8D6
:109C9000C05007EBC902A56E02EB8E00626700EBB5
:109CA00086060BFB05F2276706EB8C07C4E91E0648
:109CB0000AFB05F007EBC30303EB8202C4F8843010
:109CC0004DF2FC33E16602EB8000C4F200039842DF
:109CD000C4F88070C4F88820C4F8900004D9D4F87F
:109CE0009C0040F0200058E6814221D20A46002024
:109CF00042F8040BD4F890309A4215D2486001F132
:109D00000802D4F890309A423FBF0020886001F1E9
:109D10000C02D4F8903038BF9A4205D2C860103196
:109D2000D4F890209142E1D305B0BDE8F08F00BF98
:109D3000002005B0BDE8F08FB0B5B6B0044602A86B
:109D4000B8210025CDE93455CDE932553195F7F7E5
:109D5000E4F84DF200412068C4F20001884241D08D
:109D60004AF20041C4F20001884273D04AF2000175
:109D7000C4F20001884240F0BF80002003904FF4FD
:109D8000004002904FF080501D9002A801F0ACFE00
:109D900008B1FBF7F9FE41F2E84144F2E040C2F2BB
:109DA0000041C5F602000A68002A02F101020A60B9
:109DB00008D1C16841F48071C160C16801F480714B
:109DC000019101990168152441F0080101600068C2
:109DD000132500F00800019001980320319009211B
:109DE00033E000BF4FF4004002904FF080501D90D0
:109DF00002A8039501F078FE08B1FBF7C5FE41F219
:109E0000E84144F2E040C2F20041C5F602000A68AF
:109E1000002A02F101020A6008D1C16841F4807190
:109E2000C160C16801F48071019101990168A024A9
:109E300041F00801016000689F2500F008000190D2
:109E4000052101984FF44050319040F60040C5F68E
:109E5000020038E0002003904FF4004002904FF0E1
:109E600080501D9002A801F03FFE08B1FBF78CFE68
:109E700041F2E84144F2E040C2F20041C5F602007E
:109E80000A68002A02F101020A6008D1C16841F49F
:109E90008071C160C16801F480710191019901680C
:109EA000162441F0020101600068142500F0020050
:109EB000019001986020319040F60040C5F6020004
:109EC0000921A0F50060359131A9022232920022C9
:109ED000CDE9332200F080F905210022284600F068
:109EE00057FB284600F044FB05210022204600F0E5
:109EF0004FFB204600F03CFB36B0B0BD0000000038
:109F0000704700000000000010B34AF20001006832
:109F1000C4F2000188420FD04DF20041C4F20001AA
:109F200088420BD04AF20041C4F20001884218BFB7
:109F30007047012003E000BF002000E0022041F252
:109F4000F011C2F2004101EB4010C06900B10047BE
:109F5000704700000000000010B34AF200010068E2
:109F6000C4F2000188420FD04DF20041C4F200015A
:109F700088420BD04AF20041C4F20001884218BF67
:109F80007047012003E000BF002000E0022041F202
:109F9000F011C2F2004101EB4010406A00B10047ED
:109FA000704700000000000090F8981001290DD1C2
:109FB000022180F8981001688A6922F001028A6102
:109FC0000021C0F89C100846704700BFD0F89C10D4
:109FD00041F00401C0F89C1001207047000000000F
:109FE0007047000000000000704700000000000003
:109FF00070470000000000007047000000000000F3
:10A0000070470000000000007047000000000000E2
:10A0100010B34AF200010068C4F2000188420FD078
:10A020004DF20041C4F2000188420BD04AF20041D7
:10A03000C4F20001884218BF7047012003E000BF4E
:10A04000002000E0022041F2F011C2F2004101EBD9
:10A050004010806900B10047704700000000000018
:10A0600010B34AF200010068C4F2000188420FD028
:10A070004DF20041C4F2000188420BD04AF2004187
:10A08000C4F20001884218BF7047012003E000BFFE
:10A09000002000E0022041F2F011C2F2004101EB89
:10A0A0004010406900B10047704700000000000008
:10A0B00010B34AF200010068C4F2000188420FD0D8
:10A0C0004DF20041C4F2000188420BD04AF2004137
:10A0D000C4F20001884218BF7047012003E000BFAE
:10A0E000002000E0022041F2F011C2F2004101EB39
:10A0F0004010006900B100477047000000000000F8
:10A100007047000000000000B0B541F2A8450446C9
:10A11000C007C2F2004502D0286800B18047A007FE
:10A1200002D5686800B18047600702D5A86800B111
:10A130008047200702D5E86800B18047E00602D5D5
:10A14000286900B18047A00602D5686900B1804740
:10A15000600602D5A86900B18047200602D5E869EB
:10A1600000B18047E00502D5286A00B18047A0050C
:10A1700002D5686A00B18047600502D5A86A00B1BF
:10A180008047200502D5E86A00B18047E00402D587
:10A19000286B00B18047A00402D5686B00B18047EE
:10A1A000600402D5A86B00B18047200406D5E86B97
:10A1B000002808BFB0BDBDE8B0400047B0BD0000FA
:10A1C0008821C5F600010A68024208BF704708608E
:10A1D000FFF79ABF000000002DE9F04F85B00D6831
:10A1E0000290002D00F0E68002988E4600F1264293
:10A1F0000A2102F1FF7342F20042C5F60202002476
:10A2000090424FEAB32208BF0921082A4FF0010704
:10A2100038BF4FEAB32100264FF000080091CDF877
:10A220000CE00DE0DEF8005008F1010835FA07F007
:10A2300006F1020607F1010704F1040400F0BA80F8
:10A24000A7F1010A012000FA0AF315EA0309E9D08F
:10A25000DEF804B00BF003056A1E012A22D802982A
:10A260004FEA4801D0F808C00191032101FA06F233
:10A2700003992CEA020CD1F80CE00EFA06F1DDF895
:10A280000CE041EA0C01816041686FEA020CCBF3FB
:10A29000001299430346019802FA0AF211435960E9
:10A2A0000CE000BF0320032D00FA06F0029B6FEACA
:10A2B000000C304602D13046032526E0D968DEF88E
:10A2C000082001EA0C018240022D41EA0201D96016
:10A2D0001BD102466FF0030000EA5A010F20194417
:10A2E00004F01C0300FA03F51046D1F820E0039AAD
:10A2F0002EEA0505DDF80CE012699A40029B2A431C
:10A300000A62DEF804B00BF00305196805FA00F0E4
:10A3100001EA0C011BF4403F40EA010018603FF4E1
:10A3200081AF44F2F44140F20845C5F60201C5F69A
:10A3300000050F23086840F002000860086800F07C
:10A34000020004902AF00300049904F00C01425921
:10A350008B409A43009B03FA01F1114341514FF0A6
:10A36000B0452868DEF8041040EA0902CB0258BF65
:10A3700020EA09028B022A6040F20405C5F60005B6
:10A38000286840EA090258BF20EA09028B032A60C4
:10A39000D5F8800040EA090258BF20EA0902C90343
:10A3A000C5F88020E86F40EA090258BF20EA090298
:10A3B000EA6737E705B0BDE8F08F00000000000055
:10A3C0000069084018BF012070470000000000002D
:10A3D000002A08BF090481617047000000000000E6
:10A3E00045F6A060C2F2014000687047000000001E
:10A3F00040F2040045F6A061C2F20040C2F2014101
:10A4000000780A68104408607047000000000000EF
:10A4100080B5032000F0ECF802F0A6FA44F21841EF
:10A420004DF69053C5F60201C0F601030A680968AB
:10A4300001F00F01C2F30322595C9A5C01F01F0185
:10A4400002F01F02D04040F21002C2F2004220FA95
:10A4500001F1116040F20C01C2F2004108600F20CE
:10A4600000F00AF800281CBF012080BD00F054F85D
:10A47000002080BD00000000B0B58AB00F283ED893
:10A480000446A12000222146002500F081F8A120E9
:10A4900000F06EF840F20800C2F20040046044F29E
:10A4A000EC40C5F60200016841F08071016000686F
:10A4B00001A900F080700290029802A802F0A0F9B1
:10A4C00002F022FA4DF683614000C4F21B314EF2D5
:10A4D0000002A0FB010142F6D430C2F200404FF06E
:10A4E000FF33C4F20002026003EB9141C0E90115A1
:10A4F00040F2E731C0E9031503F096FF10B10120E7
:10A500000AB0B0BD42F6D430C2F2004003F0C0FF42
:10A510000AB0B0BD0000000081B044F2F440002257
:10A52000C5F60200016841F00201016000680F21D8
:10A5300000F0020000906FF00100009B01B000F0FD
:10A5400027B8000000000000002848BF70474EF206
:10A55000801300F01F014009CEF20003012202FA2D
:10A5600001F143F82010BFF34F8FBFF36F8F704797
:10A57000002848BF704700F01F01012202FA01F1D4
:10A580004EF200124009CEF2000242F8201070474D
:10A5900070B54EF60C5C4FF0FF36CEF2000C00F1B9
:10A5A0006045DCF80030C3F3022E8EF00703042B65
:10A5B00028BF0423BEF1030406FA03F321EA0301D2
:10A5C00000F00F0338BF0024043BB0F1FF3F6344A9
:10A5D00006FA04F003F10C0301FA04F1C8BF05F513
:10A5E000644322EA000008430001187070BD0000B7
:10A5F0004EF60C514FF6FF03CEF200010A681A40E6
:10A6000060F30A2242F0806040F0FD7008607047FD
:10A610002DE9F04F8EB04BF204430022C5F2002327
:10A620000492CDE90222059245F200090692C5F294
:10A630000029D0F800E01A68BEEB090C02F0030014
:10A6400018BF4FF0010C012876D10120029002F0D2
:10A650003000102875D002F44070B0F5807F01D131
:10A660000120049002F4A02040F20108B0F5803FE0
:10A67000C0F200186ED19003404658BF4FF0011051
:10A68000059002F0A060B0F1807F68D05A6802F0B7
:10A69000030001286ED10220029002F03000102841
:10A6A0006CD002F44070B0F5807F01D1022004909C
:10A6B00002F4A020B0F5803F40F20200C0F2010099
:10A6C00005D19503054648BF08F10105059502F03F
:10A6D000A065B5F1807F05D19201024648BF08F11F
:10A6E0000102069200250C95CDE90A55CDE90855E1
:10A6F00053F8042C1E68D2074FF4007204BF40F2D6
:10A700002222C0F20442F70705D086EA0207BF07FB
:10A710003CD401250895F7063BD586EA0207BF061B
:10A7200037D44FF0010BCDF824B006F44077B7F5DD
:10A73000407F37D134E000BF02F0300010287FF4B2
:10A740008AAF0120039002F44070B0F5807F3FF49F
:10A7500087AF87E702F0A060B0F1807F96D19001CB
:10A76000404658BF4FF0011006905A6802F00300AF
:10A77000012890D002F03000102892D102200390DE
:10A7800002F44070B0F5807F90D091E70025F70685
:10A79000C3D44FF0000B06F44077B7F5407F01D1EA
:10A7A00001270A97F7030DD586EA02077F0309D42C
:10A7B000B70319D44FF0011ACDF82CA0F70118D522
:10A7C00004E000BF4FF0000AF70112D586EA020745
:10A7D0007F010ED4B70141D44FF001140C945F688F
:10A7E000FE070AD10FE000BFCDF82C80C246F7016A
:10A7F000ECD400245F68FE0705D087EA0206B6079E
:10A8000001D402250895FE0607D587EA0206B6069A
:10A8100003D44FF0020BCDF824B007F44076B6F520
:10A82000407F01D102260A96FE0307D587EA020679
:10A83000760303D4BE0319D482460B90FE011BD5C8
:10A840007A40520118D4BA011ED404460C90D9F8AB
:10A850000000C007AEEB090014D01EE0CDF8308038
:10A8600044465F68FE07CED0C7E700BF08F1010A83
:10A87000CDF82CA0FE01E3D4D9F80000C007AEEB60
:10A8800009000AD100220FE008F101040C94D9F864
:10A890000000C007AEEB0900F4D0D9F8002022F088
:10A8A0000102C9F8002001224AF200060192B0FA22
:10A8B00080F7C5F20026D046CA463268CDF800E0DF
:10A8C000D207A646484606D0306820F00100306026
:10A8D0000198023001900CEB4C000DF108097F0942
:10A8E00009EBC006B26803EB820252F804CC2CF4E8
:10A8F000807442F8044C53F8042CD2072AD159F83A
:10A90000300000285BD003EB800050F8042C22F0CC
:10A91000010240F8042C706838B103EB800050F855
:10A92000042C22F0100240F8042CF06840B10122FF
:10A9300022EA000053F8202022F4803243F820203D
:10A940003069E0B3012222EA000053F8202022F00F
:10A95000807232E053F8040C009A524520F0010056
:10A9600043F8040C2BD103EB8500BBF1000F50F82A
:10A97000042C42F0020240F8042C07D003EB8B00B9
:10A9800050F8042C42F0200240F8042CB8F1000FDB
:10A9900008D0012020EA080053F8202042F4802249
:10A9A00043F82020BEF1000F09D00120724620EAB2
:10A9B0000E0053F8202042F0806243F8202007EB7D
:10A9C0004705086859F8356009EBC502B04215D152
:10A9D00048685768B842DDF800E034D1CF68D468E1
:10A9E000A7422FD10F691269974207462BD153F81E
:10A9F000040C40F0010043F8040C57E088689768A5
:10AA0000B84203D15768DDF800E01CE04868576899
:10AA100060B1B8420AD103EB860252F8047C27F0F9
:10AA2000010742F8047CDDF800E016E0C868D4684D
:10AA3000A042DDF800E006D008691269904202D019
:10AA400034E000BF074603EB860050F8042C22F0E8
:10AA5000010240F8042C38463FB103EB800050F867
:10AA6000042C22F0100240F8042C09EBC500826887
:10AA700003EB820252F8047C27F4807742F8047CCE
:10AA8000C26842B1012727EA020253F8227027F474
:10AA9000803743F82270006940B1012222EA0000A9
:10AAA00053F8202022F0807243F8202088684FF469
:10AAB0004072D64503EB800050F8047C08BF4FF489
:10AAC000807227F440773A4440F8042C486953F8E0
:10AAD000042C471EC2F3074297420BD9002753F8B4
:10AAE000042CCFF6FF7722F47F0207EB00401043DF
:10AAF00043F8040C53F8042C086801384AF20005A6
:10AB0000D207C5F2002553F8207027F003022BD19D
:10AB10000327D64508BF01273A4343F82020486859
:10AB200060B103EB80003022D64550F8047C08BFAA
:10AB3000102227F020073A4340F8042CC868C203CB
:10AB40002AD4019ED0B30122D64522EA000053F850
:10AB5000202003EB80044FF0A06022F0E06208BFE9
:10AB60004FF0807028E000BF42F0010243F820203F
:10AB7000486840B103EB8000012750F8042C67F3CC
:10AB8000051240F8042CC868C20329D4A8B34FF0BA
:10AB900080726FF0E06727E00122D64522EA0000CC
:10ABA00003EB800453F820204FF4A02022F4E0228D
:10ABB00008BF4FF48030019E104320600869C10334
:10ABC0002AD4C8B30121D64521EA00004FF0E06144
:10ABD00053F8202022F0E06208BF4FF0407128E0D7
:10ABE0004FF480326FF4E027012626EA000053F884
:10ABF000206037403A4343F820200869C10323D43A
:10AC0000019EC8B10121032221EA000053F820105F
:10AC100062F31A610EE000BF0121D64521EA00006F
:10AC20004FF4E02153F8202008BF4FF4403122F4C4
:10AC3000E022114443F82010F00712D1B00718D4D5
:10AC400000200EB0BDE8F08F0121032221EA0000B0
:10AC500053F8201062F3124143F82010019EF007D0
:10AC6000ECD0DAF8000040F00100CAF80000B007AC
:10AC7000E6D5286840F00100286000200EB0BDE84D
:10AC8000F08F000000000000F0B581B00446FFF72F
:10AC9000A7FB002C00F08980054600206065216D2F
:10ACA00011B101B0F0BD00BF204600F081F820686E
:10ACB00041F28836A6654FF6F40ED4E903C2636903
:10ACC0008168CFF6E00E0027CFF6FF7701EA0E018C
:10ACD00007EB024241EA0C016FF0FF0E676B114374
:10ACE0000EEB03223943E369114319438160C168C4
:10ACF000226A21F4E0211143C160216BA26B42EA78
:10AD000001410161E16B41610168626821F4F85120
:10AD10000EEB022211430160016A890609D500BFCA
:10AD2000FFF75EFB401BB04238D82068016A8906F5
:10AD3000F6D4C168A268D4E9097621F0FF01013F89
:10AD4000A3693943C160022B016821F0400141EA47
:10AD500002010160D0F80811E26A21F0A04141EA45
:10AD6000060141EA0201C0F80811016841F0010141
:10AD7000016003D1816841F002018160E068B0F1B7
:10AD8000806F05D101202065002001B0F0BD00BF1B
:10AD900002202065002001B0F0BD00BF4FF400701C
:10ADA0002065606D40F001006065012001B0F0BDDC
:10ADB0002DE9F04FB5B0044602A80830B0210025B7
:10ADC0003095CDE93355CDE93155F6F7A6F845F282
:10ADD00000012068C5F20021884203D035B0BDE8EB
:10ADE000F08F00BF4FF00070029002A803951595F8
:10ADF00000F07AFE08B1FAF7C7FE44F2E04040F2F4
:10AE00000008C5F60200C5F6020830AC022750F86B
:10AE10000C1C4FF0000941F4001140F80C1C50F8D4
:10AE20000C1C4FF0030B01F400110191019950F833
:10AE30000C1C41F4804140F80C1C50F80C1C4FF0E5
:10AE4000090A01F4804101910199016841F0010171
:10AE50000160016801F0010101910199016841F06F
:10AE600002010160016801F002010191019901688C
:10AE700041F010010160016801F010010191019998
:10AE8000016841F0080101600068214600F00800F7
:10AE9000019001984046CDE93077CDF8C890CDF8C3
:10AEA000CCB0CDF8D0A0FFF797F930A9082081E801
:10AEB000810A0620349040462146FFF78DF930A9DB
:10AEC000012008F58066042581E8810A3046214684
:10AED0003495FFF781F930A82146CDF8D0A080E85D
:10AEE000A00A3046FFF778F930A84FF400652146F4
:10AEF00080E8A00A0B20349008F58050FFF76CF929
:10AF000030A82146CDF8D0A080E8A00A08F540601E
:10AF1000FFF762F935B0BDE8F08F000000000000D7
:10AF200001680122C0F8D824002280F8CC24886966
:10AF300040F000608861486D40F08052002042F08F
:10AF400003024A6570470000F0B581B0002800F0A8
:10AF50002781044690F8950428B9002084F89404C9
:10AF6000204600F035F9032084F8950420680CF0A1
:10AF70002BFDD4E90001267CD4E9022300960CF0D5
:10AF800063FA002840F00981206800210CF024FDBC
:10AF9000002840F002812179002900F0F580A1F11C
:10AFA000010C01F0030EBCF1030F4FF0000345D379
:10AFB00001F0FC0204F19A000126002500F8865CED
:10AFC0006F1C20F86C5C00F8627C20F8487CAF1C99
:10AFD00000F83E7C20F8247CEF1C043500F8856CDA
:10AFE00000F8823CAA4240F87E3C40F87A3C40F8A7
:10AFF000763C00F8616C00F85E3C40F85A3C40F842
:10B00000563C40F8523C00F83D6C00F83A3C40F8A1
:10B01000363C40F8323C40F82E3C00F8196C00F801
:10B020001A7C078000F8163C40F8123C40F80E3CB1
:10B0300040F80A3C00F19000C0D12B46BEF1000F51
:10B040002DD003EBC3000122BEF1010F04EB8005FC
:10B050004FF000006A752B75EB852876C5E907006F
:10B0600068621CD05D1CBEF1020F05EBC50604EB47
:10B07000860672753575F5853076C6E9070070620B
:10B080000DD0981C012300EBC00204EB8202537523
:10B090001075D08500201076C2E907005062BCF11F
:10B0A000030F4FF0000237D301F0FC0004F53471B8
:10B0B000002300BF01F87C3C5F1C01F8587C9F1CFA
:10B0C00001F8347CDF1C043301F87B2C01F8782C68
:10B0D000984241E91D2241F86C2C01F8572C01F8E7
:10B0E000542C41E9142241F8482C01F8332C01F882
:10B0F000302C41E90B2241F8242C01F80F2C01F8E7
:10B10000107C01F80C2C41F8082C41F8042C0A6042
:10B1100001F19001CED11A46BEF1000F34D002EBFE
:10B12000C200BEF1010F04EB80014FF0000081F876
:10B13000550281F8542281F85802C1E99700C1F8FC
:10B14000640221D0511CBEF1020F01EBC10304EBDC
:10B15000830383F8550283F8541283F85802C3E935
:10B160009700C3F864020FD0901C002200EBC001CE
:10B1700004EB810181F8552281F8540281F85822AC
:10B18000C1E99722C1F86422D4E90001277CD4E9FF
:10B19000022300970CF080FA30B1022084F8950465
:10B1A000012001B0F0BD00BF00206074012084F8D0
:10B1B0009504207B012802D12046FFF7B1FE2068CC
:10B1C0000CF05AFA002001B0F0BD000000000000B1
:10B1D00010B5B0B002A9044601F10800B021F5F79E
:10B1E0009CFE00212068C4F20401884202D030B0E5
:10B1F00010BD00BF002003904FF4802002904FF458
:10B200004010239002A800F06FFC08B1FAF7BCFCD4
:10B2100000F03AF844F2D840C5F60200016841F067
:10B2200000710160006800F000700190019830B07A
:10B2300010BD000000000000B0B544F60C05C5F6D6
:10B24000020529684907296806D401F00701081A90
:10B2500018BF0120B0BD00BF21F0070108432860DE
:10B26000FFF7BEF8044600BF55F8080C800407D469
:10B27000FFF7B6F8001BB0F57A7FF5D90120B0BD15
:10B280000020B0BD0000000044F60C00C5F602002E
:10B29000016841F08071016070470000000000000B
:10B2A00080B501F0D9FA44F220414DF69052C5F62E
:10B2B0000201C0F601020968C1F30211515C01F0FC
:10B2C0001F01C84080BD000080B544F2304EC5F675
:10B2D000020E5EF8083C5EF8081CC1F3051C5EF81F
:10B2E000041CBCF1000FDEF8042017D0C2F3CC021E
:10B2F00001F00101514303F00303022B00EE101A89
:10B30000B8EE400A10D0012B12D01BB95EF8301CE9
:10B31000890611D49FED361A1CE000BF0021816020
:10B32000C0E9001180BD00BF9FED301A12E000BFE0
:10B330009FED2D1A0EE000BF5EF8301C49F20002AE
:10B34000C0F2D032C1F3C10122FA01F101EE101AAC
:10B35000B8EE411ADEF800109FED263A6FF35F2138
:10B3600002EE101ADEF80010C1F34621B8EE422AB0
:10B3700000EE032A00EE10CAB7EE003AB8EE400A1B
:10B3800081EE000A32EE031A02EE101AB8EE422ADB
:10B3900020EE010A32EE031A80EE011ABCEEC11A49
:10B3A00080ED001ADEF80010C1F3064101EE101A1C
:10B3B000B8EE411A31EE031A80EE011ABCEEC11A42
:10B3C00080ED011ADEF80010C1F3066101EE101ADB
:10B3D000B8EE411A31EE031A80EE010ABCEEC00A43
:10B3E00010EE101A816080BD0024744A001BB74B18
:10B3F0000024744C0000003980B544F2384EC5F684
:10B40000020E5EF8103C5EF8101CC1F3053C5EF8BD
:10B410000C1CBCF1000FDEF8042015D0C1F30011A4
:10B42000C2F3CC02514300EE101A03F003010229CB
:10B43000B8EE400A0ED089B95EF8381C890611D4DE
:10B440009FED361A1CE000BF00218160C0E90011A9
:10B4500080BD00BF9FED301A12E000BF9FED2D1A96
:10B460000EE000BF5EF8381C49F20002C0F2D03294
:10B47000C1F3C10122FA01F101EE101AB8EE411A2E
:10B48000DEF800109FED263A6FF35F2102EE101AEE
:10B49000DEF80010C1F34621B8EE422A00EE032A7E
:10B4A00000EE10CAB7EE003AB8EE400A81EE000A8C
:10B4B00032EE031A02EE101AB8EE422A20EE010A0A
:10B4C00032EE031A80EE011ABCEEC11A80ED001AAA
:10B4D000DEF80010C1F3064101EE101AB8EE411A71
:10B4E00031EE031A80EE011ABCEEC11A80ED011A8A
:10B4F000DEF80010C1F3066101EE101AB8EE411A31
:10B5000031EE031A80EE010ABCEEC00A10EE101AEA
:10B51000816080BD0024744A001BB74B0024744C2A
:10B52000000000390000000080B544F2404EC5F62E
:10B53000020E5EF8183C5EF8181CC1F3055C5EF85C
:10B54000141CBCF1000FDEF8042015D0C1F300215B
:10B55000C2F3CC02514300EE101A03F0030102299A
:10B56000B8EE400A0ED089B95EF8401C890611D4A5
:10B570009FED361A1CE000BF00218160C0E9001178
:10B5800080BD00BF9FED301A12E000BF9FED2D1A65
:10B590000EE000BF5EF8401C49F20002C0F2D0325B
:10B5A000C1F3C10122FA01F101EE101AB8EE411AFD
:10B5B000DEF800109FED263A6FF35F2102EE101ABD
:10B5C000DEF80010C1F34621B8EE422A00EE032A4D
:10B5D00000EE10CAB7EE003AB8EE400A81EE000A5B
:10B5E00032EE031A02EE101AB8EE422A20EE010AD9
:10B5F00032EE031A80EE011ABCEEC11A80ED001A79
:10B60000DEF80010C1F3064101EE101AB8EE411A3F
:10B6100031EE031A80EE011ABCEEC11A80ED011A58
:10B62000DEF80010C1F3066101EE101AB8EE411AFF
:10B6300031EE031A80EE010ABCEEC00A10EE101AB9
:10B64000816080BD0024744A001BB74B0024744CF9
:10B65000000000390000000010B584B0024641F639
:10B66000FF7300209B1A70EB01032DDA47F6FF737E
:10B670009B1A70EB010380F2798082F400430B4344
:10B6800000F0A08082F480330B4300F0E38082F46A
:10B690000022114340F01E8144F20040C5F6020032
:10B6A000816D01F44031B1F5003F00F01F81B1F52B
:10B6B000803F00F0FD80002940F0E181006800013A
:10B6C00000F17D81DBE100BF40F2FF739B1A70EB5C
:10B6D000010325DB82F480730B4300F0878082F442
:10B6E0008062114340F0F68044F20041C5F6020149
:10B6F000886DC0F34252042A00F2C18148F2000072
:10B70000C0F2BB00DFE812F0060000010601E6000F
:10B710000C0100BF0868800140F1B181E0E000BF8A
:10B7200082F400630B4300F07B8082F4805211436B
:10B7300040F0D08044F20041C5F60201086DC0F32C
:10B740000232042A00F29B8148F20000C0F2BB00E2
:10B75000DFE812F00600F800FE00C000040100BFA0
:10B760000868800140F18B81BAE000BF82F4005389
:10B770000B4300F07B8082F48042114340F0AA80AA
:10B7800044F20044C5F60204A06DC0F3027005281F
:10B7900000F27581DFE810F00600420146014A011F
:10B7A0005001520101F058F8216A4DF69052C0F64E
:10B7B0000102C1F30211515C01F01F01C84004B045
:10B7C00010BD00BF44F20040C5F60200016D01F05B
:10B7D0004051B1F1005F00F07580B1F1805F00F081
:10B7E0007B80002940F04B8160E000BF44F20041C3
:10B7F000C5F60201086D00F00702042A00F23F813D
:10B8000048F20000C0F2BB00DFE802F004BAC064F6
:10B81000C40000BF0868800140F1318160E000BFD2
:10B8200044F20041C5F60201886DC0F30262042AA9
:10B8300000F2258148F20000C0F2BB00DFE802F010
:10B8400004BCC64AD00000BF0868800140F11781DF
:10B8500046E000BF44F20040C5F60200C16C00683B
:10B86000C90319D4800140F10A8139E044F2004053
:10B87000C5F60200016DC1F30241052900F2FF8007
:10B88000DFE811F00600E600F000FA000001140005
:10B8900001F00AF804B010BD000140F1F08001A8E9
:10B8A000FFF7AAFD039804B010BD00BF0068C6E012
:10B8B0000068800040F1E38001A8FFF735FE03989F
:10B8C00004B010BD0068000140F1D98001A8FFF765
:10B8D00093FD029804B010BD0068800140F1CF8054
:10B8E00001A8FFF7F1FC029804B010BDC16C036819
:10B8F00011F04051026840F0CF8013F0040300F0D3
:10B90000CB80C2F3C100D6E00868000140F1B780E7
:10B9100055E000BF0868800040F1B18059E000BFE9
:10B92000C86C0B6810F04052086803D113F0040390
:10B9300040F0BF80B2F1805F61D110F4807040F0C0
:10B94000B1805CE00868000140F1998037E000BFF9
:10B950000868800040F193803BE000BFC86C0B6832
:10B9600010F04052086803D113F0040340F0A180A6
:10B97000B2F1805F43D110F4807040F093803EE0DC
:10B980000868000140F17B8019E000BF0868800072
:10B9900075D51EE0C86C0B6810F04052086803D1E2
:10B9A00013F0040340F08580B2F1805F27D110F4DA
:10B9B000807077D123E000BF086800015FD501A83F
:10B9C000FFF71AFD019804B010BD00BF08688000A1
:10B9D00055D501A8FFF7A8FD019804B010BD00BF20
:10B9E000C86C0B6810F04052086802D113F00403D1
:10B9F0005FD1B2F1805F02D110F4807052D108683B
:10BA000010F400301CBF43F20060C0F26E10B2F1BF
:10BA1000005F18BF002004B010BD00BF2068000107
:10BA20002DD518E02068800029D51EE02068400749
:10BA300025D520683DE000BF206824E0206843F25F
:10BA400000618003C0F26E1101EAE07004B010BD25
:10BA50000068000113D501A8FFF7CEFC029804B0DE
:10BA600010BD00BF0068800009D501A8FFF75CFD8C
:10BA7000029804B010BD00BF0168490718D4002027
:10BA800004B010BD006840F60011C005C0F23D01D1
:10BA900001EAE07004B010BDB1F1805F14D112F47E
:10BAA000807211D040F60010C0F23D0004B010BD0D
:10BAB0000068C0F3C10049F20001C0F2D03121FAA0
:10BAC00000F004B010BD00BF006810F400301CBFCF
:10BAD00043F20060C0F26E10B1F1005F18BF0020A9
:10BAE00004B010BD000000002DE9F0470446C07806
:10BAF00044F22C480007C5F6020833D5606E4FEAC1
:10BB0000305103290CD8DFE801F003111D2600BFD6
:10BB1000D8F8001041F40031C8F800101BE000BF55
:10BB200001266078C0070BD020E000BF04F10800B8
:10BB3000022107F051FF064660B16078C00715D1B9
:10BB4000354646E004F12800022107F0D9FF0646F9
:10BB50000028F2D1606ED8F8241021F44011084377
:10BB6000C8F8240000266078C007E9D0A06D04283A
:10BB70000ED83546DFE800F00412181E1E0000BF84
:10BB8000D8F80000354640F40030C8F8000011E055
:10BB900001250127607840071FD453E004F1080015
:10BBA000002107F019FF04E004F12800002107F04C
:10BBB000A7FF05462F461DB1607840070DD441E030
:10BBC000D8F82400A16D20F0070000250843C8F82C
:10BBD000240037466078400734D5D4F8A4004FEAF3
:10BBE000705005280CD8DFE800F00311171D1D1D4B
:10BBF000D8F8000040F40030C8F8000012E000BFA0
:10BC0000012501266078000720D455E004F10800E2
:10BC1000002107F0E1FE04E004F12800002107F014
:10BC20006FFF05462E461DB1607800070ED443E035
:10BC3000D8F82C00D4F8A41020F4600000250843A4
:10BC4000C8F82C003E466078000735D5D4F8A80027
:10BC50004FEA306005280DD8DFE800F00412181E06
:10BC60001E1E00BFD8F8000040F40030C8F80000E5
:10BC700012E000BF01250127E078800720D44EE0C4
:10BC800004F10800002107F0A7FE04E004F12800F9
:10BC9000002107F035FF05462F461DB1E0788007EB
:10BCA0000ED43CE0D8F82C00D4F8A81020F0E060C6
:10BCB00000250843C8F82C003746E07880072ED5C9
:10BCC000E06C4FEA301003280ED8DFE800F00903DB
:10BCD000130900BFD8F8000040F40030C8F8000095
:10BCE0002E467DB912E000BF012501266078C0060E
:10BCF00019D44CE004F10800022107F06DFE05465E
:10BD00002E461DB16078C0060DD440E0D8F8200062
:10BD1000E16C20F0300000250843C8F820003E46C2
:10BD20006078C00633D5E06D4FEA303004280DD876
:10BD3000DFE800F00412181E1E0000BFD8F8000053
:10BD400040F40030C8F8000012E000BF01250127D0
:10BD5000607880061FD44EE004F10800002107F04F
:10BD60003BFE04E004F12800002107F0C9FE05466F
:10BD70002F461DB1607880060DD43CE0D8F8240031
:10BD8000E16D20F4E04000250843C8F82400374660
:10BD9000607880062FD5206E4FEA3040052809D8FC
:10BDA000DFE800F0040E1404040400BF2E46ADB911
:10BDB00018E000BF01250126607840061FD44FE03F
:10BDC00004F10800012107F007FE04E004F1280057
:10BDD000012107F095FE05462E461DB1607840060C
:10BDE0000DD43DE0D8F82400216E20F4E020002599
:10BDF0000843C8F824003E466078400630D5D4F8A1
:10BE0000AC004FEA3070052808D8DFE800F0030DD9
:10BE1000130303032F46ADB918E000BF0125012726
:10BE20006078000620D442E004F10800012107F008
:10BE3000D3FD04E004F12800012107F061FE05466E
:10BE40002F461DB1607800060ED430E0D8F82C00E3
:10BE5000D4F8AC1020F0E04000250843C8F82C00CE
:10BE600037466078000622D5E06E58B1B0F1005F29
:10BE70000CD0B0F1805F2FD1D8F8000040F4003032
:10BE8000C8F800002E469DB908E000BF04F1080084
:10BE9000012107F0A1FD05462E464DB9D8F8240032
:10BEA000E16E20F0405000250843C8F824003E46CB
:10BEB000E078C00733D0A06C032813D8DFE800F087
:10BEC00008021A08D8F8000040F40030C8F8000052
:10BED000A946BDB91AE000BF01250126E078C007D8
:10BEE000E9D11CE001254FF00109A07840061AD5E0
:10BEF0001CE000BF04F10800022107F06DFD0546BB
:10BF0000A9461DB1A07840060DD50FE0D8F8200055
:10BF1000A16C20F0030000250843C8F82000B146BA
:10BF2000A078400602D44F4618E000BFD8F8D403EA
:10BF300040F48070C8F8D403FEF752FA064600BFFA
:10BF4000D8F8D403C00507D4FEF74AFA801B64284A
:10BF5000F6D90325032701E02F468DB12078C007CD
:10BF600061D0A06F4FEAF00005283BD8DFE800F071
:10BF700004404604040400BF002D2E4646D149E08B
:10BF8000D8F84410D4F8B000414011F4407F11D0EB
:10BF9000D8F84410D8F8442042F48032C8F844203D
:10BFA000D8F8442021F4407122F48032C8F84420AB
:10BFB000C8F84410B0F5807F40F0D082FEF710FA48
:10BFC000064641F2883A0325032700BFD8F844000B
:10BFD000800700F1C182FEF703FA801B5045F5D9B6
:10BFE000BCE700BF01250126207880071FD44CE064
:10BFF00004F10800012107F0EFFC04E004F128003F
:10C00000012107F07DFD05462E461DB120788007F1
:10C010000DD43AE0D8F82800A16F20F038000025B0
:10C020000843C8F828003E46207880072DD5606F69
:10C03000052809D8DFE800F0040E1404040400BF4A
:10C040002F46ADB918E000BF012501272078400731
:10C050001FD44DE004F10800012107F0BDFC04E00D
:10C0600004F12800012107F04BFD05462F461DB1C4
:10C07000207840070DD43BE0D8F82800616F20F00D
:10C08000070000250843C8F82800374620784007F5
:10C090002ED5D4F89000052808D8DFE800F0030D6D
:10C0A000130303032E46ADB918E000BF0126012596
:10C0B0002078800620D451E004F10800012107F027
:10C0C0008BFC04E004F12800012107F019FD05466E
:10C0D0002E461DB1207880060ED43FE0D8F82C0003
:10C0E000D4F8901020F0070000250843C8F82C0071
:10C0F0003E462078800631D5D4F88C004FEA307067
:10C10000052809D8DFE800F0040E1404040400BF79
:10C110002F46ADB918E000BF012701252078400661
:10C1200020D451E004F10800002107F055FC04E0A0
:10C1300004F12800022107F0E3FC05462F461DB15B
:10C14000207840060ED43FE0D8F82800D4F88C10B0
:10C1500020F0E04000250843C8F828003746207842
:10C16000400631D5D4F898004FEAB020052809D808
:10C17000DFE800F0040E1404040400BF2E46ADB93D
:10C1800018E000BF012601252078000620D454E0E5
:10C1900004F10800002107F01FFC04E004F128006E
:10C1A000022107F0ADFC05462E461DB120780006A1
:10C1B0000ED442E0D8F82C00D4F8981020F4E050C7
:10C1C00000250843C8F82C003E462078000634D5E8
:10C1D000D4F89C004FEA703005280FD8DFE800F053
:10C1E00004141A04040400BF2F46E5B120680107B7
:10C1F00027D4C1063ED4000355D475E0012701259C
:10C2000020680107F5D51CE004F10800002107F0C3
:10C21000E3FB04E004F12800022107F071FC05466D
:10C22000002D2F46E2D1D8F82C00D4F89C1020F431
:10C23000604000250843C8F82C00374620680107F5
:10C24000D7D5D4F88010B1F5805F0AD104F1280069
:10C25000022107F055FC002818BF01272068D4F8F8
:10C260008010D8F8282022F440521143C8F8281032
:10C27000C106C0D5D4F89410B1F5807F0AD104F17D
:10C280002800022107F03CFC002818BF0127206885
:10C29000D4F89410D8F82C2022F440721143C8F836
:10C2A0002C10000320D5D4F8A000B0F5003F0FD02B
:10C2B000B0F5803F06D078BB04F10800002107F0FC
:10C2C0008BFB04E004F12800022107F019FC05466D
:10C2D0002E4655B9D8F82C00D4F8A01020F44030E0
:10C2E00000250843C8F82C003E46A07840072BD50F
:10C2F000D4F88400B0F5401F0BD0B0F5001F11D06A
:10C30000B0F5801F2AD1D8F8000040F40030C8F8FA
:10C3100000002F46CDB90DE001260125A078400789
:10C32000E6D411E004F12800012107F0E9FB0546FD
:10C330002F4655B9D8F82800D4F8841020F44010BE
:10C3400000250843C8F828003746A078C0070AD15E
:10C350003E462168880016D533E000BF012701253D
:10C36000A078C007F4D0206DB0F5803F10D018BB86
:10C37000D8F8000040F40030C8F800002E4685B11F
:10C38000216888001DD460688A0326D467E000BF56
:10C3900004F10800022107F01FFB0546002D2E4680
:10C3A000EED1D8F82000216D20F48030002508431C
:10C3B000C8F82000CCE700BF0126012521688800CD
:10C3C000E1D504F12800022107F09AFB002818BFEC
:10C3D0000126D4E900108A0341D5E26F6FF0010312
:10C3E00003EB3223022B0BD34FEA322343B1012B51
:10C3F00040F0AC80D8F8003043F40033C8F8003087
:10C4000035B3CA022ED48A0236D44A003ED4B1F1E2
:10C41000FF3F4BDD090253D4C1075CD1810765D4CE
:10C4200041076ED4010778D4C10600F182808006EE
:10C4300007D504F12800022107F062FB002818BF8D
:10C440000125002D18BF01252846BDE8F08700BF53
:10C45000D8F8283023F440731A43C8F8282035460A
:10C46000CA02D0D5D8F82420236F22F000421A4304
:10C47000C8F824208A02C8D5D8F82420A36E22F058
:10C4800080721A43C8F824204A00C0D558F81C2CE2
:10C4900022F4004248F81C2CD4F8B42058F81C3C74
:10C4A0001A4348F81C2CB1F1FF3FB3DCD8F8202028
:10C4B000636D22F040521A43C8F820200902ABD520
:10C4C000D8F82810D4F8882021F440011143C8F886
:10C4D0002810C107A2D004F10800002107F07CFA5F
:10C4E000002818BF05466068810799D504F1080047
:10C4F000012107F071FA002818BF0546606841075E
:10C5000090D504F10800022107F066FA002818BF50
:10C510000546606801077FF587AF04F12800002118
:10C5200007F0EEFA002818BF05466068C1067FF5DF
:10C530007EAF04F12800012107F0E2FA002818BFBD
:10C540000546606880067FF57CAF72E70125CA0268
:10C550007FF559AF86E700BFD4F8B0004FF6CF7330
:10C5600058F81C2CC0F2FF0300F4407122F47C52F6
:10C5700003EA10136FF31F30B1F5407F08BF1A4371
:10C58000002548F81C2CD8F844100843C8F844008B
:10C59000FFF7C9BC000000002DE9F04381B000287E
:10C5A00000F02A8142F200080446C5F200288946BC
:10C5B000D8F8000000F00F0088420ED2D8F8000032
:10C5C00020F00F0040EA0900C8F80000D8F8000089
:10C5D00000F00F00484540F00F81206844F21847F2
:10C5E0004107C5F602070AD521693A6802F07002D0
:10C5F000914204D93A6822F0700211433960010770
:10C600000AD561697A6802F07002914204D97A68A9
:10C6100022F0700211437960C1060AD5A1697A68D7
:10C6200002F4E062914204D97A6822F4E062114394
:10C63000796081060AD5E169BA6802F07002914218
:10C6400004D9BA6822F070021143B96010F00201F7
:10C650000AD0E2683B6803F00F039A4204D93B68B2
:10C6600023F00F031A433A60C20746D0386820F41B
:10C670007061D4E90102012841EA0201396009D060
:10C6800003280DD0022811D157F8181C890340F156
:10C69000B38010E057F8181CC90540F1AD800AE0DE
:10C6A00057F8181C890140F1A78004E057F8181CBE
:10C6B000490740F1A18057F8081C21F00701084301
:10C6C00047F8080CFDF78CFE064641F2883500BF9E
:10C6D00057F8080C616800F03800B0EBC10F09D0C2
:10C6E000FDF77EFE801BA842F2D9032001B0BDE811
:10C6F000F08300BF206800F0020151B1E1683A68A0
:10C7000002F00F02914204D23A6822F00F02114364
:10C710003960D8F8001001F00F0149450DD9D8F85B
:10C72000001021F00F0141EA0901C8F80010D8F803
:10C73000001001F00F0149455ED141070AD521697A
:10C740003A6802F07002914204D23A6822F0700214
:10C750001143396001070AD561697A6802F07002F5
:10C76000914204D27A6822F0700211437960C106C6
:10C770000AD5A1697A6802F4E062914204D27A682B
:10C7800022F4E0621143796080060AD5E069B96855
:10C7900001F07001884204D2B96821F070010843A9
:10C7A000B86000F0E1F839684DF690533A68C0F689
:10C7B0000103C1F3032102F00F02595C9A5C01F0FE
:10C7C0001F0120FA01F102F01F0040F2100221FACD
:10C7D00000F0C2F20042106040F2080040F20C0289
:10C7E000C2F20040C2F200420068116001B0BDE830
:10C7F000F043FDF741BE00BF012001B0BDE8F0836A
:10C800003F22026044F21842C5F6020252F8083C88
:10C8100003F007034360136803F4706383601368D5
:10C8200003F00F03C360136803F0700303615368E0
:10C8300003F070034361536803F4E063836192681B
:10C8400002F07002C26142F20000C5F200200068EE
:10C8500000F00F000860704780B500F085F844F2E2
:10C8600018414DF69053C5F60201C0F601030A685F
:10C87000096801F00F01C2F30322595C9A5C02F0CF
:10C880001F0220FA02F201F01F0040F2100122FA0A
:10C8900000F0C2F20041086040F20C01C2F2004117
:10C8A0000A6080BD0000000080B500F05DF844F231
:10C8B000184C4DF69051C5F6020CC0F60101DCF89B
:10C8C0000020DCF8003003F00F03C2F30322CB5C3E
:10C8D0008A5C02F01F02D04003F01F0240F21003F6
:10C8E00020FA02F2C2F200431A6040F20C03C2F2D4
:10C8F00000431860DCF80400C0F30210085C00F08C
:10C900001F0022FA00F080BD80B500F02DF844F23F
:10C91000184C4DF69051C5F6020CC0F60101DCF83A
:10C920000020DCF8003003F00F03C2F30322CB5CDD
:10C930008A5C02F01F02D04003F01F0240F2100395
:10C9400020FA02F2C2F200431A6040F20C03C2F273
:10C9500000431860DCF80400C0F30220085C00F01B
:10C960001F0022FA00F080BD44F20041C5F602012A
:10C970000869C0F3C200032810D002282CD088BB5D
:10C980000868800649F20000C0F2D03058BF7047F6
:10C990000968C1F3C101C840704700BF8A6A886A4C
:10C9A000C0F3051CC86ABCF1000F4B6B20D0C3F369
:10C9B000CC0300F00100584302F00302022A00EE0B
:10C9C000100AB8EE400A15D0C2B90868800619D41A
:10C9D0009FED281A23E000BF43F20060C0F26E1002
:10C9E000704700BF40F60010C0F23D00704700BF26
:10C9F000002070479FED1E1A11E000BF9FED1B1A2B
:10CA00000DE000BF086849F20002C0F2D032C0F366
:10CA1000C10022FA00F001EE100AB8EE411A086BCC
:10CA20009FED153A6FF35F2002EE100A086BC0F31A
:10CA30004620B8EE422A013000EE032A00EE10CA6A
:10CA4000B7EE003AB8EE400A81EE000A32EE031A61
:10CA500020EE010A01EE100AB8EE411A80EE010A3A
:10CA6000BCEEC00A10EE100A704700BF0024744AE2
:10CA7000001BB74B0024744C00000039000000007C
:10CA800070B586B0002844F2E04640F2000014463B
:10CA90000D46C5F60206C5F602001DD0316800F548
:10CAA000006041F004013160316801F0040101913E
:10CAB00001994FF400710191022102910321049127
:10CAC00000210391059101A9FDF786FB56F8D00CD2
:10CAD000E40120F07E4019E0316841F0010131604D
:10CAE000316801F00101019101994FF480710191C8
:10CAF000022102910321049100210391059101A9D2
:10CB0000FDF76AFB56F8D00C20F0FE7044EA0501F0
:10CB1000084346F8D00C06B070BD000000000000CD
:10CB2000F0B581B0002800F0D5800446007844F2CA
:10CB30000046C007C5F6020622D12078800768D5D6
:10CB4000306910F03801B06A42D0182908BF5FEA96
:10CB500080703DD0E0683168002800F0258121F028
:10CB6000190108433060FDF73BFC0546306840077B
:10CB700048D4FDF735FC401B0228F7D977E100BF08
:10CB8000306900F03801B06A102905D018290BD19E
:10CB900000F00300022807D130688003CDD560681B
:10CBA0000028CAD196E000BF6068002800F03281FA
:10CBB000B0F5A02F00F04681B0F5803F00F046812F
:10CBC000306820F480303060306820F4802040E10C
:10CBD00030684007E06801D500287BD0316821F03B
:10CBE000190108433060FDF7FBFB0546306840073C
:10CBF00008D4FDF7F5FB401B02284FF00300F5D9E0
:10CC000001B0F0BD7068216920F0FE4040EA01608B
:10CC100070602078C00619D5306900F03801B06A1C
:10CC2000082906D0182940F0818000F0030001286F
:10CC30007CD13068C00502D5E06980284AD1F0680F
:10CC4000216A20F07C5040EA0160F0602078000703
:10CC500044D42078800655D42078400700F17E80A7
:10CC6000656A9DB3306900F03800182840F01481DF
:10CC7000012DB16A306B2DD001F00302A36A9A42F4
:10CC800028D1C1F30511E26A914223D10146226BFA
:10CC90006FF35F21013A91421CD1C0F34622616BD0
:10CCA00001398A4216D1C0F30642A16B01398A428A
:10CCB00010D1C0F30660E16B013988420AD1706B74
:10CCC000A16CC0F3CC00814240F09C81002001B0F7
:10CCD000F0BD00BF012001B0F0BD00BF60690028B9
:10CCE000706F4FD040F001007067FDF779FB05468B
:10CCF000706F8007ADD4FDF773FB401B0228F7D996
:10CD0000B5E000BFA0690028306871D040F48050C1
:10CD10003060FDF765FB0546306880049CD4FDF764
:10CD20005FFB401B0228F7D9A1E000BFE0690028A3
:10CD3000306800F09F8040F080003060FDF750FBCD
:10CD4000054600BF3068C0053FF579AFFDF748FBE9
:10CD5000401B02284FF00300F4D951E7D6F8000435
:10CD600040F48070C6F80004FDF73AFB054600BFAA
:10CD7000D6F80004C00529D4FDF732FB401B642817
:10CD8000F6D974E020F001007067FDF729FB054635
:10CD9000706F80077FF55DAFFDF722FB401B022817
:10CDA0004FF00300F4D92BE721F001003060FDF7CC
:10CDB00017FB0546306840077FF52BAFFDF710FBEA
:10CDC000401B02284FF00300F4D919E7A06800289F
:10CDD00000F08480052800F09B80012800F09C80F2
:10CDE000306F20F001003067306F20F0040096E0D3
:10CDF00020F480503060FDF7F3FA05463068800477
:10CE00007FF52AAFFDF7ECFA401B02284FF0030034
:10CE1000F4D9F5E6306820F480303060306820F4D2
:10CE200080203060FDF7DCFA054600BF30688003E3
:10CE30007FF583AEFDF7D4FA401B64284FF0030062
:10CE4000F4D9DDE6306840F480203060306840F48A
:10CE500080303060FDF7C4FA054600BF30688003BB
:10CE60003FF56BAEFDF7BCFA401B6428F6D90320F2
:10CE700001B0F0BD20F080003060FDF7B1FA05464A
:10CE80003068C0057FF5E2AEFDF7AAFA401B022824
:10CE90004FF00300F4D9B3E6306820F080703060C2
:10CEA000FDF79EFA022D05460CD100BF30688001C7
:10CEB00048D5FDF795FA401B02284FF00300F5D93D
:10CEC0009EE600BF306880017FF500AFFDF788FA6D
:10CED000401B02284FF00300F4D991E6306F20F098
:10CEE00001003067306F20F004003067FDF778FAFA
:10CEF000054641F28837306F80077FF5B1AEFDF708
:10CF00006FFA401BB8424FF00300F4D978E600BF37
:10CF1000306F40F004003067306F40F00100306740
:10CF2000FDF75EFA054641F2883700BF306F800793
:10CF30003FF596AEFDF754FA401BB8424FF00300A0
:10CF4000F4D95DE604F12807B06A40F2F331884372
:10CF50008ECF0843591E40EA02104FF47E426FF311
:10CF60005F21B06202EB47204FF4FE0280B2E36B18
:10CF70000844A16B02EB01414FF0FE4201F4FE01B7
:10CF800002EB0362084402F0FE4108443063F06A99
:10CF90004FF6F87120F00100F062706BA26C8843CC
:10CFA00040EAC2007063F06A216C20F00C00084374
:10CFB000F062F06A616C20F002000843F062F06AEF
:10CFC00040F48030F062F06A40F40030F062F06AC1
:10CFD00040F48020F062F06A40F00100F0623068B6
:10CFE00040F080703060FDF7FBF904463068800146
:10CFF0003FF56CAEFDF7F4F9001B02284FF003007B
:10D00000F4D9FDE5F06A20F00100F062FDF7E8F9DF
:10D010000546FDF7E5F9A842FBD0706B4FF6F871B5
:10D02000A26C884340EAC2007063F06A40F00100DD
:10D03000F062002001B0F0BDF0B581B0F8B1044657
:10D04000D0F888001E4615460F4628B9002084F8FF
:10D050008400204602F0A0FC2420C4F88800206848
:10D06000A16A0268002922F00101016002D0204675
:10D0700008F056F9204609F0F3F9012802D1012001
:10D0800001B0F0BD2068816841F480418160816811
:10D0900021F40041394381603104026841EA45517D
:10D0A0006FF3194211430160016841F00101016011
:10D0B000204601B0BDE8F04008F0A2B90000000031
:10D0C00043F600010068C4F20001884208D141F231
:10D0D000F040C2F200408069002808BF7047004756
:10D0E00070470000000000002DE9F04381B00446C5
:10D0F000066830697169D6F8089094F88180020753
:10D100000CD511F4006209D0B06940F40060B06140
:10D11000204601B0BDE8F04300F0E2BD01EA0005A1
:10D1200005F06407042F05D1616F20468847216F01
:10D130002046884705F04500012807D1216F204689
:10D14000884705F02600022804D00BE005F02600F1
:10D15000022805D1616F204601B0BDE8F0430847C1
:10D16000042F03D101B0BDE8F08300BF280715D418
:10D1700015F4587FF6D015F0400065D1A80570D49D
:10D18000E80505F020007CD4002840F08880D4F821
:10D190008400002840F09380E4E700BF20688169A4
:10D1A00041F008018161816941F01001816181696B
:10D1B00041F400618161016921F008010161806829
:10D1C00010F4404F27D0204606F036FD012084F8A9
:10D1D0008100D4F88400002840F0AB80B8F1030F40
:10D1E00000F0AE80B8F1040F00F0B080B8F1050F88
:10D1F000B8D1204601B0BDE8F04301F015B800BF3A
:10D200002068616E006B41F8040B6166B4F86A0037
:10D210000138A4F86A00B4F86A000028D3D0E068A6
:10D220001028EDD2082805D3308E616E21F8020B4C
:10D23000EBE700BF206890F83000616E0870606E08
:10D2400001306066E2E700BF2068D4F8841041F046
:10D250000401C4F88410816941F040018161A8058E
:10D260008ED52068D4F8841041F00101C4F88410F0
:10D27000816941F400718161E80505F020007FF5C6
:10D2800083AF2168D4F8842042F00802C4F88420D7
:10D290008A6942F480728A6100283FF478AF20687E
:10D2A000D4F8841041F08001C4F88410816941F001
:10D2B00020018161D4F8840000283FF453AF206836
:10D2C00009F4404240F26B33B2F5404F016821F05F
:10D2D00001010160016921EA0301016126D1816830
:10D2E00043F6095521F440418160E06FC0F6010525
:10D2F00048B10565FAF728FC28B1D4F8840040F05D
:10D300004000C4F88400A06F00283FF42BAF0565EF
:10D31000FAF71AFC00283FF425AFD4F8840040F057
:10D320004000C4F8840001B0BDE8F083012084F817
:10D330008100204601B0BDE8F043FFF7C1BE00BF49
:10D34000204601B0BDE8F04300F046BF204601B0E2
:10D35000BDE8F04300F09CBC2DE9F047002858D010
:10D3600043F6000304460068C4F2000343F2000ED3
:10D3700043F6004C9842C4F2010EC4F2000C4FF088
:10D380000001A16203D0604518BF70453ED1E16B3A
:10D390000122E568984202EB511105F108024FEABB
:10D3A000D20202FB01F118BF704525D1102930D8F7
:10D3B00094F8811031B9002084F88000204600F0F4
:10D3C0009FF82068022184F88110016821F0010192
:10D3D00001608168D4F81880B8F1806F01F4F81EFC
:10D3E000D4F804A020D1BAF1000F15D0BAF5800FFF
:10D3F0001AD1A36B03BB13E0604518BF082908D8F6
:10D40000704518BF6045D1D0D2E700BFE1680F2951
:10D41000BDD90120BDE8F087A36BB3F1805F06D1D1
:10D42000036843F4805303605FEA4A2304D4D4F8CA
:10D430000C904FF0010C0FE0D4F80C90B9F1070FED
:10D4400008D3056825F4807C256D45EA0C054FF06E
:10D45000000C04E04FF0000C056825F480750560B1
:10D46000BAF1000FE769A26A47EA0E07E36B42EAE6
:10D470000702A56842EA03022669676942EA0902CF
:10D4800082604AEA0803626B616A42EA0302A36BA4
:10D4900041EA020141EA0301226A41EA0601E36C22
:10D4A00041EA070141EA0201A26C41EA0301A36DCE
:10D4B00041EA050141EA020141EA0301C16009D1E3
:10D4C0008168012262F3CC2181608168022262F3CB
:10D4D0004A218160016DBCF1000F21F0010101655D
:10D4E00005D1C168626D21F000411143C160002087
:10D4F000C4F88400012184F88110BDE8F0870000A1
:10D500002DE9F04FB5B0044602A8B8210025CDE9B9
:10D510003355CDE931553095F3F7FFFC43F6000163
:10D520002068C4F20001884256D043F20001C4F2E0
:10D530000101884240F0DF804FF48050029002A841
:10D540004FF00008CDF80C80CDF86480FEF7CCFADF
:10D5500008B1F8F719FB44F2E04040F20044C5F688
:10D560000200C5F6020430AD4FF00209016903263E
:10D5700041F4805101610169052701F48051019155
:10D580000199016841F008010160016801F008019A
:10D5900001910199016841F002010160006829468A
:10D5A00000F00200019001988020309004F50060A6
:10D5B000CDE9319833963497FCF70EFE08202946C2
:10D5C000CDE9300920463497CDE93286FCF704FED8
:10D5D00035B0BDE8F08F00BF4FF48050029002A834
:10D5E00003951995FEF780FA08B1F8F7CDFA44F2E1
:10D5F000E04040F20045C5F60200C5F6020530AE37
:10D6000040F228088168C4F2020841F48041816038
:10D6100081684FF0020901F480410191019901688C
:10D6200041F0040101600168002701F0040101914B
:10D630000199016841F0020101600068314600F083
:10D640000200019001980620309005F58060CDF829
:10D65000C4904FF0030A32974FF0050BCDF8CCA0E1
:10D66000CDF8D0B0FCF7B8FD4FF400503146CDE90D
:10D67000300932A880E8800C2846FCF7ADFD42F264
:10D6800068052720C2F200454FF48066C5E901070E
:10D690002846C5F80080EF60C5E90467C5E906774C
:10D6A000C5E90877FAF7D0FF08B1F8F76DFAE56732
:10D6B00008F11800AC6342F2E005C2F200452860B0
:10D6C000282068604020C5E902072846C5E90467AC
:10D6D000C5E90677C5E90877FAF7B6FF08B1F8F7A4
:10D6E00053FA242005210022A567AC63FCF750FF04
:10D6F0002420FCF73DFF35B0BDE8F08F00000000AE
:10D700002DE9F04F81B0994617460E460446D0F8F1
:10D7100000A0C56BFCF764FE94F8811001290DD1BF
:10D7200080460120002E18BF002F03D101B0BDE8B4
:10D73000F08F00BF94F88000012803D1022001B0CF
:10D74000BDE8F08FA346012084F88000042084F80F
:10D7500081000020C4F884004BF8646F2646A4F8CA
:10D76000687026F86A7FE065A4F86000A4F862009B
:10D77000A168B1F5C02FC4E91C00206804D101687C
:10D7800021F40061016004E0C168022262F35241A9
:10D79000C16041684FF6FF729143394441600168AE
:10D7A00041F0010101606168B1F5800F4FF00101A6
:10D7B00003D1026842F400720260E36801EB551184
:10D7C000102B4BD33288002A00F085818DB219F1DD
:10D7D000010225D041694269D20704D13288090487
:10D7E0000CD5AA420AD2016BDBF8000001600430BC
:10D7F000CBF8000030880138308006E0FCF7F0FDFF
:10D80000A0EB0800484580F0C7803088002800F071
:10D810006281206841694269D207DFD0E3E700BF37
:10D8200041694269D20704D1328809040ED5AA425F
:10D830000CD2006BDBF8001041F8040BCBF80010A1
:10D84000308801383080308830B944E1FCF7C8FDB9
:10D850003088002800F03F812068E1E73288072BFC
:10D8600044D9002A00F0378119F1010200F0A880A4
:10D870008FB24FF6FF72551E41694069C00716D13D
:10D8800030880A040ED5B8420CD2BAF83010DBF852
:10D89000000020F8041BBAF8301020F8021C2946BA
:10D8A0000DE000BF3088890418D5012816D1BAF8D8
:10D8B0003010DBF8000020F8021B4FF6FF71CBF8A8
:10D8C00000003088084430803088002800F0038150
:10D8D000206841694069C007D2D0E8E7FCF780FDC5
:10D8E000A0EB08004845EFD356E000BF002A00F047
:10D8F000F28019F1010200F09F808FB24FF6FF72A3
:10D90000A2F1030A41694269D20725D132880B048A
:10D910001CD5BA421AD290F83000616E08702068A7
:10D92000616E4A1C626690F8300048702068616E33
:10D930004A1C626690F8300048702068616E4A1C8C
:10D94000626690F83000487050460CE0328811F45E
:10D95000C04F1BD0032A19D890F83000DBF8001014
:10D9600008704FF6FF70DBF800100131CBF80010A3
:10D970003188084430803088002800F0AC8020686E
:10D9800041694269D207C1D0E6E700BFFCF728FD34
:10D99000A0EB08004845EED3204606F04DF9D4F838
:10D9A000840040F48070C4F88400012084F8810071
:10D9B000002084F88000032001B0BDE8F08F00BF94
:10D9C0008DB241694069C0071BD130880A0413D564
:10D9D000A84211D2BAF83000DBF8001021F8040B8D
:10D9E000BAF83000CBF8001021F8020C3088023869
:10D9F0003080308898B96EE03088890416D50128C7
:10DA000014D1BAF83000DBF8001021F8020BCBF883
:10DA10000010308801383080308800285BD02068C2
:10DA200041694069C007D0D0EBE700BFFCF7D8FCE4
:10DA300030880028F3D14EE08FB241694269D207A5
:10DA40002ED132880B0425D5BA4223D290F830006B
:10DA5000616E08702068616E4A1C626690F8300042
:10DA600048702068616E4A1C626690F83000487009
:10DA70002068616E4A1C626690F830004870606EE3
:10DA800001306066B4F86A000438A4F86A0030888F
:10DA9000A8B920E0328811F4C04F17D0032A15D856
:10DAA00090F83000DBF800100870DBF8000001305F
:10DAB000CBF80000308801383080308858B12068B9
:10DAC00041694269D207BCD0EAE700BFFCF788FC95
:10DAD00030880028F3D1204606F0AEF8012084F803
:10DAE0008100002084F88000D4F88400002818BF4A
:10DAF000012001B0BDE8F08F70B5044690F88100B8
:10DB000001280BD115460A4604F1800601200029A0
:10DB100018BF002D08D10021317070BD04F18006BE
:10DB200002200021317070BD3078012802D102201E
:10DB300070BD00BF012084F88000042084F88100BB
:10DB40000020C4F884006266A4F86850A4F86A5003
:10DB5000C4E91C00A4F86000A4F86200A068B0F555
:10DB6000C02F21681AD1086820F400600860E068BE
:10DB700010281BD2082829D3E06F8069B0F5005F18
:10DB800018BFB0F5804F1DD1886820F480408860B0
:10DB9000E06F8369B3F5804F24D02FE0C86802237B
:10DBA00063F35240C860E0681028E3D3E06F8069F7
:10DBB000B0F5804F06D1886820F480408860E06F1F
:10DBC0001CE000BF01200021317070BD886820F486
:10DBD00080408860E06F8369B3F5804F08D0B3F56B
:10DBE000005F0BD1B4F86A3001335B0804E000BF7A
:10DBF000B4F86A3003339B08A4F86A3043F66153E3
:10DC000043F6515CC0F60103C0F6010CC0E90F3CBD
:10DC100043F621533031C0F60103C364002303658A
:10DC2000B4F86A30FBF754F860B1D4F8840040F0DF
:10DC30001000C4F88400012084F8810000213170B4
:10DC400070BD00BFE16FD4E90002C9694FF6FF74EF
:10DC50004368B1F5807F23EA040318BF2B44B2F573
:10DC6000800F4360816841F480418160016941F423
:10DC700050710161016841F00101016003D1016847
:10DC800041F40071016000200021317070BD00007E
:10DC900043F600010068C4F20001884208D141F255
:10DCA000F040C2F200404068002808BF70470047BB
:10DCB000704700000000000043F600010068C4F255
:10DCC0000001884208D141F2F040C2F200400069F0
:10DCD000002808BF704700477047000000000000A0
:10DCE00070470000000000002DE9F04381B01D46A0
:10DCF00017460E460446D0F80090FCF771FB94F8E6
:10DD0000811001290CD180460120002E18BF002F60
:10DD100002D101B0BDE8F08394F88000012803D15E
:10DD2000022001B0BDE8F083012184F880100320B7
:10DD300084F881000020C4F88400E665A4F86070CF
:10DD4000A4F862706066A4F86800A4F86A00A2688B
:10DD50002067B2F5C02F6067206805D101680346CF
:10DD600041F4006205E000BF034653F80C2F61F355
:10DD700052421A604FF6FF72416891433944416044
:10DD8000016841F0010101606168B1F5800F03D1C4
:10DD9000016841F400710160E268102A3CD3B4F8D4
:10DDA0006210002900F01A81691C1ED041698907A0
:10DDB00006D4FCF715FBA0EB0800A8420AD339E112
:10DDC000E16D51F8042B0262E165B4F8620001389C
:10DDD000A4F86200B4F86200002800F0FF80206818
:10DDE00041698907E5D5EBE720684169890703D4D4
:10DDF000FCF7F6FA0AE000BFE16D51F8042B02626D
:10DE0000E165B4F862000138A4F86200B4F8620079
:10DE10000028E9D1E2E000BFB4F86210072A5DD91A
:10DE2000002900F0DB80691C31D04FF6FE714E1CDA
:10DE30004169890706D4FCF7D3FAA0EB0800A84291
:10DE40001AD3F7E0B4F86210022909D3E16B39B1B3
:10DE5000E16D51F8042B0262E1654FF6FE7006E0B9
:10DE6000E06D30F8021BA9F82010E0653046B4F8E8
:10DE700062100844A4F86200B4F86200002800F0C0
:10DE8000AD80206841698907DCD4D4E72068416906
:10DE9000890703D4FCF7A4FA1BE000BFB4F86210B2
:10DEA00002290BD3E16B49B1E16D51F8042B0262F9
:10DEB000E165B4F86200023809E000BFE06D30F8B7
:10DEC000021BA9F82010E065B4F862000138A4F83C
:10DED0006200B4F862000028D8D17FE0002900F089
:10DEE0007D80691C43D04FF6FE718E1E4F1C416928
:10DEF000890707D4FCF774FAA0EB0800A8422CD3DA
:10DF000098E000BFB4F86210042909D3E16B4029FE
:10DF100006D9E16D51F8042B0262E165304617E045
:10DF2000B4F8621002290BD3E16B49B1E06D30F80F
:10DF3000021BA9F82010E0654FF6FE7008E000BF54
:10DF4000E16D097880F82010E06D0130E065384619
:10DF5000B4F862100844A4F86200B4F86200002823
:10DF60003CD0206841698907CCD4C3E72068416967
:10DF7000890703D4FCF734FA2CE000BFB4F8621030
:10DF800004290BD3E16B412908D3E16D51F8042B2F
:10DF90000262E165B4F86200043819E0B4F8621076
:10DFA00002290BD3E16B49B1E06D30F8021BA9F8EF
:10DFB0002010E065B4F86200023809E0E16D0978EC
:10DFC00080F82010E06D0130E065B4F8620001389F
:10DFD000A4F86200B4F862000028C7D1681C13D00E
:10DFE00020684069000713D4FCF7FAF9A0EB080099
:10DFF000A842F5D3D4F8840040F02000C4F884008F
:10E0000006E000BFFCF7ECF9206840690007F9D58D
:10E01000204605F011FE012084F88100002084F8DC
:10E020008000D4F88400002818BF012001B0BDE8AA
:10E03000F08300BF204605F0FFFDD4F8840040F4D3
:10E040008070C4F88400012084F88100002084F8E6
:10E050008000032001B0BDE8F08300000000000054
:10E06000F0B581B0044690F8810001280CD1002958
:10E070004FF0010000F0AE801546002A00F0AA80A3
:10E0800094F88000012803D1022001B0F0BD00BF48
:10E09000012084F88000032284F881200022C4F843
:10E0A0008420E165A4F86050A4F862506266C4E977
:10E0B0001C22A4F86820A4F86A20A268B2F5C02F38
:10E0C000266813D13068324640F400631360E2687A
:10E0D000102A14D2A06F082A82691BD3B2F5005F00
:10E0E0002AD0B2F5804F1BD00EE000BF324652F866
:10E0F0000C3F60F352431360E268102AEAD3A06F2A
:10E100008269B2F5804F17D0002084F8800001208A
:10E1100001B0F0BDB2F5804F08D0B2F5005F0BD171
:10E12000B4F862200132520804E000BFB4F8622063
:10E1300003329208A4F8622043F6895243F65953F9
:10E14000C0F60102C0F60103C0E90F2343F62152D5
:10E150000027C0F60102C2640765B26822F40042DB
:10E16000B260B4F8623006F12002FAF7B1FD68B18E
:10E17000D4F8840040F01000C4F88400012084F832
:10E18000810084F8807001B0F0BD00BFA16F4FF630
:10E19000FF77D4E90002C9694368B1F5807F23EABB
:10E1A000070318BF2B44B2F5800F4360816841F428
:10E1B00000418160016941F448710161016841F0E9
:10E1C0000101016003D1016841F400710160002088
:10E1D00084F8800001B0F0BD43F600010068C4F28D
:10E1E0000001884208D141F2F040C2F200400068CC
:10E1F000002808BF7047004770470000000000007B
:10E2000043F600010068C4F20001884208D141F2DF
:10E21000F040C2F20040C068002808BF70470047C5
:10E22000704700000000000043F600010068C4F2DF
:10E230000001884208D141F2F040C2F200408068FB
:10E24000002808BF7047004770470000000000002A
:10E2500040F20442C5F60002136823EA00000843B6
:10E2600010607047000000007047000000000000D0
:10E270007047000000000000704700000000000030
:10E28000B0B590F83C20012A02D10220B0BD00BFF9
:10E29000D1E9022323F47C5322F4705242EA0305AD
:10E2A00048F2FF73D1E900CECEF6F0730EEA030216
:10E2B00003F5006445EA020E0CEA04050C6903F557
:10E2C000C05245EA0E0522402A434D692A4303F510
:10E2D00060550C6B03F5F0432A402340134302685A
:10E2E00040F2004C42F48065C4F2010C8C69654533
:10E2F00040F2000CCEF6FF7CCD690CEA044443EA00
:10E30000050343EA040318D14FF6FF7540F2000CF1
:10E31000CDF60F458C6ACDF6F04C03EA050E0D6A7A
:10E320000CEA04544B6A44EA0E0425F0085523F025
:10E3300000532543C96A2B430B430021536480F8E3
:10E340003C100846B0BD0000B0B590F83C20012A52
:10E350004FF0020263D080F83D2040F2004C02688A
:10E36000C4F2010C42F4806363455368D2F808E0BC
:10E3700002BF23F470034C6823434DF6FF740D680D
:10E38000C4F2000423F07003A24243EA0503536081
:10E3900014DC40F2FF73C4F200039A4222DD40F61F
:10E3A0000003C4F200039A422ED040F60043C4F2A8
:10E3B00000039A4228D041F6000321E04FF6FF7394
:10E3C000C4F200039A4213DD0023C4F201039A420F
:10E3D0001AD044F20003C4F201039A4214D06245F9
:10E3E00012D016E0B2F1804F0ED040F2004307E0A9
:10E3F0004EF20003C4F200039A4205D04EF20043ED
:10E40000C4F200039A4204D12EF0800389681943B4
:10E4100091600022012180F83D1080F83C201046D8
:10E42000B0BD00000000000060B310B5044690F8D5
:10E430003D0028B9002084F83C00204600F024F874
:10E44000022084F83D002068211D06F039FA0120E1
:10E4500084F8480084F83E0084F83F0084F84000C7
:10E4600084F8410084F8420084F8430084F84400B2
:10E4700084F8450084F8460084F8470084F83D009D
:10E48000002010BD01207047704700000000000010
:10E4900090F83D10012923D1022180F83D10016838
:10E4A0004DF6FF70C4F200008142C86840F00100E0
:10E4B000C86017DC40F2FF70C4F20000814227DD23
:10E4C00040F60000C4F20000814233D040F6004024
:10E4D000C4F2000081422DD041F6000026E000BFCA
:10E4E000012070474FF6FF70C4F20000814215DD35
:10E4F0000020C4F2010081421CD044F20000C4F2AA
:10E500000100814216D040F20040C4F201000FE049
:10E51000B1F1804F0ED040F2004007E04EF2000013
:10E52000C4F20000814205D04EF20040C4F2000067
:10E5300081420BD107228868C0F20102024000200C
:10E54000062A18BFB2F5803F00D17047086840F036
:10E5500001000860002070477047000000000000C4
:10E56000F0B581B004460068C768066906EA070589
:10E57000A9071BD468072FD4280745D4E8065BD425
:10E58000E80772D117F0800718BF16F402507AD14D
:10E59000002F18BF16F4807040F08280680600F1EA
:10E5A0008980A80600F1908001B0F0BD6FF00201F3
:10E5B0000161012121778069800703D02046FFF7A0
:10E5C000CBFF05E0204600F033F9204600F01CFCAC
:10E5D000002020776807CFD520686FF00401016123
:10E5E00002212177806910F4407F03D02046FFF795
:10E5F000B3FF05E0204600F01BF9204600F004FCC4
:10E60000002020772807B9D520686FF00801016144
:10E6100004212177C069800704D02046FFF79CFFC2
:10E6200006E000BF204600F003F9204600F0ECFBB6
:10E6300000202077E806A3D520686FF01001016163
:10E6400008212177C06910F4407F03D02046FFF7EE
:10E6500083FF05E0204600F0EBF8204600F0D4FBF5
:10E6600000202077E8073FF48DAF20686FF00101AC
:10E670000161204600F028FD17F0800718BF16F44E
:10E6800002503FF485AF20686FF4025101612046CB
:10E69000FFF7EEFD002F18BF16F480703FF47EAF39
:10E6A00020686FF4807101612046FFF7DDFD680688
:10E6B0007FF577AF20686FF040010161204600F0E0
:10E6C0000FFDA8067FF570AF20686FF02001016193
:10E6D000204601B0BDE8F040FFF7CEBD00000000CD
:10E6E00070B586B041F2FF720068C4F200020021EA
:10E6F00090420591CDE90311CDE9011136DCB0F16D
:10E70000804F5BD040F20041C4F20001884240F0EB
:10E710008D8044F2E0400024C5F60200C5F60204F4
:10E7200002250026016841F001010160016801F045
:10E73000010100910099016841F002010160006847
:10E7400001A900F00200009000988020019020466E
:10E750000295CDE903660595FBF73EFDCDE9015530
:10E76000CDE90366059504F580605CE041F60001A3
:10E77000C4F2000188423BD00021C4F2010188426A
:10E7800054D144F2E040C5F60200016841F01001A6
:10E7900001600068002100F010000090C5F6020141
:10E7A00000984FF408500190022002900020CDE91B
:10E7B00003000120059001F5805034E044F2E04070
:10E7C000C5F60200016841F001010160006800F037
:10E7D0000100009000980520019002200290002086
:10E7E000CDE90300012005900020C5F602001AE0E3
:10E7F00044F2E040C5F60200016841F00201016008
:10E800000068002100F00200009000984FF40040E2
:10E81000CDE9031100210190C5F60201022002900A
:10E82000059001F5806001A9FBF7D6FC06B070BD2C
:10E8300070470000000000002DE9F04190F83C30E6
:10E84000012B03D10220BDE8F08100BF4FEAB202E4
:10E85000052A31D8DFE812F0060038007600B4004F
:10E86000DA000001036843F6FF76C4F201061C6A71
:10E87000B3421A6A24F0020422F001021A621A4614
:10E88000D3F804E052F818CF8D6844EA0504D1F8B3
:10E89000008040F3078144F20007C4F20107BB4245
:10E8A00000F00B8144F60007C4F20107BB4200F000
:10E8B000048144F20047FCE00121002280F83C2062
:10E8C0000846BDE8F08100BF036840F2004E43F403
:10E8D0008067C4F2010E1C6A77451A6A24F020048E
:10E8E00022F010021A621A465D6852F818CF8E683C
:10E8F00044EA061407D1CE686FF0400724F0C00444
:10E9000007EA0616344343F6FF76D1F80080C4F2D6
:10E910000106B34240F3EC8044F20007C4F2010761
:10E92000BB4200F0EC8044F60007C4F20107BB4292
:10E9300000F0E58044F20047C4F20107BB4200F05A
:10E94000DE80E4E0036840F2004E43F48067C4F2E6
:10E95000010E1C6A77451A6A24F4007422F480724E
:10E960001A621A465D6852F81CCF8E6844EA062483
:10E9700007D1CE6840F2FF47360224F44064BE431C
:10E98000344343F6FF76D1F80080C4F20106B34267
:10E9900040F3D48044F20007C4F20107BB4200F008
:10E9A000D48044F60007C4F20107BB4200F0CD80DA
:10E9B00044F20047C4F20107BB4200F0C680CCE03D
:10E9C000036843F6FF77C4F20107D3F820C0BB42C7
:10E9D0001A6A22F480521A621A465C6852F81C6F56
:10E9E0000D68D1F808E040F3CF8044F20007C4F28C
:10E9F0000107BB4200F0D38044F60007C4F20107D0
:10EA0000BB4200F0CC8044F20047C4E0036843F608
:10EA1000FF77C4F20107D3F820C0BB421A6A22F480
:10EA200080321A621A465C6852F8546F0D68D1F849
:10EA300008E040F3D38044F20007C4F20107BB4270
:10EA400000F0D78044F60007C4F20107BB4200F093
:10EA5000D08044F20047C8E0036843F6FF77C4F271
:10EA60000107D3F820C0BB421A6A22F480121A624E
:10EA70001A465C6852F8546F0D68D1F808E040F30C
:10EA8000D98044F20007C4F20107BB4200F0DD80E8
:10EA900044F60007C4F20107BB4200F0D68044F2FE
:10EAA0000047CEE00027C4F20107BB4205D040F288
:10EAB0000047C4F20107BB4205D1CF6824F00C0423
:10EAC00027F004073C43B34240F3E28044F20006DF
:10EAD000C4F20106B34200F0E68044F60006C4F238
:10EAE0000106B34200F0DF8044F20046D7E000BFE9
:10EAF0000027C4F20107BB4201D0734507D14F691B
:10EB000025F440658E6945EA870747EA860548F699
:10EB1000FF475D60CFF6FF6707EA0C0747EA082763
:10EB20009F614F6809699F631C629F6947F4006792
:10EB30009F619F6927F480679F61A6E00027C4F268
:10EB40000107BB4201D0734507D14F6925F44055F9
:10EB50008E6945EA071747EA06154FF68C775D6020
:10EB6000CFF6FE7707EA0C0747EA0807DF614F6830
:10EB70000969DF631C62DF6947F00807DF61DF694D
:10EB800027F00407DF61ACE00027C4F20107BB42B5
:10EB900005D040F20047C4F20107BB4204D14F69DF
:10EBA00024F4804444EA871448F6FF475C60CFF6BB
:10EBB000FF673E402CF4005746EA0524DC614E68AE
:10EBC00009691E6447EA0E371F62DF6947F4006770
:10EBD000DF61DF6927F48067DF6156E00027C4F258
:10EBE0000107BB4205D040F20047C4F20107BB4217
:10EBF00004D14F6924F4803444EA07244FF68C771B
:10EC00005C60CFF6FE7703373E402CF4003746EACF
:10EC100005045C654E6809699E6547EA0E471F62F8
:10EC20005F6D47F008075F655F6D27F004075F655C
:10EC300057E000BF0027C4F20107BB4205D040F2F5
:10EC40000047C4F20107BB4204D14F6924F4802479
:10EC500044EA872448F6FF475C60CFF6FF6707F574
:10EC600040773E402CF4001746EA05245C654E6868
:10EC70000969DE6547EA0E571F625F6D47F400675A
:10EC80005F655F6D27F480675F65090229E000BF5B
:10EC90000026C4F20106B34205D040F20046C4F299
:10ECA0000106B34206D12EF44077D1E9056537431A
:10ECB00047EA050E4FF68C75C3F804E0CFF6FE75F3
:10ECC0000CEA050747EA08079F614F6809695F6317
:10ECD0001C629F6947F008079F619F6927F004073E
:10ECE0009F611368194311600021002280F83C20C5
:10ECF0000846BDE8F081000060B310B5044690F806
:10ED00003D0028B9002084F83C00204600F024F89B
:10ED1000022084F83D002068211D05F0D1FD01206E
:10ED200084F8480084F83E0084F83F0084F84000EE
:10ED300084F8410084F8420084F8430084F84400D9
:10ED400084F8450084F8460084F8470084F83D00C4
:10ED5000002010BD0120704781B041F2FF710068B2
:10ED6000C4F20001884217DCB0F1804F2AD040F293
:10ED70000041C4F20001884241D144F2E840C5F6A6
:10ED80000200016841F002010160006800F0020029
:10ED90000090009801B0704741F60001C4F20001F4
:10EDA00088421FD00021C4F20101884227D144F2D9
:10EDB000E840C5F60200816841F001018160806889
:10EDC00009E000BF44F2E840C5F60200016841F0E6
:10EDD00001010160006800F001000090009801B09E
:10EDE000704700BF44F2E840C5F60200016841F0F8
:10EDF00040010160006800F040000090009801B000
:10EE00007047000000000000704700000000000094
:10EE100071B10A1F4FEAB202032A11D8DFE802F0EB
:10EE200002161E2400F13F031B78012B13D120E0B2
:10EE300090F83E20012A0ED1022280F83E2032E0D6
:10EE400000F143031B78012B05D112E000F14003D0
:10EE50001B78012B0DD00120704700BF00F141034A
:10EE60001B78012B05D0F6E700F142031B78012B3C
:10EE7000F1D1032A08D8DFE802F0030B0F1300BF1B
:10EE8000022280F83F200EE0022280F843200AE0B0
:10EE9000022280F8402006E0022280F8412002E0B1
:10EEA000022280F84220026801F01F00012101FACD
:10EEB00000F0116A814311624EF2FF31C4F2000189
:10EEC0008A42116A40EA0100106215DC40F6FF3008
:10EED000C4F20000824227DCB2F1804F4ED040F2F3
:10EEE0000040C4F20000824248D040F60000C4F264
:10EEF0000000824242D053E043F6FF700021C4F28A
:10EF00000100C4F20101824244F20000C4F2010097
:10EF10001EDC4EF20043C4F200039A422ED08A4215
:10EF200024D040F200431DE040F60040C4F200004F
:10EF3000824223D041F60000C4F2000082421DD07C
:10EF40004EF20000C4F20000824217D028E000BF59
:10EF500082420BD044F60003C4F201039A4205D06A
:10EF600044F20043C4F201039A4219D1536C8A421D
:10EF700043F40041516418BF82420BD107219068CD
:10EF8000C0F2010101400020062918BFB1F5803F01
:10EF900006D1704740F20040C4F201008242EDD039
:10EFA000106840F001001060002070470000000071
:10EFB000026801F01F0C012303FA0CFC136A23EA18
:10EFC0000C0343F6FF7CC4F2010C13626245136A22
:10EFD000136213DD44F20003C4F201039A4218D015
:10EFE00044F60003C4F201039A4212D044F20043F3
:10EFF000C4F201039A420CD019E000BF0023C4F20E
:10F0000001039A4205D040F20043C4F201039A4240
:10F010000DD1D2F820C041F211131CEA030F06D122
:10F02000D2F820C040F244431CEA030F12D0D2F8B9
:10F0300020C041F211131CEA030F16D1D2F820C0F0
:10F0400040F244431CEA030F0FD1136823F001037D
:10F0500013600AE0536C23F400435364D2F820C0D9
:10F0600041F211131CEA030FE8D04FEAB101042961
:10F070000AD8DFE801F0030F151B2100012180F8F9
:10F080003E100020704700BF012180F8431000208F
:10F09000704700BF012180F83F100020704700BF7B
:10F0A000012180F840100020704700BF012180F846
:10F0B00041100020704700BF012180F8421000205D
:10F0C00070470000000000004EF200010068C4F22A
:10F0D0000001884218BF7047FBF78AB900000000A2
:10F0E000704700000000000090F88410012901D151
:10F0F000022070472421C0F8881002681368116844
:10F1000023F0005321F001011160002141661360DA
:10F110002022C0F8882080F884100846704700003C
:10F120007047000000000000704700000000000071
:10F1300070B590F88420012A02D1022070BD00BF72
:10F140002422C0F888200268D0F864E0BEF1000FE5
:10F15000D2F800C0136823F001031360936823F012
:10F16000606341EA030191601AD091684EF2980EF3
:10F170009368C0F6010E5B0F4EF2A005C1F3426624
:10F18000C0F601051EF80340E95C2301B3FBF1F171
:10F190001EF80630AE5D1B01B3FBF6F302E000BFC4
:10F1A00001210123A0F86A102021A0F86830C2F8DC
:10F1B00000C0C0F88810002180F88410084670BD97
:10F1C00070B590F88420012A02D1022070BD00BFE2
:10F1D0002422C0F888200268D0F864E0BEF1000F55
:10F1E000D2F800C0136823F001031360936823F082
:10F1F000604341EA030191601AD091684EF2980E83
:10F200009368C0F6010E5B0F4EF2A005C1F3426693
:10F21000C0F601051EF80340E95C2301B3FBF1F1E0
:10F220001EF80630AE5D1B01B3FBF6F302E000BF33
:10F2300001210123A0F86A102021A0F86830C2F84B
:10F2400000C0C0F88810002180F88410084670BD06
:10F250007047000000000000704700000000000040
:10F2600045F200010068C4F20001032301F54042A9
:10F27000904208BF0123401A18BF1846032808BF50
:10F28000704700EBC00041F21051C2F2004101EBA7
:10F290008000006900B100477047000000000000D6
:10F2A000B0B50446006840F62F01C26905681140F8
:10F2B000D0F808E020290BD105F020010EF0805392
:10F2C000C91823D0616FD1B32046BDE8B0400847CC
:10F2D00040F60F010A4219D0012140F22013C1F279
:10F2E0000001C0F200430EEA010C05EA030111EB34
:10F2F0000C010BD0D10718BF15F4807140F0C68106
:10F3000091070EF0010300F1CD81D4E105EA02037B
:10F31000D906E16E14D5012912D11021016281684C
:10F32000490600F19D80B4F85C10B4F85E20B4F892
:10F330005E30002B1CBF891A5FEA01422FD1B0BD9D
:10F34000D10240F159811EF4800100F055814FF443
:10F35000801101622046BDE8B040FFF77DBF00BFCD
:10F36000206850E8000F226820F4907042E8000303
:10F37000002B1FBF206850E8000F226820F4907017
:10F380001CBF42E80003002B12D0206850E8000F99
:10F39000226820F4907042E800034BB1206850E8E6
:10F3A000000F226820F4907042E80003002BD7D1B0
:10F3B0004FF6FE70CEF6FF70226852E8022F2368E7
:10F3C000024043E80225002D1FBF226852E8022FA9
:10F3D000236802401CBF43E80225002D10D022689C
:10F3E00052E8022F2368024043E8022545B1226813
:10F3F00052E8022F2368024043E80225002DDBD1AA
:10F400002020C4F88C000020E0666067206850E887
:10F41000000F226820F0100042E80003002B1FBFFD
:10F42000206850E8000F226820F010001CBF42E85E
:10F430000003002B12D0206850E8000F226820F053
:10F44000100042E800034BB1206850E8000F22682A
:10F4500020F0100042E80003002BD7D189B227E248
:10F46000D4F8803019684A68B4F85CC091B20029B9
:10F4700000F01682614580F01382A4F85E20D969FD
:10F48000B1F5807F00F0AC8050E8000F216820F4D7
:10F49000807041E80002FAB1206850E8000F21684E
:10F4A00020F4807041E80002002A1FBF206850E865
:10F4B000000F216820F480701CBF41E80002002A80
:10F4C0000AD0206850E8000F216820F4807041E8DD
:10F4D00000020AB12068D7E7206850E8020F2168CF
:10F4E00020F0010041E80202002A1FBF206850E816
:10F4F000020F216820F001001CBF41E80202002A2F
:10F5000026D0206850E8020F216820F0010041E871
:10F510000202EAB1206850E8020F216820F00100E1
:10F5200041E80202002AD7D112E000BF206850E86B
:10F53000020F216820F0400041E80202EAB1206891
:10F5400050E8020F216820F0400041E80202A2B119
:10F55000206850E8020F216820F0400041E80202D4
:10F56000002A1FBF206850E8020F216820F04000E9
:10F570001CBF41E80202002AD8D12020C4F88C0028
:10F580000020E066206850E8000F216820F010009D
:10F5900041E80002002A1FBF206850E8000F2168E0
:10F5A00020F010001CBF41E80002002A12D02068A1
:10F5B00050E8000F216820F0100041E800024AB135
:10F5C000206850E8000F216820F0100041E8000298
:10F5D000002AD7D1D4F88000F8F71AF8B4F85CC044
:10F5E00002202067B4F85E00ACEB000081B2204638
:10F5F000BDE8B040FFF794BD11060BD505F0800CB7
:10F600000EF4000111EB0C0104D0A16F00297FF46E
:10F610005BAE94E659060BD4100240F17D8115F0E3
:10F62000804000F079812046BDE8B040FFF710BE71
:10F6300050E8000F216820F0400041E80002002A55
:10F6400000F04681206850E8000F216820F040005B
:10F6500041E80002002A1FBF206850E8000F21681F
:10F6600020F040001CBF41E80002002A00F0308179
:10F67000206850E8000F216820F0400041E80002B7
:10F68000002A00F025812068D2E700BF0121016235
:10F69000D4F8901041F00101C4F8901091070EF0D9
:10F6A000010308D53BB102210162D4F8901041F06A
:10F6B0000401C4F89010510708D53BB10421016240
:10F6C000D4F8901041F00201C4F8901011070CD545
:10F6D00005F0200151EA0C0107D008210162D4F89D
:10F6E000901041F00801C4F8901011050BD515F0E9
:10F6F000806108D04FF400610162D4F8901041F0AD
:10F700002001C4F89010D4F8901000293FF417AEEF
:10F7100012F020010AD005F020010EF08052891865
:10F7200004D0616F11B1204688472068D4F890104A
:10F73000826802F0400201F02801891800F0C080C0
:10F7400050E8000F216820F4907041E80002FAB1FF
:10F75000206850E8000F216820F4907041E8000212
:10F76000002A1FBF206850E8000F216820F4907025
:10F770001CBF41E80002002A0AD0206850E8000FB0
:10F78000216820F4907041E800020AB12068D7E7B0
:10F790004FF6FE70CEF6FF70216851E8021F226816
:10F7A000014042E80213002B1FBF216851E8021FED
:10F7B000226801401CBF42E80213002B10D02168D0
:10F7C00051E8021F2268014042E8021343B1216858
:10F7D00051E8021F2268014042E80213002BDBD1EE
:10F7E000E06E012828D100BF206850E8000F216892
:10F7F00020F0100041E80002002A1FBF206850E8F6
:10F80000000F216820F010001CBF41E80002002A10
:10F8100012D0206850E8000F216820F0100041E865
:10F8200000024AB1206850E8000F216820F0100063
:10F8300041E80002002AD7D12020C4F88C00002122
:10F84000E16620686167816849065FD550E8020F6C
:10F85000216820F0400041E80202002A42D02068DE
:10F8600050E8020F216820F0400041E80202002A1F
:10F870001FBF206850E8020F216820F040001CBF25
:10F8800041E80202002A2DD0206850E8020F2168CA
:10F8900020F0400041E8020222B32068D6E700BF12
:10F8A0008C457FF44CADD869B0F5807F7FF447ADCF
:10F8B000022020672046BDE8B040FFF731BC00BF02
:10F8C0002046FFF7CDFC0020C4F89000B0BD00BF7B
:10F8D0002020C4F888000020A0672046BDE8B04082
:10F8E00000F00ABDD4F8800080B145F27951C0F62D
:10F8F00001010165F8F728F900283FF420ADD4F89C
:10F900008000016DBDE8B040084700BF2046BDE85B
:10F91000B040FFF7A5BC00BFD0017FF510ADB5F139
:10F92000FF3FC8BFB0BD2046BDE8B040FFF7FCBBFD
:10F9300010B5E0B10446D0F8880028B9002084F85A
:10F940008400204600F028F82420C4F888002068AD
:10F95000A16A0268002922F00101016002D020465C
:10F9600005F0DEFC204606F07BFD012802D10120D7
:10F9700010BD00BF2068416821F49041416081685A
:10F9800021F02A018160016841F0010101602046F7
:10F99000BDE8104005F034BD2DE9F043B5B00021BD
:10F9A0000446CDE93311CDE93111309102A8B821D7
:10F9B000F1F7B3FA47F2FF712068C4F20001884200
:10F9C00000F3808044F20041C4F20001884200F05C
:10F9D000CF8044F60001C4F20001884200F0FA80B2
:10F9E00045F20001C4F20001884240F0EA8102A819
:10F9F000002703974FF00208CDF808801F97FCF707
:10FA000073F808B1F6F7C0F844F2E04040F600455C
:10FA1000C5F60200C5F6020530AE4FF00809816850
:10FA200041F480118160816801F480110191019994
:10FA3000016841F004010160016801F004010191D5
:10FA40000199016841F0080101600068314600F049
:10FA50000800019001984FF48050CDE93008A5F5D9
:10FA60008060CDF8D090CDE93277FAF7B5FB04206D
:10FA70003146CDE930082846CDF8D090CDE932772F
:10FA8000FAF7AAFB42F258155820C2F20045C4F218
:10FA9000020028604120C5E901074FF48060EF6053
:10FAA000C5E904072846C5E90677C5E90877F8F7E8
:10FAB000CBFD08B1F6F768F8C4F88050AC63352484
:10FAC00077E100BF47F60001C4F20001884200F070
:10FAD000CD8041F20001C4F20101884200F0FA80B9
:10FAE00041F60041C4F20101884240F06A810120E0
:10FAF000029002A8002603962096FBF7F5FF08B1B6
:10FB0000F6F742F844F2E04030ADC5F602000227B5
:10FB1000016941F080010161016901F080010191F9
:10FB20000199016841F0100101600068294600F068
:10FB300010000190019804203090349040F600406D
:10FB4000C5F60200339600F580642046CDE9317693
:10FB5000FAF742FB08202946CDE930070B20349004
:10FB60002046CDE93266FAF737FB9C2421E100BF3D
:10FB700002A800240394022502951F94FBF7B4FF0A
:10FB800008B1F6F701F844F2E040C5F602008168DA
:10FB900041F400318160816801F4003101910199E3
:10FBA000016841F008010160006830A900F0080018
:10FBB000019001987020CDE930050720349040F67F
:10FBC0000040C5F60200CDE93244FAF705FB2624D1
:10FBD000EFE000BF02A8002603964FF00208CDF820
:10FBE00008801F96FBF780FF08B1F5F7CDFF44F2C0
:10FBF000E04040F60044C5F60200C5F6020430AD10
:10FC00000727816841F480218160816801F48021A7
:10FC100001910199016841F002010160016801F060
:10FC2000020101910199016841F008010160006839
:10FC3000294600F00800019001984FF48040CDE97A
:10FC40003008A4F500603497CDE93266FAF7C4FABB
:10FC50004FF440702946CDE9300820463497CDE96D
:10FC60003266FAF7B9FA2724A3E000BF02A80024FD
:10FC70000394022502951F94FBF736FF08B1F5F7B0
:10FC800083FF44F2E040C5F60200816841F0804104
:10FC90008160816801F0804101910199016841F022
:10FCA00010010160006840F6004100F01000019072
:10FCB000C5F6020101984FF4C070CDE93005072068
:10FCC000349001F5806030A9CDE93244FAF784FA26
:10FCD00052246EE00120029002A80026039620968E
:10FCE000FBF702FF08B1F5F74FFF44F2E04040F2A6
:10FCF0005808C5F60200C4F20208016941F010017B
:10FD00000161016901F0100101910199016841F05F
:10FD100001010160006840F6004100F0010001901F
:10FD2000C5F6020101984FF4C0603090022033966E
:10FD3000CDE9310607203490A1F5406030A9FAF7EB
:10FD40004BFA42F2482508F11800C2F200454FF480
:10FD5000806728602A2068604020C5E9020628469E
:10FD6000C5E90476C5E90666C5E90866F8F76CFCDE
:10FD700008B1F5F709FFE56708F13000AC6342F21E
:10FD8000D015C2F200452860292068600020C5E92E
:10FD90000200C5E90470C5E90600C5E90800284667
:10FDA000F8F752FC08B1F5F7EFFEC4F88050AC63E9
:10FDB0002524052100222046FAF7EAFB2046FAF71F
:10FDC000D7FB35B0BDE8F083B0B50446D0F88C0061
:10FDD000202807D115460A460120002918BF002D0A
:10FDE00002D1B0BD0220B0BD4FF0000CC4F86CC011
:10FDF00040F600402168C5F60000814234D04868D2
:10FE0000000231D551E8000FD4F800E040F08060E6
:10FE10004EE8000141B300BF206850E8000F2168A0
:10FE200040F0806041E80003002B1FBF206850E8CD
:10FE3000000F216840F080601CBF41E80003002BE8
:10FE400012D0206850E8000F216840F0806041E83F
:10FE500000034BB1206850E8000F216840F080603B
:10FE600041E80003002BD7D1A2652220A4F85C5002
:10FE7000C4F890C0C4F88C00D4F88000F0B145F20A
:10FE8000A17145F62113C0F60101C0F60103C0E9D6
:10FE90000F1345F289510023C0F60101C1642168A6
:10FEA000036524312B46F8F713FF38B11020C4F84E
:10FEB00090002020C4F88C000120B0BD206938B328
:10FEC000206850E8000F216840F4807041E800028B
:10FED000002A1FBF206850E8000F216840F480709E
:10FEE0001CBF41E80002002A12D0206850E8000F31
:10FEF000216840F4807041E800024AB1206850E86F
:10FF0000000F216840F4807041E80002002AD7D138
:10FF1000206850E8020F216840F0010041E8020229
:10FF2000002A1FBF206850E8020F216840F001003E
:10FF30001CBF41E80202002A1DD0206850E8020FD1
:10FF4000216840F0010041E80202A2B1206850E8B7
:10FF5000020F216840F0010041E80202002AD7D1D7
:10FF600009E000BF206850E8020F216840F040001F
:10FF700041E80202EAB1206850E8020F216840F02F
:10FF8000400041E80202A2B1206850E8020F216857
:10FF900040F0400041E80202002A1FBF206850E8FC
:10FFA000020F216840F040001CBF41E80202002A15
:10FFB000D8D10020B0BD000080B5D0F88C30202B07
:10FFC00006D10123002918BF002A03D1184680BD9D
:10FFD000022080BD0023C36640F60043D0F800C075
:10FFE000C5F600039C4503D0DCF804301B0205D4A1
:10FFF00006F056FD0023184680BD00BF5CE800CF28
:020000040801F1
:10000000D0F800E04CF080634EE8003CBCF1000FFB
:10001000EED0036853E800CFD0F800E04CF08063E6
:100020004EE8003CBCF1000F1FBF036853E800CF4F
:10003000D0F800E04CF080631CBF4EE8003CBCF1FF
:10004000000FD5D0036853E800CFD0F800E04CF0A3
:1000500080634EE8003CBCF1000FC9D0036853E850
:1000600000CFCDE70000000045F200010068C4F2B7
:100070000001032301F54042904208BF0123401ACA
:1000800018BF1846032808BF704700EBC00041F2B4
:100090001051C2F2004101EB8000C06800B100477E
:1000A000704700000000000045F200010068C4F243
:1000B0000001032301F54042904208BF0123401A8A
:1000C00018BF1846032808BF704700EBC00041F274
:1000D0001051C2F2004101EB8000806800B100477E
:1000E0007047000000000000B0B50446D0F888005A
:1000F000202831D100294FF0010061D0002A134699
:1001000008BFB0BD21650025A4F854302120A4F813
:100110005630C4F89050C4F88800E06FF0B145F252
:10012000895245F6411CC0F60102C264226845F6B8
:10013000012E2832C0F6010CC0F6010E0565C0E99B
:100140000FCEF8F7C5FD48B11020C4F8900020206C
:10015000C4F888000120B0BD0220B0BD2068402155
:10016000016250E8020F216840F0800041E802027D
:1001700042B300BF206850E8020F216840F08000C1
:1001800041E80202F2B1206850E8020F216840F015
:10019000800041E80202AAB1206850E8020F2168FD
:1001A00040F0800041E8020262B1206850E8020F8E
:1001B000216840F0800041E802020020002AD9D1E5
:1001C000B0BD00BF0020B0BDD0F88830202B07D1D3
:1001D0000123002918BF002A04D11846704700BF28
:1001E0000220704701650021A0F85420A0F8562095
:1001F000C0F890102121C0F88810416EB1F1005F65
:10020000816835D1B1F5805F02D10169002963D0E1
:1002100046F6A971C0F601018167016851E8021F25
:10022000026841F4000142E80213002B52D0016839
:1002300051E8021F026841F4000142E80213002B5A
:100240001FBF016851E8021F026841F400011CBF92
:1002500042E80213002B3DD0016851E8021F0268FA
:1002600041F4000142E80213002BD6D132E000BF76
:10027000B1F5805F01D10169A1B346F6D961C0F63D
:1002800001018167016851E8001F026841F08001A7
:1002900042E8001363B3016851E8001F026841F0AF
:1002A000800142E80013002B1FBF016851E8001FC6
:1002B000026841F080011CBF42E80013002B09D006
:1002C000016851E8001F026841F0800142E8001314
:1002D000002BD7D10020704746F6E951C0F6010146
:1002E0009AE700BF46F61951C0F60101C9E700BF01
:1002F000002318467047000045F200010068C4F270
:100300000001032301F54042904208BF0123401A37
:1003100018BF1846032808BF704700EBC00041F221
:100320001051C2F2004101EB8000406800B100476B
:10033000704700000000000045F200010068C4F2B0
:100340000001032301F54042904208BF0123401AF7
:1003500018BF1846032808BF704741F2105100EB40
:10036000C000C2F2004151F8200008B1004700BFB0
:100370007047000000000000FEE7000000000000E1
:1003800010EE100AB6EE001A45F6DF11B7EE083A85
:10039000C5F6377120EE010AA1EB6000B0EE434ACA
:1003A00001EE100A20EE012A02EE414A24EE011A63
:1003B00020EE010A01EE403A21EE030A70470000E8
:1003C000002800F0ED800168002900F0E9809FED31
:1003D000761A80FE410A9FED751A80FE010A80EDB3
:1003E000150A91ED013A91ED004A20EE002A20EE27
:1003F000021A22EE033A01EE043A91ED024A00EEAF
:10040000043A91ED034A34EE033A80ED163A91ED49
:10041000053A91ED044A22EE033A01EE043A91EDD9
:10042000064A00EE043A91ED074A34EE033A80EDB5
:10043000173A91ED093A91ED084A22EE033A01EE9E
:10044000043A91ED0A4A00EE043A91ED0B4A34EE7B
:10045000033A80ED183A91ED0D3A91ED0C4A22EEF7
:10046000033A01EE043A91ED0E4A00EE043A91EDA2
:100470000F4A34EE033A80ED193A91ED113A91EDBD
:10048000104A22EE033A01EE043A91ED124A00EED0
:10049000043A91ED134A34EE033A80ED1A3A91EDA5
:1004A000153A91ED144A22EE033A01EE043A91ED29
:1004B000164A00EE043A91ED174A34EE033A80ED05
:1004C0001B3A91ED193A91ED184A22EE033A01EEEA
:1004D000043A91ED1A4A00EE043A91ED1B4A34EECB
:1004E000033A80ED1C3A91ED1D3A91ED1C4A22EE43
:1004F000033A01EE043A91ED1E4A00EE043A91ED02
:100500001F4A34EE033A80ED1D3A91ED213A91ED08
:10051000204A22EE033A01EE043A91ED224A00EE1F
:10052000043A91ED234A34EE033A80ED1E3A91ED00
:10053000253A91ED244A22EE033A01EE043A91ED78
:10054000264A00EE043A91ED274A34EE033A80ED54
:100550001F3A91ED293A91ED284A22EE033A01EE35
:10056000043A91ED2A4A00EE043A91ED2B4A34EE1A
:10057000033A80ED203A91ED2D3A22EE032A91EDD7
:100580002C3A01EE032A91ED2E1A00EE012A91ED8C
:100590002F0A30EE020A80ED210A002040B2704797
:1005A000FF2040B2704700BFCDCCCC3ECDCCCC3D7F
:1005B00000284BD090F88810002947D090ED170AFA
:1005C00090ED0E1A90ED1D2A20EE010A21EE021A7E
:1005D00090ED162A90ED0D3A90ED1C4A02EE030ABA
:1005E00090ED182A03EE041A90ED0F3A02EE030A7A
:1005F00090ED1E2A03EE021A90ED192A90ED103AA2
:1006000002EE030A90ED1F2A03EE021A90ED1A2A59
:1006100090ED113A02EE030A90ED202A03EE021A41
:1006200090ED1B2A90ED123A02EE030A90ED212A7A
:1006300003EE021AB1EE400A80ED130AB1EE410A50
:1006400080ED140A002040B2704700BFFF2040B286
:100650007047000000000000B0B5044600284FF0CD
:10066000FF0012D00D4681B1201D8821F0F755FC06
:10067000B5EE000A4FF07A50606520462560FFF71E
:100680009FFE012084F88800002040B2B0BD000029
:1006900050B180B504305021F0F73FFC0020BDE898
:1006A000804040B2704700BFFF2040B2704700005A
:1006B000FF22002818BF002902D150B2704700BFA6
:1006C00010B591E80C50D1E90441C26190ED010AE6
:1006D000036290ED021AC0F824C090ED032AC0F81E
:1006E00028E090ED043AC0E90B4190ED076A90EDE7
:1006F000087A30EE460A90ED096A31EE471A90ED1D
:100700000A7A90ED054A90ED065AD0ED0B0AD0ED2D
:100710000C1A80ED0D0A32EE460A80ED0E1A33EE09
:10072000471A80ED0F0A34EE600A80ED101A35EE9C
:10073000611A002280ED110A80ED121ABDE8104006
:1007400050B2704700000000FF22002818BF0029A7
:1007500002D150B2704700BF10B591E80C50D1E9FA
:100760000441426090ED076A836090ED087AC0F81A
:100770000CC0D0ED0B0AC0F810E0D0ED0C1AC0E9A7
:10078000054190ED010A90ED021A90ED032A90EDDB
:10079000043A30EE460A90ED096A31EE471A90EDC0
:1007A0000A7A90ED054A90ED065A80ED0D0A32EE78
:1007B000460A80ED0E1A33EE471A80ED0F0A34EE2A
:1007C000600A80ED101A35EE611A002280ED110AE0
:1007D00080ED121ABDE8104050B2704700000000D2
:1007E00030B3B0EE403A90ED011A90ED062A90ED4C
:1007F000074A80ED072A02EE413A90ED021A04EE14
:10080000413A13EE101A21F00041B1F1FF4F00FE02
:10081000031A90ED030A90ED043A80ED061A20EEDB
:10082000010A02EE030A90ED053A04EE030A70474E
:100830009FED010A704700BF0000000000000000AB
:10084000002808BF704710B50446F5EE400AC0ED19
:10085000000A0020F1EE10FAA061E06132DD80EEC6
:10086000200A9FED201A81EE000A0CF067FE9FED32
:100870001E1AB7EE002A20EE011A20EE004A31EED1
:10088000023A32EE410ABFEE002A34EE031A34EE89
:10089000022A34EE000A84EE013A32EE022A84ED96
:1008A000033A80EE010A84ED053A33EE034A82EE04
:1008B000011A84ED044A84ED011A84ED020ABDE8B0
:1008C000104070474FF07E516061C4E903106060D2
:1008D0009FED030A84ED020ABDE81040704700BF97
:1008E00000000000DB0F4940F304B53F00000000AA
:1008F00080B390ED031A90ED042A31EE023A90EDA8
:10090000054AB0EE406A90ED015A33EE043A80EEAB
:10091000033A13EE101A01F0FF41B1F1FF4F00FE50
:10092000033A80ED073A03EE456A90ED025A03EE72
:10093000456A16EE101A21F00041B1F1FF4F00FE9A
:10094000065A80ED065A21EE050A02EE030A04EE6D
:10095000030A70479FED010A704700BF00000000C6
:1009600010B592B0002841D090F800C0BCF1020F41
:1009700038D841F25851C2F2004151F82C1089B3D5
:1009800091F8842072B30B1D04E000BF013A03F11B
:10099000040327D0D3F800E0BEF1000FF6D09EF894
:1009A00000106145F2D1BEF802104488A142EDD199
:1009B000BEF804006946009008208DF804004FF04E
:1009C000FF30CDF805000290FC208DF80C009EF859
:1009D0000000F2F7E1FD002818BF4FF0FF3040B2F1
:1009E00012B010BDFC2040B212B010BDFE2040B2CB
:1009F00012B010BD00000000B0B518B390F800C0F0
:100A0000BCF1020F1ED841F25851C2F2004151F818
:100A10002C10B9B191F88430A3B101F1040E002279
:100A200003E000BF01329A420ED25EF82210002984
:100A3000F8D00C786445F5D14C884588AC42F1D1AA
:100A40000846B0BD0020B0BD00210846B0BD000082
:100A5000B0B592B0FE22002818BF002902D150B2D2
:100A600012B0B0BD90F800C0BCF1020F00F29C8043
:100A700041F25852C2F2004252F82C20002A00F0F3
:100A8000938092F88430002B00F08E80043204E0D2
:100A9000013B02F1040200F08780D2F800E0BEF1D1
:100AA000000FF5D09EF800406445F1D1BEF8024039
:100AB0004588AC42ECD1B3EE0E2A91ED020A9FEDCF
:100AC0003C1AB2EE084A30EE010A91ED011A31EEFD
:100AD000021A9FED383A9FED392A91ED035A20EE24
:100AE000030A9FED353A21EE021A91ED046A25EED4
:100AF000025AB1EE047A80EE030A9FED313A81EE9C
:100B0000031A91ED003A33EE043A9FED2E4A26EE99
:100B1000026ABEF8040085EE044A009023EE022A21
:100B2000B3EE083A86EE075A0820BDEEC00A8DF8EB
:100B3000040082EE032ABDEEC11ABDEEC43A10EEE7
:100B4000101ABDEEC54ABDEEC22A11EE102A13EEF0
:100B5000103A080A14EE105A8DF8061012EE104AD8
:100B600011018DF8050010098DF8070041EA1320E6
:100B7000210A8DF8080028098DF809308DF80A003F
:100B800041EA05108DF80B0069468DF80C409EF87F
:100B90000000F2F701FD0246002818BF4FF0FF32B7
:100BA00050B212B0B0BD00BFFC2250B212B0B0BD06
:100BB000DA0F494100FF7F47DA0FC94100F07F4556
:100BC000000070420000FA43F0B581B0002841D027
:100BD00006780446022E4FD841F25857C2F2004719
:100BE00057F82600D0B357F82660002E44D096F868
:100BF0008400002846D0002103E000BF0431814278
:100C00003ED206EB810253681BB15B886788BB420A
:100C10001BD04B1C834233D293681BB15B8867881F
:100C2000BB4212D08B1C83422AD2D3681BB15B8893
:100C30006788BB4209D0CB1C834221D21269002AAB
:100C4000DCD0528863889A42D8D1FD2040B201B0EE
:100C5000F0BD00BFFE2040B201B0F0BD8820F2F729
:100C60001BFE47F8260038B188210546F0F755F9F4
:100C70002E702678022EB6D9FF2040B201B0F0BD0A
:100C80001F28F9D83020F2F707FE0028F4D03021D1
:100C90000546F0F742F920686168C5E900010020C7
:100CA00028722078E27961882A760322F1F768FFBA
:100CB00030B12846F2F73CFDFF2040B201B0F0BD54
:100CC00096F8840006EB8001013086F8840000204D
:100CD0004D6040B201B0F0BDF0B595B040B10246F4
:100CE0000078022808D9FC2148B215B0F0BD00BF39
:100CF000FE2148B215B0F0BD41F25851C2F2004198
:100D000051F820C0BCF1000F48D09CF88430002B73
:100D100044D0002404E000BF0434FC219C42E3D210
:100D20000CEB84056F681FB179885688B1421BD0DF
:100D3000611C994232D2AF681FB179885688B1429E
:100D400012D0A11C994229D2EF681FB17988568828
:100D5000B14209D0E11C994220D22F69002FDBD08B
:100D600079885688B142D7D16A460023F1F7ACFDA5
:100D7000C0B1F2F7C1FED7E90423801A48F2A1629C
:100D8000C0F201029941801A71F10000C0F0C680E2
:100D900000203872FF2148B215B0F0BDFC2148B2E6
:100DA00015B0F0BD01203872F2F7A6FEBDF80E2096
:100DB0009FED5C1AC7E9040112049DF81110B3EE0F
:100DC000084ABAEE085A10BA00EE100A9DF8100050
:100DD00001F00F039DF812200001B8EEC00A40EAAE
:100DE000111042EA032102EE100A03EE101A20EE5F
:100DF000010A9FED4D1A9DF81300B8EEC22AB8EE15
:100E0000C33A80EE010A9FED4A1A22EE011A9FEDC5
:100E1000472A23EE043ABBEE0E4A30EE020A9FED5B
:100E2000452A81EE021A87ED070A83EE023AB5EEF3
:100E3000400A31EE042A33EE051A03EE100AF1EEF1
:100E400010FA87ED082AB8EE433A87ED091A87EDC4
:100E50000A3A49DA9FED383A30EE030AB5EE400A15
:100E6000F1EE10FABFBF30EE030AB5EE400AF1EE24
:100E700010FA30EE030ABCBFB5EE400AF1EE10FAEC
:100E800006DA30EE030AB5EE400AF1EE10FAE3DBC3
:100E900087ED070A9FED283AB4EE430AF1EE10FA07
:100EA00029DB9FED264A30EE040AB4EE430AF1EE48
:100EB00010FAA1BF30EE040AB4EE430AF1EE10FAC4
:100EC00030EE040AA4BFB4EE430AF1EE10FA06DBDA
:100ED00030EE040AB4EE430AF1EE10FAE3DA87EDDD
:100EE000070AF87948B914E09FED133AB4EE430AC3
:100EF000F1EE10FAD5DAF87958B133EE400AB1EED6
:100F0000422A87ED070AB1EE410A87ED082A87EDEC
:100F1000090A002148B215B0F0BD00BFFF2148B258
:100F200015B0F0BDDA0FC94100FF7F47DA0F49C1A4
:100F30000000704200F07F45DB0FC940DB0FC9C0E5
:100F4000B0B5E8B3017802293AD841F26452C2F24E
:100F5000004252F821C0BCF1000F31D09CF884E06F
:100F6000BEF1000F2CD0002204E000BF04320021AB
:100F7000724528D20CEB8203596819B14C88458818
:100F8000AC4220D0511C71451CD2996819B14C88D3
:100F90004588AC4217D0911C714511D2D96819B15E
:100FA0004C884588AC420ED0D11C714508D21969D5
:100FB0000029DBD04B884488A342D7D103E000BF8F
:100FC0000020B0BD00210846B0BD000000000000B8
:100FD000D0B180B592B041880078009148F6080100
:100FE000ADF804100021CDF80610CDF809106946BF
:100FF000F2F7D2FA002818BF4FF0FF3012B0BDE868
:10100000804040B2704700BFFE2040B270470000F1
:10101000F0B581B0002841D006780446022E4FD8A2
:1010200041F26457C2F2004757F82600D0B357F890
:101030002660002E44D096F88400002846D0002177
:1010400003E000BF043181423ED206EB81025368C7
:101050001BB15B886788BB421BD04B1C834233D2D9
:1010600093681BB15B886788BB4212D08B1C83429C
:101070002AD2D3681BB15B886788BB4209D0CB1CDE
:10108000834221D21269002ADCD0528863889A42B6
:10109000D8D1FD2040B201B0F0BD00BFFE2040B26B
:1010A00001B0F0BD8820F2F7F7FB47F8260038B111
:1010B00088210546EFF731FF2E702678022EB6D92B
:1010C000FF2040B201B0F0BD1F28F9D83020F2F760
:1010D000E3FB0028F4D00546A0882821A8802068DA
:1010E000286005F10800EFF718FF20786279618821
:1010F0002A760322F1F744FD30B12846F2F718FBB7
:10110000FF2040B201B0F0BD96F8840006EB8001EC
:10111000013086F8840000204D6040B201B0F0BD7F
:101120009FED010A00F004B800000000000000007C
:101130002DE9F04192B048B10146007802280BD960
:10114000FC2250B212B0BDE8F08100BFFE2250B2C6
:1011500012B0BDE8F08100BF41F26452C2F2004219
:1011600052F82030002B63D093F884C0BCF1000FFC
:101170005ED0B7EE001ACCF1000EACF101080025EC
:1011800080FE410ABFEE001A80FE010A04E000BFA3
:101190000435FC22AC45D4D003EB850672681AB145
:1011A00052884F88BA421AD0A84541D0B2681AB1C5
:1011B00052884F88BA4212D00EEB0507BA1C37D0BE
:1011C000F2681AB152884C88A24208D0FA1C2FD07B
:1011D0003269002ADCD052884C88A242D8D14979A1
:1011E000B1EE401A009200294AF2081101914FF025
:1011F000000100FE010A9FED111A8DF80810ADF8EC
:101200000B10694620EE010ABDEEC00A10EE102A4E
:101210008DF80920120A8DF80A20F2F7BDF902466E
:10122000002818BF4FF0FF3250B212B0BDE8F08175
:10123000FC2250B212B0BDE8F08100BF00000045B2
:1012400070B596B040B102460078022808D9FC215A
:1012500048B216B070BD00BFFE2148B216B070BDD6
:1012600041F26451C2F2004151F820C0BCF1000FBC
:1012700041D09CF884E0BEF1000F3CD0002303E095
:101280000433FC217345E3D20CEB83056C681CB17D
:1012900061885688B1421BD0591C71452BD2AC686D
:1012A0001CB161885688B14212D0991C714522D276
:1012B000EC681CB161885688B14209D0D91C7145CF
:1012C00019D22C69002CDBD061885588A942D7D16E
:1012D00001AA0023F1F7F8FA90B1F2F70DFCD4E976
:1012E0000423801A40F2E9329941801A71F100001A
:1012F0004CD300202072FC2148B216B070BD00BF54
:1013000001202072F2F7F8FBC4E90401BDF91300D3
:101310009FED213A9FED1F1A217900EE100ABDF8CA
:1013200017006279022902EE100A9DF91200B8EE48
:10133000C00A4FF00001B8EE422A20EE011A82EEF8
:10134000032A03EE100ABDF9150038BFB0EE410ABA
:101350009FED121A002A22EE012A18BF404284EDA6
:10136000090A002A00EE100A31EE421AB8EEC33A1A
:1013700084ED0A3AB8EEC00A84ED080A02FE010ABA
:1013800084ED070A48B216B070BD00BFFF2148B215
:1013900016B070BD0000043C00FF7F47DB0FC94062
:1013A0002DE9F04141F26458C2F20048D8F80060DB
:1013B000B6B196F8841069B3371D0024002502E009
:1013C00001358D420DD257F825000028F8D0FFF7DF
:1013D00037FF002818BF4FF0FF3496F88410EFE76E
:1013E0000024D8F80460D6B196F88410B9B1371D3E
:1013F000002502E001358D4211D257F82500002862
:10140000F8D0FFF71DFF002818BF4FF0FF3496F803
:101410008410EFE70024D8F80460002EE4D1D8F857
:101420000850ADB195F8841091B12E1D002702E04F
:1014300001378F420CD256F827000028F8D0FFF76A
:10144000FFFE002818BF4FF0FF3495F88410EFE737
:1014500060B2BDE8F0810000E0B180B592B0B0F8B4
:101460000110007801F14071009108218DF80410FD
:101470000021CDF80910CDF805106946F2F778F88B
:10148000002818BF4FF0FF3012B0BDE8804040B2D6
:10149000704700BFFE2040B270470000000000000F
:1014A000B0B5E8B3017802293AD841F27052C2F2DD
:1014B000004252F821C0BCF1000F31D09CF884E00A
:1014C000BEF1000F2CD0002204E000BF0432002146
:1014D000724528D20CEB8203596819B14C784578D3
:1014E000AC4220D0511C71451CD2996819B14C787E
:1014F0004578AC4217D0911C714511D2D96819B109
:101500004C784578AC420ED0D11C714508D219698F
:101510000029DBD04B784478A342D7D103E000BF49
:101520000020B0BD00210846B0BD00000000000052
:10153000C2B200F0F853B3F1007FC0EA024C024699
:1015400008BF0CF10072012918BF0246104670470F
:1015500080B541F23150C0F60100F1F785FB00285B
:1015600018BF4FF0FF3080BD2DE9F04393B0FE224D
:10157000002818BF002903D150B213B0BDE8F08392
:101580000278022A00F2E68041F27053C2F2004370
:1015900053F82290B9F1000F00F0DC8099F884C074
:1015A000BCF1000F00F0D680CCF1000EACF10108C8
:1015B000002503E00435FC22AC45DDD009EB8506AF
:1015C00072681AB157784478A7421DD0A84500F038
:1015D000C180B2681AB154784778BC4214D00EEB7F
:1015E0000507BA1C00F0B680F2681AB15478437847
:1015F0009C4209D0FA1C00F0AD803269002AD9D093
:1016000053784478A342D5D191ED041A037991ED32
:10161000000AB1EE413AB1EE404A002B91ED012AA9
:10162000B3EE046A01FE031A9FED4D3AB1EE425A41
:101630009FED527A00FE040A9FED4D4A81FE431A47
:101640008E6802FE052A9FED475A80FE440ACD6847
:1016500081FE051A9FED475A82FE462A80FE050A42
:10166000BBEE045A31EE031A91ED023AD1E900378C
:1016700030EE040A9FED3C4A82FE052A91ED035AA2
:1016800081EE041A9FED3C4A80EE040A9FED3C4A2D
:1016900032EE062A9FED3C6A83FE443A096985FED4
:1016A000465A936482EE072A9FED367A83FE073A04
:1016B000D76485FE075A9FED2D7A21EE071A16652D
:1016C00083EE043A556585EE064A9165BCEEC11A73
:1016D000417823EE073A007820EE070A22EE072A27
:1016E00011EE102A24EE074ABCEEC33ABCEEC00A43
:1016F000BCEEC22A41EA0221BCEEC44A13EE106AD3
:1017000010EE102A01F1807112EE103A0191F1B23F
:1017100014EE105A52BA23F0FF0742EA03622DBAC0
:1017200045EA0121082541EA1621CDF80D1042EACB
:101730000721CDF8091001A98DF80850F1F718FF1D
:101740000246002818BF4FF0FF3250B213B0BDE878
:10175000F08300BFFC2250B213B0BDE8F08300BF9D
:1017600000007042000070C20000F04200FF7F479E
:10177000B81E4941B81E49C1B81EC94100002042E7
:1017800000409C45000000000000C842000000002E
:10179000F0B581B000283DD006780446022E4BD823
:1017A00041F27057C2F2004757F82600B0B357F81D
:1017B0002660002E40D096F88400002842D00021F8
:1017C00003E000BF043181423AD206EB8102536844
:1017D0001BB15B786778BB422ED04B1C83422FD263
:1017E00093681BB15B786778BB4225D08B1C834222
:1017F00026D2D3681BB15B786778BB421CD0CB1C68
:1018000083421DD21269002ADCD0527863789A4252
:10181000D8D111E0FE2040B201B0F0BD8820F2F72F
:101820003BF847F8260038B188210546EFF775FBED
:101830002E702678022EBAD9FF2040B201B0F0BD3A
:101840001F28F9D86020F2F727F80028F4D00546C1
:10185000A0885421A8802068286005F10800EFF7CF
:101860005CFB61782379A2782B76207842EA01210B
:1018700041EA0241032201F10071F1F781F938B127
:101880002846F1F755FFFF2040B201B0F0BD00BF80
:1018900096F8840006EB8001013086F88400002071
:1018A0004D6040B201B0F0BD42F6E871C2F20041B5
:1018B000FFF75ABE000000002DE9F04381B02DED86
:1018C000108B96B030B181460078022804D9FC27ED
:1018D00055E000BFFE2752E041F27051C2F20041D4
:1018E00051F82010002941D091F88420002A3FD0DF
:1018F000002303E00433FC27934240D201EB83062C
:10190000776827B17D7899F80140A5421ED05F1C09
:1019100097422FD2B76827B17D7899F80140A54248
:1019200014D09F1C974227D2F76827B17D7899F889
:101930000140A5420AD0DF1C97421FD23769002F11
:10194000D8D07D7899F80160B542D3D199F80210CA
:10195000002341EA052242EA014101AA01F1007592
:101960002946F0F7B1FF88B1002708E0FC2706E020
:10197000FC2704E0FC2702E0FC2700E0FC2778B20B
:1019800016B0BDEC108B01B0BDE8F083BBEE04CA0D
:10199000B2EE04FA9FED718A4FF001089FED709A44
:1019A00001AE9FED70AA9FED70BA9FED70DA9FEDCA
:1019B00070EADFED708ADFED709A52E009BAB0EE9E
:1019C0004C3A090C00BA01EE101A000C02EE100A93
:1019D0003879B8EE411A0028BDF81700B8EE422A4F
:1019E00087F8088081EE081A00BA82EE082A4FEACA
:1019F000104001EE0B3AB0EE4E1A05EE100A02EE60
:101A00000D1A38EEC02AB8EE455A00FE020AB1EEB1
:101A1000432A87ED0C0AB1EE414A87ED070A03FE1F
:101A2000022A01FE040A87ED0D2A85EE0F1A87EDC2
:101A30000E0A87ED090A87ED082AB6EEC10A87ED7E
:101A40000F1A87ED0A0AF2F757F8C7E9040199F867
:101A50000000002329463246F0F736FF00287FF4C5
:101A600083AF029A02F0F850B0F1007FEFD1BDF8D9
:101A70001100BDF8131000BA000C00EE100A100A95
:101A800087F84700C2F3004087F84600C2F34040A1
:101A9000B8EE400A87F84500C2F3804087F844005A
:101AA000C2F3C04080EE081AB0EE4A0A87F843003D
:101AB000C2F3005087F84200C2F3405087F841005B
:101AC00001EE090ABDF81500C2F3815287F84020E3
:101AD000B5EE400AF1EE10FA1CDA30EE280AB5EE47
:101AE000400AF1EE10FA15DA30EE280AB5EE400A97
:101AF000F1EE10FABEBF30EE280AB5EE400AF1EE64
:101B000010FA07DA30EE280AB5EE400AF1EE10FAC4
:101B1000E3DB00BFB4EE680AF1EE10FA7FF74EAFD8
:101B200030EE290AB4EE680AF1EE10FAC1BF30EEC9
:101B3000290AB4EE680AF1EE10FA30EE290AC4BFA1
:101B4000B4EE680AF1EE10FA7FF738AF30EE290AEA
:101B5000B4EE680AF1EE10FAE2DC2FE700FF7F47EF
:101B6000B81EC941B81E49C1000020420000F04221
:101B7000000070C2DB0FC940DB0FC9C000000000CD
:101B80002DE9F04141F27058C2F20048D8F80060E7
:101B9000B6B196F8841069B3371D0024002502E021
:101BA00001358D420DD257F825000028F8D0FFF7F7
:101BB00083FE002818BF4FF0FF3496F88410EFE73B
:101BC0000024D8F80460D6B196F88410B9B1371D56
:101BD000002502E001358D4211D257F8250000287A
:101BE000F8D0FFF769FE002818BF4FF0FF3496F8D1
:101BF0008410EFE70024D8F80460002EE4D1D8F870
